:0E0000000C943E0D0C9400000C9400000C9427
:10000E0000000C9400000C9400000C9400000C9462
:10001E0096610C9400000C9400000C948B150C94BB
:10002E0000000C9400000C9400000C9400000C9442
:10003E0000000C9446150C9400000C944C5E0C942D
:10004E0000000C94885E0C9400000C9400000C943C
:10005E0000000C9400000C9400000C9400000C9412
:10006E0000000C9400000C9400000C94F15F0C94B2
:10007E0000000C9434610C9400000C9400000000FD
:10008E000100020004000800100020004000800063
:10009E000001000200040008001000200040008053
:1000AE0000010204081020408000B803C10B80102C
:1000BE000000BC03C10B821F0000C603C10B8103ED
:1000CE000000CE03C10B01040300D803C20B0106CE
:1000DE000500E203C40B01800000EE03CB0B020F00
:1000EE000000F603C50B020F0000FE03C70B020F44
:1000FE00D0120604C90B011000001004190C0110D7
:10010E0000001A04CA0B000100002204CD0B0108E6
:10011E0001002C04CE0B030801003A04CF0B030799
:10012E0000004204E50B017F3F004C04E40B010488
:10013E0000005604D00B030400005E04E30B0164C0
:10014E001E006A04D10B000100007604D20B0001E0
:10015E0000008204E20B010200008E04D30B0001AA
:10016E0000009C04D40B020F0000A804D60B020F53
:10017E00E703B204180C0163000010051A0C0110FD
:10018E0000001A051B0C01020200BE04D80B030866
:10019E000100C404D90B03080000CA04DA0B0308DB
:1001AE000000D004DB0B03080000D604DC0B0308B0
:1001BE000000DC04DD0B03080000E204DE0B030884
:1001CE000000E804E60B040A2E00F004F00B040A0B
:1001DE002E00F804FA0B040A2E000005040C040A83
:1001EE002E0008050E0C040A2E0000000000FF0071
:1001FE000000220500022A05040430050807360512
:10020E000C0536058C063C0580094405100B4C0583
:10021E00500C560540035E05140A68051808700553
:10022E001C0100000002280060009800D0000801A8
:10023E004001210C58002D0B2D002B0B2B004D0ACD
:10024E004D00808182838400002188898A8B8C8D69
:10025E008E8F310B312041424300320B3220444508
:10026E004600330B3320474849004D0A4D0000002D
:10027E000000340B34204A4B4C00350B35204D4ECC
:10028E004F00360B3620505152002B0A2B00000027
:10029E000000370B372053545500380B3820565773
:1002AE005800390B3920595A2F002D0A2D00000005
:1002BE000000430C430000000000300B3020202EC5
:1002CE002C002C0A2C00000000003D0A43520000B6
:1002DE00000000004A01460032002100004B004A97
:1002EE0001460032004D000096004A0146003200E1
:1002FE00540000E1004A01460032003D0000F000CB
:10030E000000320050002D0000F00050003200506E
:10031E0000470000F000A000320050004B0000F03B
:10032E0000F000320050002B00005800B400040012
:10033E0038003800213803006A6100008700C800C9
:10034E00640032003D4603006E65696E00000800D1
:10035E00C80064003200215603004B004A014600DB
:10036E0032004D00000001000100E60063004D0068
:10037E0000000000A0001B00007105D700A0001AAD
:10038E000200710569000000180400730569001E63
:10039E0001190600730550726F64756B74200000AE
:1003AE00537061727465202000005F4944005F52F3
:1003BE0073323332494400005F526F7461746500CA
:1003CE005F54617374656E5800005F546173746599
:1003DE006E5900005F44656661756C744B657900FB
:1003EE002A436F64653000002A436F646531000054
:1003FE002A436F64653200002A4D61784D6F647533
:10040E006C005F4572774D6F64756C002A5469738A
:10041E00636845005F4D795465726D4E72005F4D95
:10042E0061737465725465726D7300005F454D6F34
:10043E00646500005F4543726564577472005F52D5
:10044E0073304D6F646500005F5634756E64350011
:10045E005F50756C736554696D6500005F41736B19
:10046E0043726564697400005F53656E644465622F
:10047E00697400005F4372656469744D6F64650052
:10048E005F4372656469744D6173746572002A54BA
:10049E0061626C655374617274002A5461626C659A
:1004AE00456E64002A4669727374426F6E50000086
:1004BE002A4A6F6231002A4A6F6232002A4A6F62FC
:1004CE0033002A4A6F6234002A4A6F6235002A4A84
:1004DE006F6236002A4A6F6237005F4572726F7222
:1004EE0031005F4572726F7232005F4572726F72C9
:1004FE0033005F4572726F7234005F4572726F72B5
:10050E0035005F4672656967616265005F4B6F6DAE
:10051E006D61000054617374657200004C69745A09
:10052E0000004C656974540050756C730000546182
:10053E0073742030000073657269656C6C007365AE
:10054E007269656C203200005461737420320000B1
:10055E0054617374207061720000466F6C6765544D
:10056E0000005377697463680000706F7274696F6E
:10057E006E696572656E00002E666F6C67650000B1
:10058E00506F7274696F6E656E2073696368657201
:10059E006E00436865662D4D656E75004B206C6967
:1005AE007374656E00004B206C6F65736368656EC7
:1005BE0000004B20647275636B656E0054206C698D
:1005CE007374656E000054206C6F65736368656E9E
:1005DE0000005420647275636B656E0053797374FA
:1005EE00656D0000506F7274696F6E004B726564BA
:1005FE00697465004B7265642E436C7200006D6108
:10060E006E2E506F7274696F6E00546573740000B5
:10061E00506172616D657465720050726F64756BB6
:10062E00746500004B656C6C6E65720056656E7479
:10063E00696C6500436F6C6F7273000030A00531FA
:10064E00AA0532B40533C00534CA0535D40536E0E3
:10065E000546EA0541F20543FA054402064A0C0630
:10066E000000000030EA05371806391E0638280645
:10067E00423206453A066342060000004572726F2A
:10068E0072004F70742E0000496D70756C7300000F
:10069E0054696D656F7574008A062F0C0005000095
:1006AE009006320C000300009606300C0005000088
:1006BE009E06310C001400002E202C304142433196
:1006CE0044454632474849334A4B4C344D4E4F35DC
:1006DE00505152365354553756575838595A2F3958
:1006EE000500C11100000300D90B00000300C11169
:1006FE000300170E0300D90B00000500E0080000F0
:10070E000A00C1110A00170E0A00D90B0A00C11106
:10071E000A00170E2800D90B000000000000000090
:10072E0000000000000000000000000000000000BB
:10073E000000070C182022204D994D401140489181
:10074E004720222018C007000000070C1F3FEE3F75
:10075E007277727FFF7F777F783FEE3F1FC0070073
:10076E000000000000000C183DEE3F3FEE3F1FC89A
:10077E000F07000200000000000000000000000251
:10078E0007080F1FCE3F1FC80F0700020000000012
:10079E00000000000007080F0F880F376F7F7FFFE4
:1007AE007F3260070F800000000000000002000290
:1007BE0007080F1FCE3F3FEE3F1AC0070F80000005
:1007CE00000000000000000000000006000F0F00F7
:1007DE0006000000000000000000FFFFFFFFFFFF0B
:1007EE00FFFFFFF9FFF0F0FFF9FFFFFFFFFFFFFF35
:1007FE00FFFF00000000000006000910881010889E
:10080E0010090006000000000000FFFFFFFFFFFFC1
:10081E00F9FFF6EF77EFEF77EFF6FFF9FFFFFFFF48
:10082E00FFFF000000000E01006A1E332861618880
:10083E006133001E000000000000000000078C0C59
:10084E00186618186C0C078003030C0F03000300C6
:10085E000000020003038C0302CC0202800202009D
:10086E000E1E001E0C00000000000C000E0B0809EE
:10087E000CC40E0B4C0938C478784C3103CC0301F0
:10088E0080000000020202271FCC18306770306C07
:10089E00181FC227020002000000000000100018FE
:1008AE001C001E1F081F1F001E1C00181000000039
:1008BE0000000000000088010388070F881F0F88C2
:1008CE000703880100800000000000000207080FE7
:1008DE001FC0020200020200021FC80F0700020022
:1008EE00000000081919881919881919881919880A
:1008FE0019198000198819000000000E1F36CC66E9
:10090E0066CC6636CC1E06CC0606CC0606CC060099
:10091E00000000081F30C03030081F30CC301F8C54
:10092E000000CC301F80000000000000000000001E
:10093E00000000000000000000000E1F1FEE1F0050
:10094E0000000200070F8C1F0200020200020200CC
:10095E00021FC80F0700021FC00000000207080F89
:10096E001FC0020200020200020200020200020088
:10097E000000000002020002020002020002020059
:10098E00021FC80F07000200000000000000000058
:10099E0001080101CE3F01C8010100000000000066
:1009AE00000000000000000004000C1C0E3F1C00A4
:1009BE000C04000000000000000000000000000019
:1009CE00000000000000400040400040400E7F004C
:1009DE000000000000000000088C1838EF7F38EC93
:1009EE001808800000000000000000000000000059
:1009FE0000000207080F1FCE3F7FF000000000002E
:100A0E000000000000000000000F7F3FEC1F0F8071
:100A1E0007020000000000000000000000000000BF
:100A2E0000000000000000000000000000000000B8
:100A3E0000000600060F000F0F000F0F0006060045
:100A4E0006000000060006000000000000198819CC
:100A5E0019881900000000000000000000000000CE
:100A6E0000000006060666063FFC0C0CC819198C21
:100A7E007F3300333300000000000600061F8C3F5A
:100A8E003600363F8C1F06CC063FC81F06000600F8
:100A9E000000000000001338387E3801C80307003C
:100AAE000E1C0E3870EE600000000000070D881955
:100ABE0019801B0E001E3E063333C8313BC61E0086
:100ACE0000000E000E0E000606000C0000000000D6
:100ADE00000000000000000000000380060E000C65
:100AEE001C001C1C001C1C001C0C000E0608030025
:100AFE0000001C0006070003038803038803038815
:100B0E000303000706001C000000000000000C3666
:100B1E0036C81F0F0C3F0F081F36CC3600000000E2
:100B2E000000000000000000060006060C3F3FC05B
:100B3E000606000600000000000000000000000095
:100B4E0000000000000000000000000E0E000E0667
:100B5E00000C000000000000000000000C3F3FC031
:100B6E000000000000000000000000000000000077
:100B7E0000000000000000000000000E0E000E003D
:100B8E00000000010000370000EC010380070E009A
:100B9E001C3800706000000000000F8E3F30676050
:100BAE0060FB616333666C33787036303FE80F005C
:100BBE0000000300071F001F0300030300030300D0
:100BCE00030300031FEE1F0000001FCE3F70736073
:100BDE00607E0001C80307000E1C00387FFF7F00F7
:100BEE0000001FCE3F7073600037000FEC0F0063E4
:100BFE00006037703FEC1F00000001CC0307CC0EE5
:100C0E001CCC3870CC607FFF7F00CC0000CC000085
:100C1E0000007FFF7F600060600C7F3FE7000033C5
:100C2E00006037703FEC1F00000003CC070E001C65
:100C3E003800307FCE7F7073606037703FEC1F00DE
:100C4E0000007FFF7F00660000CC000188010300DA
:100C5E00030600060C000C0000000F8C1F38E63057
:100C6E00306E381FCE3F7073606037703FEC1F00E0
:100C7E0000001FCE3F7073606037703FFF1F006E25
:100C8E000001C8031F001E0000000000000000004D
:100C9E000E000E0E00000000000E000E0E000000F2
:100CAE0000000000000000000E000E0E000000000C
:100CBE00000E000E0E000606000C00CC010380078D
:100CCE000E001C3800381C000E07080301CC000073
:100CDE000000000000000000000E3F3FE000000E8C
:100CEE003F3FE0000000000000003000381C000E06
:100CFE0007080301CC010380070E001C38003000EA
:100D0E0000001F8C3F70E66060EC01038007060058
:100D1E00060600000600060000001FCE3F306B677F
:100D2E006FBB6D6DBB6D6DBE6F67C0703FCC0F003E
:100D3E0000000600060F000F0F081919881930CC95
:100D4E003F3FC6606066600000007F087F61CC6038
:100D5E0060CC617F8C7F60E660606E607FC87F00D4
:100D6E0000000F8C1F38E63060006060006060008D
:100D7E0060306E381FC80F0000007F087F61CC60A6
:100D8E0060666060666060666060CC617F807F00D8
:100D9E0000007FEE7F6000606000607F887F6000F3
:100DAE00606000607FEE7F0000007FEE7F6000607D
:100DBE006000607F887F600060600060600060009F
:100DCE0000000FCE1F38603060006063EE63606617
:100DDE00603066381FEE0F0000006066606066606F
:100DEE006066607FEE7F6066606066606066600071
:100DFE0000001F881F0600060600060600060600F5
:100E0E00060600061F881F00000000660000660030
:100E1E00006600006600006660606C703FC81F00D0
:100E2E000000606E6061C86367006E7C007C6E00BF
:100E3E0067638C6160E660000000600060600060C7
:100E4E006000606000606000606000607FEE7F00A8
:100E5E000000606E7070EE7979E66F6F666666669A
:100E6E006060666060666000000060667070667844
:100E7E006C666C66666663666361EE6060E6600073
:100E8E0000000F081F39CC306066606066606066D7
:100E9E006030CC391F800F0000007F8C7F60E660D1
:100EAE0060666060EC7F7F80606000606000600064
:100EBE0000000F081F39CC306066606066606066A7
:100ECE006333CC391FE60F0000007F8C7F60E66035
:100EDE0060666060EC7F7F8067638C6160E66000B7
:100EEE0000001F8C3F70E6606000703F8C1F00E6B4
:100EFE0000606E703FC81F0000003FCC3F0600062A
:100F0E000600060600060600060600060600060097
:100F1E000000606660606660606660606660606665
:100F2E0060606C303FC81F000000606660606C300F
:100F3E0030CC3019881919800F0F000F06000600EB
:100F4E000000606660606660606660606666666629
:100F5E006F79EE7070E66000000060666030CC3035
:100F6E0019800F0600060F081930CC30606660003D
:100F7E00000060666030CC301988190F000F060033
:100F8E00060600060600060000007FEE7F00CC007D
:100F9E000180030600060C00183000307FEE7F0043
:100FAE0000001F881F1800181800181800181800C5
:100FBE00181800181F881F00000000004060007005
:100FCE0038001C0E0007038C0100E7000030000003
:100FDE0000001F881F018801018801018801018816
:100FEE00010188011F881F0000000200070F8C1DE1
:100FFE0038E77060300000000000000000000000C4
:10100E0000000000000000000000000000000000D2
:10101E00000000000000007FFF7F000007070007B0
:10102E0006000603000000000000000000000000A3
:10103E000000000000000000000C1F3FE6001FEE45
:10104E003F6066607FEE3F00000060006060006001
:10105E0060086F7FCE70606660606E607FC87F00D4
:10106E00000000000000000000081F3FC670600076
:10107E00606006703FC81F0000000066000066003A
:10108E0000661F3FEE716066606066703FEE1F0087
:10109E00000000000000000000081F3FC6707FEC3B
:1010AE007F6000703FC81F00000007880F1C0018EB
:1010BE001800187F007F1800181800181800180064
:1010CE000000000000000000000E1F3FE670606E82
:1010DE00703FE61F006E003FC83F6000606000601A
:1010EE0060006F7F8C7160CC6060CC6060CC600003
:1010FE00000000000006000600000E0E00060600AE
:10110E00060600061F881F0000000000000188016F
:10111E000008030388010188010188010188191F55
:10112E00800F3000303000303008313380373E00D1
:10113E003E37083331CC300000000E000E0600069C
:10114E000600060600060600060600061F881F009B
:10115E0000000000000000000008597FCE7F666688
:10116E0066666666666666000000000000000000A7
:10117E0000083F3FCE30306630306630306630008B
:10118E00000000000000000000081F3FCE706066E7
:10119E0060606E703FC81F0000000000000000007D
:1011AE0000087F7FCE6060666070EC7F6F8060604D
:1011BE000060000000000000000E1F3FE670606639
:1011CE006070EE3F1F660000660000000000000029
:1011DE00000C373FE6383000303000303000300041
:1011EE00000000000000000000003F7F80607F08CC
:1011FE003F0188017F803F00000000001818001892
:10120E0018007F7F00181800181800181F880F008C
:10121E00000000000000000000066060666060666E
:10122E0060606E703FE61F000000000000000000CE
:10123E00000660606C3030C81919800F0F00060070
:10124E000000000000000000000666666666666626
:10125E00666F6C3F39C810000000000000000000EF
:10126E00000C6071C83B1F000E1F083B71CC600064
:10127E000000000000000000000C3030C81919807A
:10128E000F0F000606000C0C0018000000000000F6
:10129E00000C7F7F800306000C1800307FCC7F008F
:1012AE00000003CC070E000C0C000C1C00381C00B8
:1012BE000C0C000C0E0C0703C00006000606000600
:1012CE0006000600000606000606000606000600DA
:1012DE0000003C003E070003030003038C01038063
:1012EE000303000307003E3C00000000001C6C36A8
:1012FE0063800000000000000000000000000000FD
:10130E00000000000000000006000F198C3060661F
:10131E00607FEE7F00000000000000001E006007EE
:10132E007E0700F01EF060F77EF7FBDE1F00E00781
:10133E00FF0700F81FF8E0FFFFFF00000F00E002BC
:10134E00EF0200780F78E07AEF7AF7BD1F00E00722
:10135E00FF0700F81FF8E0FFFFFF23000002000068
:10136E00100000050000FE0500182800FE040018FD
:10137E002400F90F00F80F0070001F718023728097
:10138E002A73111574111C75151B76151A77181CF6
:10139E00781521050100FF000000013F2B0200100F
:1013AE00072100000100072300100000FD30000798
:1013BE003300113068FF0000E500800001000100DD
:1013CE0001020004033010040000080202090000AC
:1013DE000A00000C00000D00000F000010000011AC
:1013EE000700120000130000FD500010B01B110783
:1013FE0000FD5000121E01FD500013001F291F009A
:10140E00FD5000200000210000FE01002B0C00FE0C
:10141E0000002B2000300000310603320002350799
:10142E00013604043706063805013907073C000665
:10143E003D070850000051EF00520000533F01FEDF
:10144E0001006000A7FE00006000276101006A0035
:10145E0000800000810000820000830000840000F4
:10146E00850000901000920007930700953F0397A8
:10147E000000980000070100FD500007210007231F
:10148E0000FD5000077301FD000000000000007C0D
:10149E000000000001C000C00000000000000000BD
:1014AE000000038380000000063007387FFFFC3FFA
:1014BE00FFE007FFFFC00400F0000000080E080860
:1014CE00FFFFF8FFFFFC0FFFFFF008000E00FC1FF0
:1014DE001001F018FFFFF9FFFFFE0FFFFFF01000E5
:1014EE0001810330D0000019FFFFF3FFFFFE1FFF45
:1014FE00FFF8100000C100C0D0000039FFFFE7FF69
:10150E00FFFE1FFFFFF8100000620000C800003051
:10151E000FFC07FE0FFE1FF81FF820000032000020
:10152E00C80000601FFC07FE0FFC3FF83FF82000CC
:10153E0000340000C80000601FFC0FFC1FFC3FF0D1
:10154E003FF8200000340001880000C01FF80FFC97
:10155E001FFC3FF03FF0300000640001880000C027
:10156E003FF80FFFFFF87FFFFFF0100003E40001CC
:10157E00880001803FF81FFFFFF87FFFFFE01C008F
:10158E000F840003080001803FF01FFFFFF87FFF6C
:10159E00FFC004003C040003100001807FF01FFF19
:1015AE00FFF07FFFFF000200700400061000030032
:1015BE007FF03FFFFFF0FFFFFC000200600400061B
:1015CE00200003007FE03FF07FF0FFE0000002000C
:1015DE006004000C20000300FFE03FE07FE0FFC04E
:1015EE0000000200C004000C40000300FFE07FE09A
:1015FE00FFE1FFC000000200C004001880000100DF
:10160E00FFC07FE0FFE1FFC000000101800200305B
:10161E0080000181FFC07FC0FFC1FF80000001017B
:10162E008002007100000181FFC0FFC1FFC3FF8077
:10163E00000001030002006300000181FF80FFC172
:10164E00FFC3FF8000000103000300C2001E0183E0
:10165E00FF80FF81FF83FF000000018600010381F0
:10166E00807F0303FF81FF83FF87FF00000000CE12
:10167E000001C70080E18703FF01FF83FF87FF00A2
:10168E000000007C00007E00F780EE07FF01FF03E4
:10169E00FF07FE0000000030000038003F007C070E
:1016AE00FF03FF07FF0FFE00000007FE03FE07FF0C
:1016BE000FFE000FFE000007FE0000000FFE0000F0
:1016CE000FFE0000000FFE00000FFE0000001FFFC7
:1016DE0000000FFC0000001FFFFFFFFFFFFFFFFFDA
:1016EE001FFFFFFFFFFFFFFFFF3FFFFFFFFFFFFF9C
:1016FE00FFFF3FFFFFFFFFFFFFFFFF3FFFFFFFFF6C
:10170E00FFFFFFFE7FFFFFFFFFFFFFFFFE7FFFFFDD
:10171E00FFFFFFFFFFFE7FFFFFFFFFFFFFFFFCFF4F
:10172E00FFFFFFFFFFFFFFFCFFFFFFFFFFFFFFFFBE
:10173E00FCFFFFFFFFFFFFFFFFF87FFFFFFFFFFF35
:10174E00FFFFF87FFFFFFFFFFFFFFFF82564002B71
:10175E00003E3E006B65696E204B726564697400D5
:10176E00436F6C6F72546F75636820567320312E01
:10177E0035300049443D00202047433D00202036AF
:10178E00346B004B653A00496E3A0043616C6962F6
:10179E00726174696F6E004F4B00546F74616C20F0
:1017AE00002D2D2D2D0054696E79200054696E790F
:1017BE0020626164006B65696E20454570726F6DC5
:1017CE00004D4F44554C2053544F500044617461AA
:1017DE002000696E69740000533F000066616C73EF
:1017EE00636865722054697363682000546973637B
:1017FE006820766F6E204B20004665686C657220FF
:10180E000056656E74696C20616B7469760054695C
:10181E006D656F757400435349204E722000436FFF
:10182E00646520006B65696E204B72656469740097
:10183E0066616C73636865722054697363680054E3
:10184E006973636820766F6E204B005831393931D9
:10185E00303000504C5520203A00436F6465203ADA
:10186E00005469736368203A004D42005053004B98
:10187E00656C6C6E657220004D31004F3100535017
:10188E000043500044590062757379004D5000209A
:10189E0067657370657272740025640041627265CB
:1018AE0063686E756E67004B656C6C6E65722000BA
:1018BE00546F74616C004D6F64756C2000202000B5
:1018CE00433F0073656300496D7000504C553A20DC
:1018DE00005370617274653A20005072313A2000E4
:1018EE005072323A200046756E6374203A200054CE
:1018FE0079703A20003A20563A2020302B203000C2
:10190E003A003A20544F3A20003A2050733A2000C1
:10191E0053703A004B204D6F6465204A6F62204A27
:10192E006F62466C616773004B20004D6F646520DB
:10193E00004A6F62202000562020204572722050EF
:10194E00676C20496D7020544F0056200050617511
:10195E007365004B656C6C6E65723A004D49004DB7
:10196E0042004D43004D50004D4C00746573742081
:10197E002E2E004F4E0025303258002530345800A0
:10198E00253664002533642E2530326400253564F7
:10199E0000256400253264002533640044440000B1
:1019AE004B23004253004221004246005423005470
:1019BE004F004952004D5A004251004252004353CB
:1019CE0000565300564300494C00426600004B231C
:1019DE000054230042450043450042410044530059
:1019EE0043420023502241534349492D492F4F2250
:1019FE002C22312E3030222C323030382D30312DF9
:101A0E0030313B0023482245636F222C22312E3089
:101A1E0030222C323030382D30312D30313B0023F6
:101A2E00532245636F222C22312E3030222C32303D
:101A3E0030382D30312D30313B00504F0050463272
:101A4E00333B5055002564002B302B303B00256472
:101A5E000025303258002E3030004F4E000001006D
:101A6E002D4E414E00000100DE0E6C1A0000F8945F
:101A7E00EE27ECBBF1E0F5BFE5BFE0936C00F8E1BB
:101A8E00F1BDE1BD8DE0A2E0BB27ED938A95E9F7AC
:101A9E0080E090E1A0E0B1E0ED930197E9F7E4E793
:101AAE00FAE185919591009761F0A591B591059018
:101ABE001590BF01F00105900D920197E1F7FB0122
:101ACE00F0CFEFEFEDBFE0E1EEBFC0E0D3E00C945E
:101ADE00F9160A9902C0E1E00895E0E008951A931C
:101AEE001FEFE2E00E94126CE3EFE1BB85E38A9503
:101AFE00F1F7E0EFE1BBE4E4E09374000E941B6CAD
:101B0E000E94AE66E03091F4E981EE0FE0520E9441
:101B1E00206C41F4EDB7FEB7FA93EA931F930E943F
:101B2E00256C1F910E94BF660E94296CE0E0E09335
:101B3E0071000E94296CE12F72C30E942E6C10E07E
:101B4E001430F0F400E00430C8F4A12FECE30E944E
:101B5E00326C0E94366C0E943B6CE15BFF4FFA9335
:101B6E00EA930E94406C0E94406CE02FEE0FEE0F45
:101B7E00E10FEA930E942B4C0F5FE5CF1F5FE0CF82
:101B8E00ECE0E0930F04E0E0E09310040E94456C5B
:101B9E000E94C4490E944B6C0E947743E030D9F4F6
:101BAE000E94526C0E94526CE6E9F0E00E94576C63
:101BBE000E94526C0E94526C0E9415470E94616CEA
:101BCE000E94CE410E94686C0E94CE41EEE1F0E090
:101BDE000E946F6CE1CF0E947A4341C4E881E030ED
:101BEE0011F01C9A01C01C9832C00E94526C0E94C7
:101BFE00526C0E94736CEFE3F0E00E94786C0895D3
:101C0E001A93A0910403A43081F4E0910F04E093A1
:101C1E00100410E0183048F4ABE01A9FF001E052C7
:101C2E00FD4F0E947E6C1F5FF5CF42C0A091040352
:101C3E00A43039F4E881E0931004E0E0E0930F045F
:101C4E0006C0E881E0930F04E0E0E09310042196D3
:101C5E0008951A93A0910403A43031F110E01430CA
:101C6E0018F50E94826C3196E491EA93DFDFE0E092
:101C7E00E09310040E948B6C3896FA93EA93EBE093
:101C8E00F1E00E948E6C0E948E6CFA93EA930E9491
:101C9E00826CE491EA930E94826C32960E94936C5D
:101CAE000E9438441F5FDBCF0E94966C0E949B6C93
:101CBE00199108952A970E94A17D30E010E000E06E
:101CCE0047ED50E028E0E091190CE03019F020E1EA
:101CDE0049E650E03217F0F50E949F6CE13098F122
:101CEE000E949F6CE03870F0EEE00E94A56CEAE571
:101CFE00F7E1FA93EA930E949F6CEF70EF5F0E94F8
:101D0E00AD6C07C0ECE0EA9391DFE8E5EE83E0E02E
:101D1E00EF830E948B6C38960E94366CE7E3F0E0FE
:101D2E000E941B7BE40FF51F0E948E6CFA93EA93C0
:101D3E00EDE2F0E0FA93EA930E949F6CEA930E9420
:101D4E00526C0E94B76C1F5F143011F410E00F5FDD
:101D5E003F5FC0CF0E94966C0E94C4490E94A87D2E
:101D6E00619608950E94BD6CECE0EA935FDF0E94DD
:101D7E00456CEBE0EA935ADF0E94C16C0E94C66C80
:101D8E00EAEAF0E00E94CB6CE0913A0CF0913B0C49
:101D9E00E491EA93E0913A0CF0913B0C31960E945B
:101DAE00D26C0E94384401E00E94D56C0E94D86C1F
:101DBE0011F00F5FF9CF0E94E66C031718F4E0E004
:101DCE00E093C0050E94E66C11E00E94ED6C0E944B
:101DDE00D86C11F0153008F021C00E94C16C0E9421
:101DEE00F06CE0E4F0E00E941B7B3496FA93EA93E9
:101DFE00E2EEF0E00E94CB6C0E94ED6C0E94F36C60
:101E0E00E491EA930E94ED6C0E94F36C31960E946D
:101E1E00D26C0E9438443F5F1F5FD7CF0E949B6CED
:101E2E000E94AA7D36C427970E94A17D22E354E02A
:101E3E00A0910403A43011F426E453E010E0143012
:101E4E0010F00C94750F00E0051710F00C94730F42
:101E5E00E12FEE0FEE0FE00F3E2F0E94ED6C0E9471
:101E6E00FF6C3196E4910E94A56C0E94ED6C0E946D
:101E7E00FF6C3296FA93EA930E941169ED85E03079
:101E8E0039F4AF81A13210F4E0E0EF83E0E0E887AF
:101E9E00A02FBB27E22FE85FF0E00E941B7B389655
:101EAE00FA93EA930E94F06CEAE3F0E00E941B7B47
:101EBE00E55BFF4F0E94046D0E948E6CFA93EA93CD
:101ECE000E94ED6C0E94FF6CE491EA930E94526CAA
:101EDE000E94B76C0F5FB8CF1F5FB1CF0E949B6C93
:101EEE000E94A87D2E96089522970E94096DA1301A
:101EFE0059F40E940E6DABE2B1E00E94467B2E2F8C
:101F0E0057E1E2ECF0E008C00E940E6D0E94126DE7
:101F1E002E2F53E0E7EEF0E0EE83FF830E94176D65
:101F2E00A0911908A13081F4E9ECF0E00E942E6D29
:101F3E000E94356D0E943A6DEBE2EA93EDE5F7E112
:101F4E000E94936C0E943844E3E0F0E00E942E6DF4
:101F5E00EA85FB850E94406D0E94436D0E94476D8D
:101F6E003F5FE091C10BAFEE0E94257BF0E0EE8368
:101F7E00FF8311E0E091C20B1E17B0F500E0E09177
:101F8E00C10B0E1778F50E944D6D49F10E94546DEC
:101F9E00E09310040E94D56CAE81BF810E941B7B22
:101FAE0033960E94046D0E94F06C0E941B7BDF0131
:101FBE000E945E6D0E94616DEA85FB8534970E94DA
:101FCE00406D0E94436D0E94476D3A930E946121BD
:101FDE00EF3F29F0ADE05A9FF0010E94666D3F5F22
:101FEE000F5FCDCF1F5FC6CF0E94966C0E949B6C79
:101FFE00C8C022970E94A17DE2E5F7E0EE83FF8341
:10200E0040E0443190F4AE81BF8111960E946E6D16
:10201E001396EFEFEC93AE81BF81EC93EE81FF81CF
:10202E003496EE83FF834F5FECCFE091C10BA0EFB0
:10203E000E94257B2E2F0E940E6DA0E4B1E00E941F
:10204E00467B5E2F0E94176D21FE23C00E94736D8A
:10205E000E94736DEFEAF0E0FA93EA930E94786DB6
:10206E000E94436D0E94476D0E944B6CE6EBF0E0C0
:10207E00FA93EA930E94736D0E94356D0E94786DFB
:10208E00EFE7EA93EFE5F7E1FA93EA93E0E0F0E0A9
:10209E0011C00E94736D0E94736DE8EEF0E0FA932A
:1020AE00EA93E52F0E947E6DFA93EA930E94436DA8
:1020BE00EAE8FBE0FA93EA930E9438443F5F11E0AE
:1020CE00E091C20B1E1710F00C94C21000E0E091CC
:1020DE00C10B0E1710F00C94C0100E944D6D11F430
:1020EE000C94BD10A0919A0BE0E8EA23E03821F0A1
:1020FE00A091E20BA23019F40E94546D0AC00E9406
:10210E00816DE03011F4E0E001C0E8E0E0930F04EF
:10211E00E7E0E0931004A02FBB27E22FF0E00E942F
:10212E001B7B3396FA93EA930E945E6D0E94F06CCD
:10213E000E941B7B33960E94406D0E94786D0E9418
:10214E00436D0E94476D4E2FA0911E08E32F0E94F3
:10215E00866DEA0FFB1F43833A930E946121EF3F86
:10216E0029F0ADE04A9FF0010E94666D3F5F0F5F60
:10217E00AECF1F5FA5CF0E94966C0E949B6C0E94F3
:10218E0058360E94A87D28960895E1E0E0930D044C
:10219E00E2E0E0930E04E0E0E0931004ECE0E09364
:1021AE000F04ECE5F3E00E947E6CEAE0E0930F048E
:1021BE00EAE4F3E00E947E6C0E94C44908951A93EB
:1021CE00A981A43029F4A0E021FCA1E0A03009F4FB
:1021DE0026C0E9810E948D6D0490E9810E94936D65
:1021EE00E491A02DAE1BA2501A2F0E944B6CE4EB73
:1021FE00F0E0FA93EA93EB810E94936D0E94CE7BFE
:10220E003296FA93EA93EAE3F0E00E949B6DEFE7D1
:10221E00EA93EFE5F7E10E94936C0E94384418812F
:10222E00229608950E942E6CE0E0EA930E945C19BB
:10223E000E94816D0E2FE4E3F2E00E94CE7B339775
:10224E001E2F0E94526C0E94526C0E94736C0E9450
:10225E00A26D0A930E942B4C0E94406C0E94A76DA7
:10226E000E943047E2E0E0930E04E091980BEF708D
:10227E00E09310040E94AC6DEFE0E0931004AA818D
:10228E00A13051F40E94B46D0E94C66C0E94154795
:10229E00E2E6F7E10E94B96D21FE0DC0E4E0EA939B
:1022AE008EDFECE3F2E00E94BD6DEEE3F2E00E9401
:1022BE00BD6D0E94DF49A4DC80C0E8810E94936D51
:1022CE000E94BD6DEA810E948D6D0E94BD6D0E94BF
:1022DE006D47E881EA9373DFCAC11A930A93EC81C2
:1022EE00EA93EBDF1AEEEC810E948D6D0490EC8187
:1022FE000E94936DE491A02DAE1BA2500A2FAC81CB
:10230E00A43029F4A0E021FCA1E0A03009F409C01A
:10231E001EEAAA81BB811B96E0E0EC93EC81EA9366
:10232E004EDF0E94546DE0931004EC810E94C26D4A
:10233E00FF93EF930E94736DEE810E94936D0E9446
:10234E00CE7B31960E949B6D0E94D56CFA93EA93D8
:10235E00EC85E058EA930E94526C0E94C86D0E9470
:10236E003844AF91BF91EC93EC810E94936D0E9423
:10237E00BD6DEE810E948D6D0E94BD6D0E94DF4984
:10238E0019810881259608950E94CD6D0E94126DC7
:10239E008F010E94526C0E94526C0E94736C0E94BC
:1023AE00D06D0E94B46D0E941547EA81EA930E9497
:1023BE005C190E94AC6D0E94D76D1981088123961D
:1023CE0008950E94CD6D0E94126D8F010E94526C75
:1023DE000E94526C0E94736C0E94D06D0E94B46D6C
:1023EE000E941547EC81FD810E94B96DAA81BB81C7
:1023FE000E94977D24F4A030E0E1BE070CF006C0E9
:10240E00EA81FB81FA93EA930E94D741AA81BB81AC
:10241E00A130E0E1BE0724F0A030E1E1BE070CF0F0
:10242E000AC0A6EEBBE0EA81FB81E150F0410E94BA
:10243E00E16D0E94E96D0E94D76D19810881269683
:10244E0008950E94CD6D0E94126D8F010E94526CF4
:10245E001A930A930E94DF49E0E0E0933C0C099145
:10246E0019910895E881EA930E945C190E943D201B
:10247E00E03051F10E94EF6D0E94526C0E94F36D9C
:10248E000E94AC6D0E94F76DE881EA930E94A8212C
:10249E00E8830E94FB6D3B9734F00E94FB6D0E9417
:1024AE00066EE9E40BC0A3EEB6E00E940A6E0E942F
:1024BE000D6E0E94126E0E94176EE3E7EA930E9461
:1024CE00B346E2E0E0930E04D2C00E94AE68E0E0B4
:1024DE00E0930F04A0910403A43019F4E8E6F3E0AE
:1024EE0002C0E4E7F3E0FA93EA930E9418440895D9
:1024FE000E943C470E94AE680E94D568E1E0E093DE
:10250E000D040E94EF6DE6E0F0E00E941B6EEEE619
:10251E00F7E10E94B96D0E94526CE7E0F0E00E9474
:10252E001B6EE1E8F7E10E94B96D0E941F6EEA93FF
:10253E000E94E441E5E8F7E10E94B96DE0910403E1
:10254E00EA930E94E441EBE8F7E10E94B96D089529
:10255E002A971A930A930E94526C0E94526C0E9400
:10256E00736CE4E6F0E00E94786C00E010E0153049
:10257E00B0F4053020F40E94246EE03009F40DC052
:10258E000E94526C0E94D56C0E941B6E0E942B6E94
:10259E000E94246E0E94306E0F5F1F5FE8CF0E9474
:1025AE00326E0E941547E1E9F7E10E94B96DE091A4
:1025BE003108EA930E94E4410E94C16C0E94B46DFE
:1025CE000E941547E5E9F7E10E94B96DE0912306F7
:1025DE00EA93E5E0EA930E949A41E091190CE0300B
:1025EE0079F10E94C16C0E94A76D0E941547E0917F
:1025FE0028060E94356E0E94736D0E941547E09169
:10260E002806E295EF70E695E695AE2FE091290645
:10261E00EE0FEE0FEA0F0E94356E0E94C66C0E94FE
:10262E001547E0912906E295EF70AE2FE0912A064C
:10263E00E295E07FEA0FEA93E6E0EA930E949A4180
:10264E000E94C16C0E94A76D0E941547E0913F0C3D
:10265E00EA930E94EA41198108817DC1E881E06414
:10266E00E7B9369A349BFECF349AE4B1F5B1219690
:10267E000895E881F981AA81BB81AE17BF071CF4CA
:10268E00EA1BFB0B06C0A881B981EA81FB81EA1B1C
:10269E00FB0B2496089528970E94A37DEFE0E0930C
:1026AE006100E1E0E09362000E941B6CE5E0E093C4
:1026BE0061000E941B6C0E943B6EE0936F05F093CD
:1026CE007005E0917B05F0917C05E0936D05F0932C
:1026DE006E05E1E0EA93C2DFE0937B05F0937C05A3
:1026EE00EFE0E0936100E8E0E09362000E941B6C73
:1026FE00EAE0E09361000E941B6C0E94406EE09342
:10270E006B05F0936C05E0917905F0917A05E093F5
:10271E006905F0936A05E0E0EA93A0DFE09379059E
:10272E00F0937A050E94406EA0916B05B0916C05F6
:10273E00EA0FFB1FA0917905B0917A050E94456EB4
:10274E008F010E943B6EA0916F05B0917005EA0F4C
:10275E00FB1FA0917B05B0917C050E94456E9F01E9
:10276E00E0916B05F0916C050E944C6EFF93EF9318
:10277E000E94406E0E944C6EAF91BF91EA0FFB1FFC
:10278E00FF93EF93E0917905F0917A050E944C6EDC
:10279E00AF91BF91EA0FFB1FE0937505F09376059D
:1027AE00E0916F05F09170050E94526EFF93EF93CA
:1027BE000E943B6E0E94526EAF91BF91EA0FFB1FBB
:1027CE00FF93EF93E0917B05F0917C050E94526E92
:1027DE00AF91BF91EA0FFB1FE0937705F093780559
:1027EE00A0917505B0917605E4E1F0E00E94ED7AD6
:1027FE000E2EA0917705B0917805E4E1F0E00E94ED
:10280E00ED7AE02919F00E94E845A3C00093710506
:10281E00109372052093730530937405A09164058F
:10282E00A63428F4E0916405EF5FE09364050E94FE
:10283E00586E989724F40E945D6E98970CF00EC017
:10284E00A0916405AA3019F4E1E0E0936105A0912E
:10285E006405A83219F4E2E0E09361050E94586E17
:10286E00999724F00E945D6E99970CF472C0E091D6
:10287E006705EF5FE09367050E94626E0E94586ED7
:10288E000E94676E0E946E6E0E94736E0E94207B85
:10289E007F936F93FF93EF93A2E0B0E00E94E97BEA
:1028AE000F010E94626EDF01F001EA1BFB0BAF917C
:1028BE00BF918F919F910E947C6E0E946E6E0E94BE
:1028CE00816E0E945D6E0E94676E0E94866EAC8164
:1028DE00BD818E819F81EFE3F1E060E070E00E94A8
:1028EE00207B7F936F93FF93EF93A6E0B0E00E945F
:1028FE00E97B0F010E94816EDF01F001EA1BFB0BE9
:10290E00AF91BF918F919F910E947C6E0E94866EB7
:10291E00E0911204E03049F4E885F985E093590519
:10292E00F0935A05EC81FD810AC0EC81FD81E093A4
:10293E005905F0935A050E94736E0E94B57AE09382
:10294E005B05F0935C050E94616C0E94686C0E94AE
:10295E0070450E94AA7D2C9608951A930E943C47BA
:10296E00E2E0E0930E04E2E3F0E00E948E6C0E943F
:10297E008B6EE9E9F7E10E94B96DE4E1EA930E94FA
:10298E004341E0E9F1E00E948F6EE4E1EA930E9498
:10299E004341A0916705A13010F0A895FACF10E041
:1029AE00143010F00C943315E2E0E0930D040E9405
:1029BE00936EDF010E94BD6DFD0132960E94BD6DCA
:1029CE000E9430470E94936E3496E491EA930E94DF
:1029DE00B346E1E0E0930D04A0916705AF3110F42A
:1029EE00A895FACFEAE0EA930E9443410E94936EC3
:1029FE00DF0135960E94CE7BBF01FD010E94996ECC
:102A0E00DB010E94F97BE2E3F0E0FA93EA930E9485
:102A1E00F06CE8E2F0E00E941B7BE65AFF4F0E944A
:102A2E008B6E0E94936E0E94996E0E94066EA0910C
:102A3E006705AE3110F0A895FACF0E94936EDF01B4
:102A4E000E94BD6DFD0132960E94BD6DE8E1F0E081
:102A5E000E94576C1F5FA4CFE2E3F0E0FA93EA9373
:102A6E00EAEFF0E00E948B6EE5EAF7E10E94B96DA5
:102A7E00E0EDF7E00E948F6E0E943C474DC10E9430
:102A8E00A06E0A93E4E6E2BF78940E94324503DE1C
:102A9E00E6B3AFEFEA27E0933108A2E6BBE00E946F
:102AAE00AF6EE091620BE77031F4A0910A04E0E49E
:102ABE00EA27E0930A04E091620BEF7131F4A091E2
:102ACE000A04E3E8EA27E0930A040E947C660E9467
:102ADE004922E2B3EF700E2EA0911408B0911508A2
:102AEE00EFE0F0E0AE27BF27EA23FB230E94CE7A69
:102AFE00E029E2BBE0911408E07111F41D9A01C0C7
:102B0E001D980991199115C00E94A06EE6E0E4BDD2
:102B1E00E0B1E295EF70AE2FE0916300E071E15FFE
:102B2E00EA231E2F0E94A26D0E9420220E9456664A
:102B3E001991E991EFBFF991E991B991A991999103
:102B4E00899179916991F9901990099018950E943F
:102B5E0080650E9406660E9471510E94791F089539
:102B6E001A93A8950E944943E13011F00C9418165F
:102B7E00E091C605E1501E2FA091C505A13021F4AC
:102B8E000E94B56EE03009F40CC0ADE01A9FF00162
:102B9E00E15FFC4FBF01E081E260DB01EC930E943C
:102BAE00BC6EA091C505A23011F0A43089F40E942C
:102BBE00B56EE093DB050E94C16E31F0FD01E15F61
:102BCE00FC4FE081E27009F403C01A930E94CA6EB2
:102BDE00A091C505A33019F41A930E94F927A0916C
:102BEE00C505A53029F4E091C605EA930E94302868
:102BFE00A091C505A830A9F4E0E0EA93E091C605DE
:102C0E00EF77EA930E942F191E2F1F3F51F0E0E03D
:102C1E00EA930E944341E12FE058E093DB05E093F5
:102C2E002D06E0910A04E078D1F0E0910A04EF77E6
:102C3E00E0930A040E94084AE0910A04E07131F020
:102C4E00E0910A04E270EA930E941A46A0913208BB
:102C5E00A13328F0E2E0EA930E94760D1E2FA09198
:102C6E003C0CA13039F4E0913D0CF0913E0C0E94E9
:102C7E00CE6E09F401C0E5DB6ADF4EC01A930E94E6
:102C8E003C47E1E0F0E00E94936C0E94154710E093
:102C9E000E94D86E0E94526C0E94A26D0E9415472F
:102CAE00E0912108E03049F4E8EAF7E10E94B96DBD
:102CBE000E94DE6E0E94176E1E5FA0912108A13049
:102CCE00F0F0E0912108E150EA930E948B19A09157
:102CDE00B30BAD3229F40E94E76E0E94937D79F01A
:102CEE00E3EBFBE00E94E96DE6E0F0E0FA93EA9395
:102CFE000E94F46E0E94E76E0E94176E1E5FE091B6
:102D0E002108EF5FE09321081C3020F4A0912108E8
:102D1E00AB3008F001C0BECF199108951A930E94EE
:102D2E003C47E981E03019F4E0E0E0931E08A98108
:102D3E00A230A9F410E0A0911E08A13010F01C30B2
:102D4E0008F00DC0E0911E08E150E0931E080E94AD
:102D5E00F86E19F40E94066F09F01F5FECCF0E9407
:102D6E00D86E10E00E94526C0E94A26D0E94154710
:102D7E00A0911E08A03408F50E94F86E19F40E9466
:102D8E00066FD1F0E0911E08EA930E945C190E9432
:102D9E00AC6D0E94526C0E94F46E0E94116F0E94E4
:102DAE00066EE8E7EA930E94B3460E94F76D0E9412
:102DBE00166F0E94176E1E5F05C0EFEAF7E10E94C4
:102DCE00B96D1E5FE0911E08EF5FE0931E081C3088
:102DDE0020F4A0911E08A13408F001C0C3CF1881C1
:102DEE0022960895E0E0E5BFE0936D00E0936C005D
:102DFE00EBBBEFEFEABBE0E0E8BBE7BBE5BBEFEF19
:102E0E00E4BBE0EFE2BBE1BBE0E2E3B9ECEBE2B93D
:102E1E00E0E0E0936200E0936100EFE0E093650094
:102E2E00E0936400E0E0E0BFE7E0E3BFE4E6E2BF8A
:102E3E00E0E0E1BFEFBDEEBDEDBDECBDE7BDE6BD33
:102E4E00EBBDEABDE9BDE8BDE0937900E093780003
:102E5E00E3E0E5BDE6E0E4BDE0E0E3BDE0938B003A
:102E6E00EAE0E0938A00E0E0E0938900E0938800D6
:102E7E00E0938100E0938000E2E1E0938700E4E3D9
:102E8E00E0938600E0E0E0938500E0938400E09319
:102E9E008300E0938200E0936A00E0E3EABFE0E49F
:102EAE00E9BFE8BFE1E4E7BFE0E0E0937D00EBB906
:102EBE00E8EDEAB9E6E0E0939500E0E0E0939000FB
:102ECE00E7E6E9B9E0E0E0939B00E8EDE0939A00D5
:102EDE00E6E0E0939D00E0E0E0939800E3E3E0930A
:102EEE009900E0E8E8B9E0E0E0BDE0E4E7B9E7E842
:102EFE00E6B9E0B5EF7EE0BDE0E2E0937000E0E021
:102F0E00E0937200E4E4E0937400EFE1E1BDEFE0E2
:102F1E00E1BD0E94295E0E94C74B0E940B46789429
:102F2E000E94C74B0E940B46E1E0EA930E94F50D0A
:102F3E000E941F6EE53128F0A9E0B0E0E0E00E94AB
:102F4E00017CD6DA21E030E0E0E0EA930E94760DD3
:102F5E00E0933208EAE0F0E00E948F6E3F5FA091AE
:102F6E003208A43511F03A3008F001C0EDCF0E94BE
:102F7E00B46D0E94C16C0E941547A0913208A43511
:102F8E0081F4E1E0EA930E94760DE0933208E4EBDF
:102F9E00F7E10E94B96DE0913208EA930E94B346C0
:102FAE0007C0E0E0E0933208EAEBF7E10E94B96D6A
:102FBE0094D0E03059F40E94B46DE9E0F0E00E9444
:102FCE001B6EE3ECF7E10E94B96D20E00E94626E89
:102FDE000F01A2E0B0E00E94E97B0E161F0654F42A
:102FEE000E94816E0F01A6E0B0E00E94E97B0E16F2
:102FFE001F060CF0B2DC203071F40E94B46DEAE0D2
:10300E00F0E00E941B6EEFECF7E10E94B96DA895FF
:10301E000E941F6FFCCF0E943F370E94B46DE9E003
:10302E00F0E00E941B6EEAEDF7E10E94B96D0E947E
:10303E00031CE03019F0E0EEF7E102C0E5EAF7E13B
:10304E00FA93EA930E94CA460E948E66E1E0EA93E2
:10305E000E94434100E010E00436E0E01E0724F435
:10306E000E940666E03009F007C0EAE0F0E00E9438
:10307E008F6E0F5F1F4FF0CF0436E0E01E072CF06F
:10308E00A0916705AF3108F068DC6ADD0E949C32C2
:10309E000E94351EFACFFFCF0E94226F17FD02C08D
:1030AE00103011F4E0E063C3E12F61C30E94226F80
:1030BE0017FD10E01A3008F41F5F0E942F6F57C3E0
:1030CE000E94226F17FD02C0103011F4E0E04FC3D2
:1030DE0011500E942F6FE1E04AC31A930A9310E039
:1030EE00E4E6F0E00E948F6EA8950E94AE66E03096
:1030FE0021F4E0EA0E943A6F09F002C001E001C03B
:10310E0000E00E94BF661F5F003011F4153008F01A
:10311E0001C0E6CFE02F0991199108950E943F6FEB
:10312E0043C40E943F6F0E944C6F0895A881B981DD
:10313E000E94977D24F4A83EE3E0BE070CF005C084
:10314E000E94526F0E94216713C3E0E011C3A88151
:10315E00B9810E94977D24F4A83EE3E0BE070CF0EF
:10316E0005C0EA81E03011F4EFEFEA830E94526F5E
:10317E00ED81EA930E944D6760C10E94A37D20E01D
:10318E0030E0283EE3E03E077CF4A8953A932A937C
:10319E00CDDF1E2F1F3F29F0EFEFEA933A932A93CC
:1031AE00D6DF2F5F3F4FEDCF0E94AA7D4FC01A93FF
:1031BE000A93E0E0F0E0E093400CF093410CAA811A
:1031CE00A03468F40E945B6FE55FFB4F8F010E9495
:1031DE00626F1A930A93E0E4FCE00E94656FE0913F
:1031EE00400CF091410C27C11A931FEF1F5F1A93E9
:1031FE00DEDFA981BA81EA17FB0711F0113408F05E
:10320E0001C0F4CFE12F188118C11A930A93A0912F
:10321E00C10BE091C20BEA9FF001A0911E08EA0FCC
:10322E000E2F013408F00FE310911E08101758F4FA
:10323E001A93BDDFAA81BB81EA17FB0711F4E12FB8
:10324E0003C01F5FF3CFEFEF198108812496089515
:10325E000E94A17D10E0103418F50E94F06CE8E297
:10326E00F0E00E941B7BE050FC4FAF01E0EAEA93D6
:10327E00FA0170960E94696FEC713E2FE0EAEA93B4
:10328E00FA013F960E94696F0E2FEF81E31719F432
:10329E00EE81E01709F002C0E12F03C01F5FDBCF04
:1032AE00EFEF0E94A87D289608951A930A93E09155
:1032BE00890BAA81EA17C1F0A03468F40E945B6FF3
:1032CE00E050FC4F8F010E946D6F0E94656FEA8186
:1032DE00E093890B09C0EFEFE093890B0E94786FA2
:1032EE000E947D6FE093940BA6C01A930A930E94DE
:1032FE005B6FE050FC4F8F01AA81A03420F40E9436
:10330E006D6F0E944C6F97C01A930A93E091B20BA7
:10331E00AA81EA17A1F00E94876F40F40E94936F72
:10332E000E94656FEA81E093B20B09C0EFEFE09364
:10333E00B20B0E949E6F0E947D6FE093BD0B7BC00F
:10334E001A930A930E94876F20F40E94936F0E9433
:10335E004C6F71C01A930A93E091330CAA81EA174D
:10336E0061F10E94A36F18F50E94626F1A930A937F
:10337E00E4E3FCE00E94656FEA81E093330CE0E049
:10338E00E0932B06A091350CA13020F0A091350CC6
:10339E00A83008F00BC0A8EDBBE0E091350C0E9400
:1033AE00AD6FAE0FBF1FEC91E0932B0606C0EFEF93
:1033BE00E093330CE0E0E093340C3DC01A930A9393
:1033CE000E94A36F40F40E94626F1A930A93E4E383
:1033DE00FCE00E944C6F2FC01A930A93E0912E0CC2
:1033EE00AA81EA17C1F00E94B06F70F4E0EAEA9386
:1033FE000E94C66C1A930A93EFE2FCE00E94656F7E
:10340E00EA81E0932E0C07C0EFEFE0932E0C0E94A2
:10341E00BA6F0E94E6680FC01A930A930E94B06FAB
:10342E0050F4E0EAEA930E94C66C1A930A93EFE214
:10343E00FCE00E944C6F19810881239608950E942A
:10344E00BA6F0E94E668E881EF5FE093300CD2C15C
:10345E0024970E94A17D0E94C16F0E94E668AA85F2
:10346E00A03478F5AB85A13010F0A63008F007C077
:10347E00EB850E94AD6F0E94C86F0E94DB6FEB85DB
:10348E00E030F9F4E0E0EE83EF83E887E98740E08F
:10349E0050E020E030E02530E0E03E0784F4F90112
:1034AE000E94C86F0E94DB6F0E94116F4E0F5F1F4C
:1034BE000E94166F0E94E06F2F5F3F4FECCF0E946D
:1034CE00EB6F3FC11A930A93AB81A13010F0A63077
:1034DE0008F01CC0EB810E94AD6F0E94D27A0E9450
:1034EE00CE7ADF01EA810E94FC6FE8E0F0E00E94F4
:1034FE001B7BE050FA4E8F01E0EAEA930E94C16C0A
:10350E001A930A93ECE1FCE00E944C6F198108813A
:10351E000C94771F0E94A37DEC810E940070E8310D
:10352E0009F459C00E940570309729F00E94057069
:10353E000E940A70EC830E9431200E2F10E01017AB
:10354E0010F00C94F21A0E940E7082DFAEE1BCE015
:10355E000E94AF6EA091200CB091210C8091220C94
:10356E009091230C0E9413700E94B07AE093200C6D
:10357E00F093210C6093220C7093230C0E940E701A
:10358E00A1DFE0EAEA93EE810E94AD6FEE0FFF1F1E
:10359E00E050F04F0E94696FE270D9F4ED81E09334
:1035AE00240C0E940570309751F40E941F6E0E94E9
:1035BE001A70EF5EF84DDF010E94207002C00E946B
:1035CE000570E093250CF093260C0E9425700E9446
:1035DE002A701F5FB4CF0E94AA7D269608951A9373
:1035EE000A930E943070ECE2F0E00E9437700E9465
:1035FE003B700E94407010E01034D8F41A9355DEE0
:10360E00E0912208EA931A9323DF0E944970EA0F91
:10361E00FB1F0F010E9449700E945170DF01CB0108
:10362E000E94166F0E94B07AD0010E94C97B1F5F64
:10363E00E3CFA0911908A330B9F500E00031A0F551
:10364E000E94D56C0E94567069F510E01A3050F544
:10365E00E02FE05DEA93E6EEF7E10E945B70E12F6A
:10366E00E05D0E946270E1F40E9467700E946E70CD
:10367E00EA0FFB1FFF93EF930E946E700E94517032
:10368E007F936F93FF93EF930E947262AF91BF91FE
:10369E008F919F910E94B07AAF91BF910E94C97B8A
:1036AE001F5FD4CF0F5FCACF10E01A3090F40E9484
:1036BE006E700E945170A0912908B0912A088091D5
:1036CE002B0890912C080E94B07A0E9440701F5FC8
:1036DE00ECCF0C94BF1F24970E94A17DEA85EA933C
:1036EE0066DD9F01022E032A39F13A932A937CDD7F
:1036FE001E2F40E050E0E0E0EE83EF83E887E9879D
:10370E00AA851A17B1F4012F003498F40A934FDDED
:10371E002E173F0761F4EB85EA930A9399DE0E9418
:10372E00116F4E0F5F1F0E94166F0E94E06F0F5FAA
:10373E00EBCF0E94EB6F05C0EB85EA93EB85EA9326
:10374E0087DE0E94A87D2C9608951A93A895A981CC
:10375E00A63068F40E94C16F0E94E66810E0103433
:10376E0030F4E981EA931A93ADDE1F5FF8CF18812A
:10377E00229608951A9311E0163020F41A93E5DF7D
:10378E001F5FFACF67C3E1E0E093340CE093350C92
:10379E0031C0A8950E949E6FEEEAF3E0FA93EA9389
:1037AE000E94C16C0E947570E093BB0B0E947E70EC
:1037BE00E093BC0BE0E0E093BD0B1CC0A895E9E8DC
:1037CE00FBE00E948570E9E2F0E00E9437700E94F3
:1037DE00786FE4EAF3E0FA93EA930E94C16C0E94D8
:1037EE007570E093920B0E947E70E093930BE0EB6A
:1037FE00E093980B219608950E94A17D0E948A70F5
:10380E00E03228F0AAE0B0E0E0E00E94017C00E0A7
:10381E0085DCA091BE0BB091BF0BA633E2E1BE07D3
:10382E0041F110E01A3030F41A93B3DF1A9388DDA9
:10383E001F5FF8CF10E0103430F41A93BFDF1A93E5
:10384E0054DD1F5FF8CF10E0103830F41A939BDF71
:10385E001A93B4DD1F5FF8CF8DDFA9E0B0E0E0E092
:10386E000E94017CE6E3F2E1E093BE0BF093BF0B06
:10387E0001E010E0183210F00C94961C0E948F702C
:10388E009F010E948F70AF010E9499703496E4914F
:10389E00E03011F0E13069F4D901AC910E949970D9
:1038AE003596E491EA1720F40E9499700E94A07058
:1038BE0034C0E23091F4DA010E94BF7BE031A7E21E
:1038CE00FA0714F4FF2342F40E94997036960E9470
:1038DE00CE7BDA01ED93FC9320C0E33049F4D9019D
:1038EE00AC91AF3F21F40E9499700E94A07015C058
:1038FE00E43099F4D901AC91AF3F79F400E00E9425
:10390E0099703596E4910E1740F40E9499700E94BA
:10391E00A0702F5F3F4F0F5FF2CF1F5FABCF01DC69
:10392E0010E0153060F41A9357DDA0912F0CA630DD
:10393E0020F01A9384DD1A936FDD1F5FF2CFE02F14
:10394E000C944721E881EF5FE883A881A43610F03C
:10395E00E0E0E883E8810C94C0210E940A6EA5E0A5
:10396E00B0E00E941B7B30960C94C021A091370CC6
:10397E00BB27E091360CA6C0F9DF329774F00E9497
:10398E00A570E091360C0E94AC700E944C6FE091D5
:10399E00360CEA93D7DFE093360C08950E94A5709B
:1039AE00E091370C0E94AC70FA93EA930E946E6716
:1039BE000895E4E2FCE00E94B4700E94A570E091CC
:1039CE00370C0E94AC700E944C6FE091370CEA935A
:1039DE00B9DFE093370C08950E94A37DE0E0E093F9
:1039EE00360CE093370C10E030E0343680F5A895B5
:1039FE000E94A5703A93B1DFFA93EA93E4E2FCE0F9
:103A0E000E94656F00E0A091240CA13010F0A03848
:103A1E0008F001C001E0E12FE03041F4013029F45B
:103A2E003093370C3093360C11E00FC0E13031F487
:103A3E00003019F43093360C12E007C0E23029F44E
:103A4E00013019F43093370C13E03F5FCECF46C2EE
:103A5E001A93A091CF0BA870B9F010E0E981FA810A
:103A6E000E94F06CAE17BF077CF4ED81E093240C3E
:103A7E00EB81FC81E851FC4F0E94BB70E0E0F0E06E
:103A8E000E942A701F5FEACF18810C944921E881A9
:103A9E00EF5FE883A881A43610F0E0E0E883E881C8
:103AAE000C94C021E881E150E883A881A43610F07F
:103ABE00E3E6E883E8810C94C021A091390CBB2782
:103ACE00E091380CF0E031960E94C070EC59FF4F37
:103ADE00DF01E4E6F0E00E94787B08950E940A6E12
:103AEE00A5E0B0E00E941B7BE050FE4F0C94C0217D
:103AFE00E9E2FCE00E94B470E881EA93BBD10C9439
:103B0E00C0211A933ADBE1E0E093860BA3C1A8959E
:103B1E0010E0143680F41A93A6D1A091290CAF3F71
:103B2E0031F40E94C570AF3FEFEFBE0711F01A934C
:103B3E00DFDF1F5FEECF0E94CA70689420F88AC143
:103B4E000E94A37D1091390CAD81AA23CAF5E09194
:103B5E00380CE11719F0AD81AA230AF030C01A9380
:103B6E0082D10E94C570EE81FF81EA17FB0729F40E
:103B7E00E885A091290CEA1709F01EC00E94D070AA
:103B8E00EC81FD810E94BA7AEA17FB0744F40E9489
:103B9E00D5700E94DE70E0E0EC83ED830BC00E94D6
:103BAE00D570EC83FD83E0E0F0E00E94DE70E0E093
:103BBE00E093290C1A935ED10E94E370C8CF46C0E1
:103BCE00E091380CE11729F0AC81BD810E94977D00
:103BDE000CF01BC01A9347D10E94C570EE81FF8175
:103BEE00EA17FB0729F4E885A091290CEA1709F0DA
:103BFE0009C00E94D5700E94DE701A933BD1E0E09E
:103C0E00EC83ED830E94E370DBCFAC81BD810E941B
:103C1E00977D1CF452DF33970CF418C0E885E093BF
:103C2E00290CEE81FF810E94E870EC81FD810E94DB
:103C3E00DE70E091380CEA931DD1E091380CEA93D6
:103C4E0026DFE093380CE0E0EC83ED83689420F8F7
:103C5E00EC81FD810E94AA7D299608951A93A09168
:103C6E00420CA03059F4E091450CF091460CFA93B9
:103C7E00EA93E8EBFBE00E94ED7009F40BC0E1E083
:103C8E00E093420CE091380CE093440CE091380C38
:103C9E00E093430CA091420CA13011F00C94B31E92
:103CAE00E091390CA091440CEA1711F40C94A41E67
:103CBE00E091440CEA93F6DEE093440CEA93D3D001
:103CCE00A091290CA13010F0A03808F035C0E09179
:103CDE00430CEA93E7DEE093430CA091440CEA1701
:103CEE0059F1EA93C7D0E091E20BE030E9F410E02D
:103CFE001530D0F4ABE01A9FF001DF01E352FA4F1A
:103D0E00E081E03049F0FD01E452FA4FE081AE2F40
:103D1E00E091440CEA1709F005C00E94F370A091DF
:103D2E00430CA0831F5FE4CFE9E2FCE00E94B47075
:103D3E00E091440CEA939ED00FC0E091430CE093C7
:103D4E00390CE0E0E093420C689420F80E948868F9
:103D5E00E093450CF093460C7DC01A93A8951091F4
:103D6E00390CE091380CE117C1F00E94F9700E94F5
:103D7E00977D64F4EB81A091290CEA1739F40E9427
:103D8E00C570E981FA81EA17FB0709F003C0E12F3C
:103D9E001881A6C00E94E370E4CFEFEF1881A0C097
:103DAE000E94D0700E94977D84F4E0912B06E870FB
:103DBE0031F4E0912F08A091290CEA1731F40E94FA
:103DCE00FD700E940A70E03408F001C05CC10C94D2
:103DDE001E22A895E091380CA881EA1761F0E881BF
:103DEE000E94027119F0E8810C94C021E881EA93D7
:103DFE004EDEE883EFCFEFEF0C94C0211A93A89517
:103E0E001091390CE091380CE117E1F00E94F97035
:103E1E000E94977D8CF4E0912B06E87031F4E091CE
:103E2E002F08A091290CEA1739F40E94C570E98178
:103E3E00FA81EA17FB0709F002C00C9405220E94D2
:103E4E00E370E0CFEFEF0C9406221A931091390C29
:103E5E001A93BFDF19910895E881EA9318DEE8837B
:103E6E00EA93B7DF86C20E94A5700E9409710E9474
:103E7E00656F7FC20E94A5700E9409710E944C6FEF
:103E8E0078C20E94A37D0E94CA7010E030E03436E2
:103E9E0028F5A8953A93E7DF00E0A091290CA03809
:103EAE0008F401E0E12FE03041F4013029F43093C1
:103EBE00390C3093380C11E00FC0E13031F4003082
:103ECE0019F43093380C12E007C0E23029F40130B7
:103EDE0019F43093390C13E03F5FD9CF0E94AA7DBD
:103EEE00249608951A930A93A0911908A43009F400
:103EFE003FC010912F080091510CE0913108E03035
:103F0E0059F0E0932F08689424F80E941271E0E0B3
:103F1E00E0933008E0E520C0E0913008E03021F079
:103F2E00E0932F08E2E518C0E0E0E0932F08E0935D
:103F3E00510CE091C40BE03031F0E091C40BE15034
:103F4E00EA930E94B119A091340CA17039F0E0915E
:103F5E00C40BE0932F08E4E4E093510CA0912F08DA
:103F6E001A1721F4A091510C0A1711F0689423F836
:103F7E000991199108950E941871EBE0EC93EC8170
:103F8E00D8011696EC93EB81D8011796EC93D801D5
:103F9E001896E0E0F0E0ED93FC93D80112960E94A3
:103FAE002571D80114960E9425710E942A71F2C0C3
:103FBE000E941871ECE0EC930E942A7121C21A93B0
:103FCE0018E0113108F5E0911408F0911508A98157
:103FDE00BA81EA27FB27BF010E943671E623F72339
:103FEE00309781F00E943671A981BA81EA23FB23B2
:103FFE00309731F01A93E0E0EA931A93BCDF02C0D7
:10400E001A93D6DF1F5FDDCFFAC1A0911A0CA9302B
:10401E0030F0E091590CA091580CEA1709F414C035
:10402E00E091590CE03021F4E3E6EA93C1DF08C0D9
:10403E00E0911A0CEA93E0E0EA93E3E6EA939BDF61
:10404E00E091590CE093580C0895A0919A0BECE175
:10405E00EA230895A0919A0BA07411F0E2E008955E
:10406E00A0919A0BA07809F0E2C10DC0A091890B26
:10407E00AF3F09F4DCC1E9DFE43009F4D8C1E5DF74
:10408E00E03109F4D4C1E1E008950895A881AF3F6D
:10409E0011F4E0E06EC1D9DFE43011F4E1E069C162
:1040AE00E0E067C1A881A23019F4CFDFE83011F04B
:1040BE00E1E05FC1E0E05DC1E881A3E2EA9FF001CB
:1040CE00ED55F94FE081E13010F0E43108F002C017
:1040DE00E1E04FC1E0E04DC1A881A13118F0E881C7
:1040EE00E051E883E8810E9441710E944B71A091DA
:1040FE00D00BA13018F0A881A43009F006C0E6E973
:10410E00F0E00E94CE7B0E944B7133C1A881A1309A
:10411E0010F0A63008F006C0E8810E945671E15CEE
:10412E00F94F26C1E0E025C1A881A13010F0A630DC
:10413E0008F006C0E8810E945671EC5BF94F18C179
:10414E00E0E017C10E94A37DEC81EA93EDDFEF73EF
:10415E001E2F1030E1F0EC81EA93E6DFE0743E2F83
:10416E00E12FE150A1E00E94C67AA0912306EA2336
:10417E000E2F303011F4003009F002C0E1E008C01B
:10418E00303011F0003009F402C0E1E001C0E0E08F
:10419E000E94AA7D259608950E94A17D00E005301B
:1041AE00A0F50A930E94F3190E945B71A7E10A9F82
:1041BE00F001EE5CF94F0E948570E4E1F0E00E94A0
:1041CE003770E091300CDA015096EC93A0912F0CE1
:1041DE00EFE3EA23AE2FE091320CE295E07FEE0F93
:1041EE00EE0FEA0FDA015596EC93E091300CE150A8
:1041FE003E2F3F3F41F0E091310C0E941A70DA01E0
:10420E005196ED93FC930F5FCACF10E01034C0F5BA
:10421E001A930E945C191A9339DFE13079F5E09117
:10422E009D0BEA9373DFE1500E2F0F3F39F10E9481
:10423E005B71E12FDA011396EC93E0919D0BDA019D
:10424E001496EC93E091A30BF091A40BDA01169661
:10425E00ED93FC930E941370A4E6B0E080E090E032
:10426E000E94207BDF01CB01E091A30BF091A40B08
:10427E000E947C6EDA011A96ED93FC931F5FC6CFF7
:10428E000E94A87D26960895A0911908A23031F0BB
:10429E00A83021F0A73011F0A53009F40AC00E9411
:1042AE003070EFEFF0E00E94377076DFE0E0E093E1
:1042BE00A20608951A93E981E058E98310E01530BB
:1042CE00C0F4A3E21A9FF001EB55F94FE081AE2F37
:1042DE00E981EA1749F4F001EC55F94FE081AE2F70
:1042EE00E0912F08EA1709F002C0E12F03C01F5F0B
:1042FE00E6CFEFEF1881229608950E94A37DED81FF
:10430E00EA93D8DF1E2F1F3FC1F00E9462719F01FA
:10431E00D9011296EC91EF77EC93EC81D9010E94C2
:10432E006871EF5EFC4FBF01E081EF77DB010E9409
:10433E006871E15FFC4FA1E0A083E12F0E94AA7D8E
:10434E00E2C40E940A6EED55F94FE081E03061F44F
:10435E00E0914B0CEF5FE0934B0C0E940A6EED5513
:10436E00F94FA0914B0CA0830E940A6EED55F94FA8
:10437E00E081219608951A931FEFE091D40BF091EE
:10438E00D50BA981BA81AE17BF073CF0E091D60BD1
:10439E00F091D70BEA17FB070CF412C00E946F7155
:1043AE000E949D181E2F103031F01F3F21F0E0911A
:1043BE002F08E11729F4E1E0E093590CE0E01FC06B
:1043CE00E0E0E093590C1AC01A930E946F71D3DF8C
:1043DE001E2F103099F01F3F39F4EAEEF7E1FA93F1
:1043EE00EA93EB81FC8106C0EAEFF7E1FA93EA93D8
:1043FE000E947471FA93EA930E94E811E12F1881DA
:10440E0023960895E0916505E03009F00895E09156
:10441E002C06E03009F008950AC0E0916605E03000
:10442E0009F00895E0912D06E03009F00895E0E0DE
:10443E0008950E94A37DE0912606F0912706AC8197
:10444E00BD81EA27FB279F0110E0153090F4F9019A
:10445E00E17049F0A7E11A9FF001EF5CF94FDF011F
:10446E00EC91EF5FEC93D9010E9477719F011F5F72
:10447E00ECCFEC81FD81E0932606F09327060E9497
:10448E00AA7D41C428970E94A17D3091260610E096
:10449E001530B8F5A7E11A9FF001EB5BF94F0081DB
:1044AE00E12FA1E00E94C67A2E2FE22FE32391F096
:1044BE00003810F0003C08F001C00F5F003C31F4F2
:1044CE00E22FA0912306EA2BE0932306003808F48E
:1044DE0000E80FC0003408F40F5F003439F4EFEF3A
:1044EE00E227A0912306EA23E0932306003808F082
:1044FE0000E0A7E11A9FF001EB5BF94F00831F5F0D
:10450E00C7CFE0E0E0932C06E0E0F0E0E093160881
:10451E00F0931708E091590CE03021F0E0911A0C5D
:10452E00EA93DADDE0911D08EF5FE0931D08E0915C
:10453E00E30BA0911D08EA1751F4E091E30BF0E0B4
:10454E00A0E0B1E00E94E27BEA1BE0931D08A0917F
:10455E001908A13019F0A93009F096C0A091620B8C
:10456E00B091630BE4E1F0E00E94787B309719F490
:10457E00E1E0E0931F0846DFE03019F04EDFE0780F
:10458E0009F462C04ADFEF775E2F5A930E945C19DE
:10459E000E945E6DED55F94F5081503011F40C9420
:1045AE002B2364DDE13031F4E0911A08EA937ADDD1
:1045BE00E03009F449C00E947C710E94FC6FEC91BE
:1045CE00EC71EC3021F4E0911D08E07851F40E947A
:1045DE008171EC91EA9380DD0E948671EC91EA93F1
:1045EE007BDD0E948171AC91A63070F5A3EEB6E032
:1045FE000E945E6D0E940D6E0E94AF6E0E948171D0
:10460E00EC91EA9383DD1E2F1130F0F00E948B7136
:10461E000E948E71CF010E948B710E940D6E6D9162
:10462E007C91E12F0E945671EF5CF94F0E949371BD
:10463E00E60FF71FDC01ED93FC93E12F0E945671FC
:10464E00EF5CF94FA0E0A08310E01530E8F40E9473
:10465E00967113965C915F3FA9F05A9372DE5E2FAE
:10466E000E94A0710E948B710E948E71BF010E94E8
:10467E008B710E940D6E0E94A671AE81BF81129643
:10468E00E0E0EC931F5FE1CFA0911908A23039F062
:10469E00A83029F0A53019F0A73009F0E4C1E0E008
:1046AE00E093200800E0053010F00C943A25A3E2C8
:1046BE000A9FF001ED55F94FEA87FB87AA85BB8566
:1046CE00AC91A03019F0A281A07809F0CAC1E09196
:1046DE002008EF5FE0932008AA85BB8513960E9401
:1046EE00BF7B309771F0AA85BB8513960E94B3717C
:1046FE000E94B97129F4AA85BB8513960E94257173
:10470E00B0C180DEE03021F00E94B97109F4A9C178
:10471E0020E030E0333010F00C94E7240E94C17199
:10472E00DF010E94ED6C0E94E16DE887F987A1819F
:10473E00A27021F4A481B581109709F40CC1E8850B
:10474E00F985A181A47011F40C940D24A181A87097
:10475E0021F40E941C34E03009F457C00E94C77146
:10476E00EBE0EC93A885B9850E94D471A885B98534
:10477E001396EC91AC85BD851796EC93EC85FD8573
:10478E0038960F01E885F985A181E1E0EA230E94C0
:10479E00DB71ED93FC93A885B98514960E94BF7BBF
:1047AE00AC85BD851296ED93FC930E94DE71AC85AF
:1047BE00BD851496ED93FC93A02FEAE0EA9FF001DD
:1047CE00E30FEF5F0E94E471E885F985A085B1855E
:1047DE00E2E0F0E00E941B7BA885B9851896ED9368
:1047EE00FC930E94DE71309739F4A885B98518962E
:1047FE00E8EEF3E0ED93FC93E885F985A181E8E01E
:10480E00EA2BA885B9851196EC936CC0E885F985DD
:10481E00A181A17031F4A885B98514960E94B37157
:10482E0041C00E94ED7172DCE1501E2F0E94967104
:10483E001296EC91E030F1F4AE81BF8153960E9456
:10484E00AF6EEE81FF81A189B289109751F0038876
:10485E001488AE81BF8151960E94BF7BE015F10591
:10486E000CF007C00E94F27111F00E94F7710E94C5
:10487E00FF710EC0E885F98534960E9407720E947A
:10488E00DB710E94C0700E940F7253960E942571B8
:10489E00E885F985A581AA232AF4A885B9851496F9
:1048AE000E942571A885B985EC91EC71EC3021F44C
:1048BE00E0911D08E078B1F4E885F985A481B58111
:1048CE005E971CF4A181A07209F404C0E885F985F5
:1048DE00A28106C00E94ED71FFDBE885F985A381F8
:1048EE00AA93FADB0E94DE71309781F0A885B98514
:1048FE0018960E94B3710E94DE71309739F40E94AF
:10490E00F27111F00E94F7710E94FF710E94ED7119
:10491E0019DCE03001F10E94F27159F00E94F7713A
:10492E00AA85BB85EC91E150ADE0EA9FF0010E94B3
:10493E00666DAA85BB851296EC91E058AA85BB855B
:10494E001296EC93E3E0E09324060E94ED71ECDB0B
:10495E00EF73E0932506A885B98514960E94BF7B58
:10496E00309761F52F5F323048F5A885B9851696D8
:10497E000E94BF7B309789F0E885F985A681B781C3
:10498E000E941672AA85BB851396ED93FC93A8859B
:10499E00B98516960E94257111C00E94C171DF0162
:1049AE00E32FEF5FF0E00E94E16DE887F987A181C8
:1049BE00EDEFEA23A885B9851196EC933F5FAACE59
:1049CE00233011F00C9438250E94F27111F00E94E0
:1049DE00F7710E941C34E03069F00E94C771E8E064
:1049EE00EC93AA85BB850E94D471AA85BB85EC91F8
:1049FE000E94E471AA85BB85E0E0EC93EA85FB8515
:104A0E00A581ECE1EA23E83061F50E941F6EAE2F1E
:104A1E00EA85FB85E38DEA1741F4EA85FB85E48D93
:104A2E00E150EA930E945D181CC00E941C34E030D5
:104A3E00C1F00E94C771E3E0EC93AC85BD85EFEF4A
:104A4E00EC931896EA85FB85E38D0E941B72AC856C
:104A5E00BD851296EA85FB85E48D0E941B720E942D
:104A6E001F720F5F20CE0E94257249F4A091190883
:104A7E00A23021F0A83011F0A53009F401C050C0C9
:104A8E0010E0153010F00C9497250E949671139635
:104A9E005C915F3F11F40C9495250E94A071AE813C
:104AAE00BF81BD010E94A671EE81FF8138960E94E2
:104ABE0007720E942B720E940F720E94BF7BDF0151
:104ACE000E94977DB4F4EE81FF81A681B7810E948A
:104ADE00977D7CF4AE81BF810D901C90AE81BF811D
:104AEE0016960E94BF7BD001AE1BBF0B0E94977D16
:104AFE000CF014C0AE81BF81BD010D901C90EE81F3
:104B0E00FF81A681B781F001EA1BFB0BDB01ED9360
:104B1E00FC935A93E5E0EA930E9467431F5FB1CF7F
:104B2E00E0911C08E03041F4E0911608F09117086E
:104B3E00E0931408F09315080E94A87D2E96089510
:104B4E000E94A37DA091C10BE091C20BE150EA9FA0
:104B5E00F001EF5F1E2F2FE330E000911E08A091B1
:104B6E00180CA13080F0E091180CE150A0911E08B5
:104B7E00AE1728F0E091180CE1503E2F04C0E091E2
:104B8E00180CE2502E2FEC81E03049F1EF3F51F43A
:104B9E00A0911E08A11BA31720F0E0911E08E11B97
:104BAE000E2F1DC0EE3F59F4E12FA0911E08AE0F3F
:104BBE00A21720F4A0911E08EA0F0E2F10C0EC3F92
:104BCE0049F4A091180CA13020F0E091180CE1509E
:104BDE000E2F05C0AC81A1501A9FF0010E2FE0914F
:104BEE001E08E01751F00A930E945C19A0918A0BDF
:104BFE00AD3209F4032F00931E080E943C47A0918A
:104C0E001908A83019F40E94001002C00E947B0FF0
:104C1E000E94AA7D259608950E94A17D16DAE031A4
:104C2E0011F40C94872620E030E040E050E010E0D4
:104C3E00133060F50E942F720E940D6E0E94BF7B92
:104C4E00309711F10E9432720E9441712E2B3F2B30
:104C5E000E943272EA9376DAE03029F0E3E0E093D4
:104C6E002406E0E04EC00E9439720E9441712E2B44
:104C7E003F2B0E943972EA9365DAE03029F0E3E0C7
:104C8E00E0932406E0E03DC01F5FD2CF00E0053088
:104C9E0068F5A3E20A9FF001ED55F94FE081E0308F
:104CAE0019F110E0133000F50E94C171DF010E946E
:104CBE0074710E944072AE0FBF1F1296EC910E944B
:104CCE0041714E2B5F2B0E94C171DF010E947471E6
:104CDE000E944072AE0FBF1F1396EC910E9441715D
:104CEE004E2B5F2B1F5FDECF0F5FD1CFF901E42379
:104CFE00F523309729F0E1E0E0932406E0E001C0CF
:104D0E00E1E00E94A87D269608951A93E0914F0C3B
:104D1E00E03011F40C94D326E091E40BE13059F419
:104D2E00A0914F0CA13311F4EFE001C0E0E0EA9343
:104D3E000E94C15E31C0E23059F4A0914F0CA133F4
:104D4E0011F4E6E001C0E5E1EA930E94C15E24C0E1
:104D5E00E330B1F410E0173040F40E947471E05C5F
:104D6E00F64F0E9447721F5FF6CFA0914F0CA133F2
:104D7E0011F4E1E301C0E0E3EA930E94C15E0CC0CE
:104D8E000E944B72E9E4EA930E941663E0914F0C85
:104D9E000E9452720E94577285C422970E94A17D72
:104DAE0030E0A0911908A23029F0A83019F0A530F2
:104DBE0009F014C1A985A03410F00C94F427E091E9
:104DCE002F08E03009F40AC1E9850E940070E03135
:104DDE0031F4E1E3E0934F0C98DFE1E0FFC046D9F8
:104DEE00E03009F4FBC010E0153058F40E946271F7
:104DFE00E081AE2FE885EA1711F4E0E0EFC01F5F07
:104E0E00F3CF0ADFE03011F40C94F42710E00E9487
:104E1E006271EE83FF83AE81BF81EC91E03011F0C1
:104E2E000C94ED2713960E94257100E0033010F0CC
:104E3E000C94BD27A3E21A9FF001E855F94FDF014C
:104E4E000E94D56C0E94E16DAF01DA0116960E94A8
:104E5E0025710E945C72DA011296EC930E946372C5
:104E6E00DA011396EC93A0919A0BEEEFEA23DA0196
:104E7E00EC930E946A72DA011196EC93E6D8E43153
:104E8E0039F0FA01A181E2E0EA2BDA011196EC93F6
:104E9E000A9308D9E03011F40C949F27FA01A281ED
:104EAE00AA9334D9E1502E2F2F3F81F0A7E12A9FEC
:104EBE00F001EF5CF94FA0E0A083A7E12A9FF0017B
:104ECE00EE5BF94FA0E0B0E0A083B1830E94727256
:104EDE000E940D6E0E94BF7BDA011496ED93FC9337
:104EEE00013040F00E9472720E940D6E0E94BF7BD4
:104EFE00309709F00EC0AE81BF811596E02F0E944B
:104F0E00AD6F0E944072AE0FBF1F1196EC91E06222
:104F1E00EC93AE81BF815A96EC91E062EC93023035
:104F2E0030F40E947572DA0116960E941B7204C04C
:104F3E00DA0114960E94257188D8EC3019F4E0E05D
:104F4E00E0931D080E947C720E941A70DA01189676
:104F5E00ED93FC93FA01A281A63030F0A181E4E03A
:104F6E00EA2BDA011196EC930F5F60CFA09119082E
:104F7E00A23011F0A53019F4A885AF3F08F007C094
:104F8E00E0912F08EA93EA85EA930E94911AE88548
:104F9E00AE81BF81EC93E0912F08AE81BF81119657
:104FAE00EC93E985AE81BF811296EC93A885A4316E
:104FBE0030F4E885E1500E948372A1E0A083AE81B7
:104FCE00BF811696EC91ED7FEC9331E01F5F303090
:104FDE0011F4153008F001C01ACFE32F0E94A87DFE
:104FEE002A9608951A930A93A0911908A23011F0E7
:104FFE00A53049F4EA810E948372A0E0A083EA8181
:10500E00EA930E94CA6EA0911908A830F1F4EA81C1
:10501E000E948372A0E0A083EA81EA93E1E0EA9322
:10502E000E949E47E091E20BE03069F4EA810E9413
:10503E008972E081EF771E2FABE01A9FF001EA51E3
:10504E00FA4FA0E0A083689420F819810881239676
:10505E00089564970E94096DA23039F4E0912F08EB
:10506E00EA93EB8DEA930E94911AA0911908A83049
:10507E0011F00C94A6280FEF20E0253050F4A7E194
:10508E002A9FF001EE5CF94FE081AE2FEA8DEA1710
:10509E0009F402C02F5FF1CFA7E12A9FF001E15D75
:1050AE00F94FAF01DA0115960C910F3F11F40C94E4
:1050BE00A6280E948F7210810E94F9700E94977D1F
:1050CE00ECF4ACE2BCE00E94B3710E9495720E94B7
:1050DE00D070A083B1831A930E94411FABE00A9F48
:1050EE00F001E252FA4F30810A93FE0137960E9488
:1050FE009B723A93FE0137960E949F720E94A57290
:10510E00F1F40E948F72AFEFA083DA011396EFEFE6
:10511E00EC93DA011596EC930E9495720E94AB7295
:10512E00E0E0F0E00E94DE70E0E0E093290C1A93DC
:10513E000E94411F0A930E946411689420F80E94F5
:10514E00A87D6B9608951A9310E01031B0F4A7E184
:10515E001A9FF001EC5BF94FE081EF73AE2FE981FE
:10516E00EA1729F41A930E94A920E03009F403C02B
:10517E00E1E01881E0C01F5FE8CFE0E01881DBC0FE
:10518E001A93E091520CF091530CFA93EA93E4EFD8
:10519E00F1E00E94ED70F9F00E94B07210E015304F
:1051AE00D0F4A091560CAF5FE5E00E94757BE093C2
:1051BE00560CEF5FEA93C7DFE03059F0E3E0E0937F
:1051CE002406E091560CF0E0EF5FFF4EE0932506CB
:1051DE0069C21F5FE4CF66C21A93E0912306E09383
:1051EE004E0CE8E7F0E0FA93EA93ECEDF0E0FA9378
:1051FE00EA930E946D4710E01530D8F4E12FEF5F6F
:10520E00EA93A1DFE03099F00E94526CE12FEA5F41
:10521E00F0E00E941B6EE7E0F8E10E94B96DA6EE89
:10522E00BBE00E9474710E94E16D0E94E96D1F5FE8
:10523E00E3CF38C2A5DFE0912406E13029F4EFE098
:10524E00F8E10E94B7723CC0E23029F4ECE1F8E1DB
:10525E000E94B77235C0E33051F4E7E0F8E1FA93FB
:10526E00EA93E0912506F0E0E050F04F29C0E430DB
:10527E0019F4E4E2F8E11FC0E53031F4E0912506BF
:10528E00EA930E94CB1120C0E63019F4ECE2F8E16B
:10529E0012C0E73029F4E2E3F8E10E94B77210C0C1
:1052AE00E83029F4EEE3F8E10E94B77209C0E93064
:1052BE0059F4EDE4F8E1FA93EA93E0912506F0E073
:1052CE00FA93EA930E94E811E0E0E0932406089531
:1052DE00A881B9811196E1E0EC930E94FD70A8813E
:1052EE00B9811296ED93FC930E943120A881B98169
:1052FE001796EC930E941F6EA881B98118960E9492
:10530E001B72E091C605A881B981EC93E091290C3E
:10531E00A881B9811696EC93E091890BA881B98189
:10532E001A96EC93E091AC0BF091AD0BA881B9817C
:10533E001496ED93FC932296089564970E94A37D94
:10534E00A091E20BA230E1F4EB8DEA930E945C197E
:10535E000E943120ACE2BCE00E941B72AAE2BCE0CB
:10536E00EB8D0E941B72E0912F08E093290C0E9496
:10537E000570309721F00E9405700E94E87014C0ED
:10538E00AA8DAF3F09F4CAC0EA8DEA930E943A1F74
:10539E00AB8DAF3F29F40E94FD700E940A70EB8F17
:1053AE00EB8DEA930E945C190E9431200E2FA98D7D
:1053BE00AF3F21F00E943D20E03009F001C0AEC0A9
:1053CE000E94D0700E94D56CAE17BF071CF024DC73
:1053DE00E13009F0A3C0A091D10BA03021F4A0912F
:1053EE00E20BA23011F50E941F6EE13041F00E94D7
:1053FE001C34E03021F00E943234E03009F002C05B
:10540E000E94BC720E941F6EE13021F40E94223471
:10541E00E03009F409C00E94C872EE55F84FFA93B5
:10542E00EA9356DF0E94CE7277C0EB8DEA93EA8D37
:10543E00EA93B3DC1E2F113011F00C94932AA09135
:10544E00D30BA13059F4E0912F08EA930E94FD701E
:10545E00FA93EA93EFEFFFEF0E94D4720E94D0709E
:10546E000E94D56C0E94C0700E94DE70689420F875
:10547E00A091E20BA03019F4A88DAF3F09F437C00C
:10548E000E94D872EE51FA4F0E94D070A083B18361
:10549E00E88D0E94C26D3081E88DEA93FE0135964B
:1054AE000E949B72E88D0E94C26DE081EA93FE011C
:1054BE0035960E949F720E942C20E03131F00E949E
:1054CE00D872EA51FA4FA1E005C00E94D872EA5193
:1054DE00FA4FA2E0A0830E94D872EC51FA4FFF93CC
:1054EE00EF930E948868AF91BF91ED93FC930E9459
:1054FE00A57219F4E0E0E093290CEA8DEA930E947C
:10550E00411FE0912F08EA930E9405700E94DD7200
:10551E00FA93EA930E942F1DE1E001C0E0E00E94A1
:10552E00AA7D6C96089578DBE13041F40E941C341C
:10553E00E03021F00E943234E03009F007C00E94C2
:10554E0005700E94E8700E94BC7226C32EC30E9492
:10555E00A37D0E94E0721F3F11F40C94052BE09185
:10556E004F0CE03011F00C94042B1A930E945C192E
:10557E00E5E0E093240610932506A0911908A230C9
:10558E0031F40E94E9720E94EB21E03009F010C064
:10559E00A091500CA13331F4E0912F08EA931A93A5
:1055AE000E94911AE1E3E0934F0C0E94AA7DE2C2A1
:1055BE00A0911908A830A1F40E9405700E94ED7206
:1055CE000E2F0A930E9492343E2F1A930A93EFEFF6
:1055DE00EA933A93B2DEE03019F00E94AA7DCAC275
:1055EE00A0911908A53031F49EDFE03019F00E9429
:1055FE00AA7DC0C2E0E3E0934F0C06C0E0E3E09367
:10560E004F0CE4E0E09324060E94AA7DB3C2E09121
:10561E0040090E94F17208951A93E6E0EA930E94FF
:10562E00C15E0E944B72A0914009A83539F4E9E59C
:10563E00F8E10E94FD72E0E00E945772A0914009CD
:10564E00A33509F510E0A0911908A83021F0A23079
:10565E0011F0A53009F411E3E3E5EA930E94166315
:10566E001A930E941663E0E8EA930E941663E0E83C
:10567E00EA930E941663E0E80E945272E0934F0C88
:10568E00E0E00E945772A0914009A93459F40E949B
:10569E000173E09325060E940B73EC91E093500C7E
:1056AE0056DF33DB199108950E94A37DA0913F0927
:1056BE00A53411F00C94A22B0E941073E2E3F0E0DB
:1056CE00E093490CF0934A0CA0914009A73741F49E
:1056DE00E4E4F9E00E9417730E941C730E94F172B9
:1056EE00A0914009A03310F0AA3308F023C02091F6
:1056FE00270830912808E0E4F9E00E941773E2E0F1
:10570E00EA930E94BC620E2F0E941C73E093250642
:10571E000E941C730E9420730E94E0720A931A93D7
:10572E000E94911A2093270830932808E2E5EA9305
:10573E000E94C15E1CC0E091470CF091480CFA9398
:10574E00EA93E091490CF0914A0C0E94ED7079F0C9
:10575E00E0E0E0933A09E5E4EA930E94C15E0E941C
:10576E001073E8ECF0E0E093490CF0934A0C0E94C1
:10577E00AA7D00C20E9425730E942B730E94526C58
:10578E000E94526C0E941547A0911B08A23021F472
:10579E00E1E6F8E10E94B96DA0911B08A13021F459
:1057AE00E8E6F8E10E94B96DE0911B08E03021F4C3
:1057BE00EFE6F8E10E94B96D0E9435730E94936C7A
:1057CE000E9415470E9438730E943D73FA93EA9324
:1057DE00E0915F05F09160050E9443730895E1E04A
:1057EE0003C0E0E001C0E2E0E0931B08C3DF0895D0
:1057FE000E942C20EC3109F0D8C1E091990BE336D0
:10580E0031F4A0911908A23009F4EBDF17C0E2368B
:10581E0031F4A0911908A23009F4E5DF0FC0A09170
:10582E00C505A23011F0A63021F4E091990BEA9350
:10583E0087D9A091C505A43009F4D1DFADC10E946E
:10584E00EF6D0E94526C0E94F36D0E94526C0E948A
:10585E00526C0E941547E8E7F5E00E94B96DE091A1
:10586E001A080E944773E6E8F5E00E94B96DE2E07F
:10587E00E0930E0408950E943070E0ECF0E00E9478
:10588E003770E881E03009F406C0A0911A08AF5FC6
:10589E00E3E00E94757BE0931A08E1E0E0934B0C85
:1058AE000E94D32072C20E94A37D10E0103410F02B
:1058BE000C94A72C0E947471ED55F94F30813F3F27
:1058CE00E9F11A930E945C1900E00E944B730E944A
:1058DE000D6E0E94BF7B3B9794F00E944E730F019A
:1058EE000E944B730E940D6E0E9454730E945A7355
:1058FE000E94FC6FEC91EE7FD001EC9301E00E94D0
:10590E005F730E940D6E0E94BF7B759794F00E948C
:10591E004E730F010E945F730E940D6E0E945473AE
:10592E000E945A730E94FC6FEC91E160D001EC93DF
:10593E0001E0013019F41A930E947C191F5FB6CF53
:10594E000E94AA7D17C11A930A9323FE03C00E94D8
:10595E0062733FD70E947743E030C1F1E0E00E94CE
:10596E006973103820F5113219F40E94627331D721
:10597E001D3439F40E9470730E942C64E3E0E093AE
:10598E0018081B3271F40E947573EAE2EA93EAE793
:10599E00F8E1FA93EA93E0911A08E05DEA930E9427
:1059AE002C641F3219F4E1E0EA93CAD848DF1038AC
:1059BE0068F00E947B731A930E94A82119DFE030D1
:1059CE0011F4103208F002C0E4EDF6E20E94142247
:1059DE000E2F0038C8F10F770034A8F5E0911F089C
:1059EE00E03031F00A930E943912E0E0E0931F0894
:1059FE00E091570CE01739F10A930E945C190E944E
:105A0E008171AC91A83028F40E948671AC91A830B7
:105A1E00A8F0E02FEF5FE093A2060A930E94A82160
:105A2E000E948171EC91EA930E948671EC91EA9347
:105A3E00E091A206EA930E94C21F03C0E0E0E09349
:105A4E00A2060093570C0EC0A091570CAF3F51F019
:105A5E00E091A206E03019F0EA930E94DF1FEFEF0B
:105A6E00E093570C099119910895A881A03310F075
:105A7E00AA3308F01DC00E947F730E948473AAE0AF
:105A8E00B0E00E941B7BDF01E8810E948973EA0F60
:105A9E00FB1FE0932508F0932608E2E0E0930E0446
:105AAE000E9435730E94936C0E94F36D0E943873AE
:105ABE00A881A33451F40E942B730E9435730E9467
:105ACE00936C0E94F36D0E9438735FC11A930A9310
:105ADE00A0E023FCA1E0A03019F0AA81A03009F0CB
:105AEE0016C0E89423F8E7E0E09318080E945C469D
:105AFE00A0913108A03019F40E948C7309F407C0EC
:105B0E00E7E0EA930E94917364D6E89424F824FEA9
:105B1E0024C00E949473EAE5F0E00E949B7319F092
:105B2E00AA81A130C9F481D6E030B1F00E94A173F0
:105B3E000FEF1FEF0E94E9720E94C221E03021F4A4
:105B4E000091270810912808EB81EA93E0912F0825
:105B5E00EA931A930A933DD60BC00E949473ECE21B
:105B6E00F1E00E949B7321F40E94A873E093300829
:105B7E001981088124960895E091C70BF091C80B06
:105B8E000E94AC7311F4E2E00895E091C50BF09120
:105B9E00C60B0E94AC7311F4E1E00895E091CB0BBB
:105BAE00F091CC0B0E94AC7311F4E0E00895EFEF8E
:105BBE000895A0911908A23021F40E943C470E943A
:105BCE007B0FA0911908A83009F462D6A09119088C
:105BDE00A53009F449D1D9C0E2E0EA930E944341CD
:105BEE00E2E0E0930E04E881EA933FDFA881AF374D
:105BFE0021F4E0912B06E37009F403C0E2E0E09398
:105C0E001808A881A13239F0A33421F40E947F73C1
:105C1E00109709F004C0A0911908A23009F011C024
:105C2E00A0911B08A33009F4DEDDA0911B08A23061
:105C3E0019F4E1E0EA93BDDFE0911B08E03009F4CE
:105C4E00D0DDA881AD3311F00C94882E0E945C46F5
:105C5E00E0911B08E030B1F4E0912508F0912608A0
:105C6E00FA93EA930E94EB21E03051F4E09125087B
:105C7E00F09126080E942073E0E0EA939ADF01C0BB
:105C8E00B0DD3FC0E13079F477DFEF3F41F0E3E084
:105C9E000E94B0730E9470730E94B67303C0E1E05D
:105CAE00EA9387DF2EC0E230F1F40E947F73A034B6
:105CBE00E0E0BE07B4F4E0912508EA930E94BD73BC
:105CCE00E2E0E0930E040E94526C0E94526C0E941D
:105CDE0015470E94AC6D0E94CC10E3E0E0931B08C8
:105CEE0001C081DD0EC0E33061F4E0912508EA9336
:105CFE000E945C19E0912508EA93EEEFEA934DD8E5
:105D0E0072DDA881AD3409F46ADDA881A43521F4D1
:105D1E00A0911908A23009F001C063DDA881AB3251
:105D2E0021F4EEEFEA930E94A725A881AD3221F46B
:105D3E00EFEFEA930E94A725A881A73421F4E1E0B2
:105D4E00EA930E94A725A881AB3421F4ECEFEA93E5
:105D5E000E94A7251AC00E944B210E943C47E0E0FA
:105D6E00E0931B08A881A13039F40E948C7321F0B6
:105D7E00A091CA0BA03009F402C033DD06C00E9408
:105D8E007B0F0E94E9720E94C221219608951A93F8
:105D9E000A930E94C1730E940C200E947743E03048
:105DAE0091F10E94CA7378F10E947B7321DDE0307D
:105DBE0051F50E94D2730E948421EF3F09F006C56F
:105DCE000E94E9720E94EB21E03021F40E943D20F6
:105DDE00E13009F018C00E942C20E83119F40E941D
:105DEE00D77309F001C0F2C40E94D2730E94D42668
:105DFE000E2F013021F4A091990BA03009F403C0AD
:105E0E001A930E94CB11A0912E06AF3F61F1109113
:105E1E002E06EFEFE0932E061A930E945C190E9455
:105E2E00E9720E94EB21E03021F40E943D20E13026
:105E3E0009F019C00E942C20E83119F40E94D77382
:105E4E0009F001C0C3C41A93EEEFEA930E94D42660
:105E5E000E2F013021F4A091990BA03009F403C04C
:105E6E001A930E94CB11B2C40E944B210E94D320E0
:105E7E00E89421F8E0E0E0931E080E94DE730E9491
:105E8E003C470E94526C0E94526C0E941547E09152
:105E9E0032060E94306EE09133060E94306E0E94F0
:105EAE00526C0E94B46D0E941547E0913F060E940D
:105EBE00306EE0913906F0913A060E94066E089512
:105ECE000E94A37D0E94C1730E947743E03049F087
:105EDE000E94CA7330F00E947B738ADCE03009F4B2
:105EEE0022DBE091540CF091550C0E94CE6E11F411
:105EFE000C94E12F0E94DE730E94526C0E94A76DDB
:105F0E000E94F36DE0913706F09138060E94066EFE
:105F1E00E0913B06F0913C060E94066E00E00530D3
:105F2E0010F00C94E12FA7E10A9FF001E15DF94F0B
:105F3E009F01F901A381AF3FD9F1D9011A960E94B1
:105F4E00126E7F936F93FF93EF930E94E573AF9161
:105F5E00BF918F919F910E94DD7A0E94207BDF017D
:105F6E00CB010E94EA73D9011C96ED93FC93F901C3
:105F7E0004841584D9011E960E94BF7BE015F1059D
:105F8E00B9F0F90104841584A685B785F001EA1BE2
:105F9E00FB0BE093AC0BF093AD0BC5DAE13041F4A3
:105FAE00D9011C960E94BF7BD9011E96ED93FC93DE
:105FBE000F5FB5CF0E94AA7D2AC40E94A37D0E94C6
:105FCE00C1730E940C200E947743E03011F40C94B0
:105FDE007A300E947A430E2F0A93FEDD003820F0AD
:105FEE00A091C605A03808F429C00F770A930E9425
:105FFE00F1730E94ED721E2FA091E20BA03011F4EE
:10600E001F3F09F416C030E0353098F4ABE03A9FEC
:10601E00F001E452FA4FE081E11749F43A9FF001A2
:10602E00E252FA4FE081EF5FE093C605232F3F5F08
:10603E00EBCF0A930E94D2732A9354C0A091E20B25
:10604E00A03021F4003810F0053808F00AC00F77A0
:10605E000E948F721081EFEFEA930E94D2730A931F
:10606E006CD9A091E20BA03011F0003808F43BC0BF
:10607E000F770A930E945C19BBDBE030A1F50E94FA
:10608E00F4730E948421EF3F19F00E94AA7DBFC3D2
:10609E000E943D20E13039F50E943120E03049F474
:1060AE000E94F4730E94D426E03011F00E94F9731E
:1060BE001AC00E942C20E83141F40E94D77321F0BF
:1060CE000E94F4730E94D4260EC0A0911E08E02FE9
:1060DE000E94866DAE0FBF1F1C910A930E94D27351
:1060EE00EFEFEA932AD9A0912E06AF3FF9F0009177
:1060FE002E06EFEFE0932E060A930E94F1730E9494
:10610E00ED721E2F0A931A93EEEFEA93EFEFEA93D6
:10611E0014D91F3F41F4A0919D0BA03021F4A09102
:10612E00A00BA03009F002C00E94F97320FE0AC035
:10613E00E89420F8E091E20BE03019F4FFD350D54B
:10614E0001C0AFD530E0353080F5ABE03A9FF001BD
:10615E00DF01EA51FA4FE081E03049F0AC51BA4F1D
:10616E000E94FF73E8EEF3E00E94ED7099F4ABE04D
:10617E003A9FF001EA51FA4FE081E23051F43A9F32
:10618E00F001EC51FA4FDF010E94BF7B0E94CE6EF0
:10619E0009F409C0ABE03A9FF001EA51FA4FA0E0D2
:1061AE00A083689420F83F5FCECF0E94AA7D2FC3B4
:1061BE000E94096DA33011F40C949832E0913A08C4
:1061CE00ED3411F00C94C131E0913B08EA3511F039
:1061DE000C94763124FC83C0E0913C08E0532E2FC2
:1061EE00E0913D08E0533E2FEEE3F8E00E94177376
:1061FE000E940B73AC91AB3429F40E9404740E947C
:10620E0048620E2F0E940B73AC91A43529F40E94A4
:10621E0004740E944862AF01E091CD0BE31731F593
:10622E00E0E0E0934D0C0E94A17340932708509339
:10623E002808A09130080A1759F0E7E0E0931808F3
:10624E000093300820934C0CE0E0E0932F080DC033
:10625E00A0914C0C2A1721F0A0912E08A03009F025
:10626E0004C02093180820934C0C35C0A091300820
:10627E00A03049F4A091CE0B0E94ED6CE255FF4F79
:10628E00E491EA2309F40CC0E7E0E09318082093A8
:10629E004C0CE0E0E0932F08E0913908E0934D0CB0
:1062AE00E0913908A0914D0CEA17A9F44093270804
:1062BE0050932808009330080E94A173A0914C0CB3
:1062CE002A1721F0A0912E08A03009F004C02093C7
:1062DE00180820934C0C273011F40E941271E09193
:1062EE003B08E93439F4E7E00E94B0730E94A873CA
:1062FE00E0932F08E0913B08E23439F4E4E00E9489
:10630E00B0730E94A873E0932F08E0913B08E0352C
:10631E0019F4E1E0E0931808E0913B08EC3449F4FD
:10632E00E4E0E0931808E0913C08E053EA930E9401
:10633E009516E0913B08E334E9F4A0913C08A133B3
:10634E0020F0A0913C08A93308F014C00E940774F5
:10635E00E0912208EA930E94AC1BE0913908EA937F
:10636E00E6E8F8E1FA93EA930E943B700E94D27B32
:10637E000E941F64E0913A08E03521F4A0911908BB
:10638E00A13009F003C00E94757359DAE0913A0802
:10639E00EF3459F4E0913B08EE3439F4E0913908CA
:1063AE00EA93E9E8F8E10E940D74E0913A08E335CA
:1063BE0069F5E0913B08EF3349F5A0913C08A03315
:1063CE0020F0A0913D08A03308F420C00E9407746D
:1063DE00E0913D08E0531E2FA0912208A63010F444
:1063EE001A3008F013C0103011F40E94F61AE09122
:1063FE003908EA93ECE8F8E1FA93EA930E946E709A
:10640E000E9451700E94D27B0E941F64E0913A0854
:10641E00E33411F00C946032E0913B08EF3311F04D
:10642E000C946032E0913D08E03319F4EFEFE09305
:10643E002308A0913C08A033F8F00E940774A091A5
:10644E002208A630C8F4E0912308EF5FE0932308FA
:10645E00E0912208EA93E0912308EA930E94721BCE
:10646E00A0911E0CB0911F0C109721F4A09123083F
:10647E00A03408F001C0E7CFE0912308EA930E9410
:10648E005C190E941374EFE8F8E10E94FD720E94FD
:10649E00116F0E9418740E941D740E94166F0E9444
:1064AE00D27B0E941D740E94786F0E94A0630E948E
:1064BE00EF63E0913A08E434A1F5E0913B08E4344F
:1064CE0081F514E0E1E0E0933909103538F40E94CB
:1064DE007471E85CF74FE081E03208F41AC00E9454
:1064EE007471E85CF74FE081E33259F40E947471E5
:1064FE00E75CF74FE081E053EA930E94C15E1F5FB5
:10650E0006C00E947471E85CF74F0E9447721F5FCD
:10651E00DCCF0E941374E2E9F8E10E94FD720E9442
:10652E00EF630E94A87D269608951A930A930E94FF
:10653E00257211F40C941833E0E0E093590CE091BD
:10654E001808EF770E2F009318080E943C470E9400
:10655E00B46DE4E0F0E0FA93EA930E94154701303F
:10656E0021F0A0911908A13009F00BC0EEE8F5E07A
:10657E000E94B96D98D9E4EFF1E00E946F6C0E9411
:10658E003C47073049F40E944B21E0E0E0931B08A2
:10659E000E946C120E94F328043031F4E5E9F8E110
:1065AE000E94B96D0E94300E083019F40E942374B7
:1065BE006FD1053019F40E94237456DC013051F46A
:1065CE00E89423F8E0E0EA9356D90093190837D9F6
:1065DE000E947B0F093071F4E0E0EA934CD9E0E0C1
:1065EE00E0931E08E89423F80E947B0F0E942D74FE
:1065FE00E093590C023069F4E0E0E0931E08E0E00D
:10660E00F0E00E942073E89423F80E942D74EA9320
:10661E00A2DB033011F40E94F540009319080E948A
:10662E000C20A0911908A73011F00C94C633E091FC
:10663E00520CF091530C0E94CE6E21F0A0911B08CB
:10664E00A03009F00AC00E94B072E0914E0CA091E9
:10665E002306EA1711F00E94F3280E947743E030D8
:10666E00E9F0E2E00E9469731A93FFD91D3409F430
:10667E00B6D81D3399F40E945C467EDAEF3F41F0A6
:10668E00E3E0E09318080E9470730E94B67306C090
:10669E00E7E8E0931808E0E0E0931B08A0912F08CC
:1066AE00A03031F0E0912F08A0912E08EA1709F4DE
:1066BE0057C0E0912F08E150EA930E94B119A091C2
:1066CE00340CE1E0EA23E13021F4E0912B06EF7C7B
:1066DE0009F429C0E0E0E0932E08E0914C0CE03084
:1066EE0019F0E09318081EC012E0E0912B06EC7032
:1066FE0009F018E0E091C40BA0912F08EA1781F081
:10670E00E0912B06E07439F011E0EAE2EA93EAE94F
:10671E00F8E10E940D74E0912B06E07809F019E083
:10672E00109318081DC00E943C470E946C120E94D4
:10673E00B46DE4E0F0E0FA93EA930E941547EBE4BF
:10674E00EA930E94B346E0912F08EA930E94E44137
:10675E00EDE9F8E10E94B96DE0912F08E0932E0863
:10676E00A0912F08A03021F4A0912E08A03009F49A
:10677E0006C0E0E0E0932E08E7E8E0931808A09149
:10678E001908A33011F40E94F23EA0911908A1300D
:10679E0009F4D9D8A0911908A23009F4F8DAA09119
:1067AE001908A83009F409DCA0911908A53009F4DC
:1067BE0087DBA0911908A93049F4E0E0E0932008A6
:1067CE00E0911908EA93E0E0EA9380D909911991D2
:1067DE0008950E943474E652F84FA6E0A0830E94FA
:1067EE003474E752F84FAB81A0830E943474E152A7
:1067FE00F84FAA81A0830E943474E552F84FA88105
:10680E00B981A083B1830E941F720E947151249698
:10681E0008950E943A74A881B981AC91A53020F0F8
:10682E00A881B981E0E0EC9387C0A0911308BB2743
:10683E00E091120805C0A0911108BB27E091100845
:10684E00F0E031960E94C0703596DF01E5E0F0E091
:10685E000E94787B08951A9310911308E091120804
:10686E00E117A1F0ABE01A9FF001E652F84FE0817C
:10687E00E13011F0E23011F4E1E04BC0EDB7FEB7BC
:10688E00FA93EA931F93C5DF1F91E8CFE0E041C072
:10689E001A930E944B21ECEDF5E00E9485700E9448
:1068AE00356D0E94E66810E0153068F40E94F370B2
:1068BE00AFEFA083ABE01A9FF001EE51FA4F0E94AA
:1068CE00AB721F5FF1CF10E0153048F4A7E11A9FAD
:1068DE00F001EC5CF94FAFEFA0831F5FF5CFE091B5
:1068EE002B06E37019F00E948C7309F402C06894B1
:1068FE0001C0E89421F8EFEFE0932D08E091E20B50
:10690E00E03029F41BD06CD1E89420F802C00E942C
:10691E000010199108951A9310E0153058F40E9442
:10692E00F370E081AE2FE981EA1711F4E12F03C075
:10693E001F5FF3CFEFEF18812296089522970E94E2
:10694E00A17D00E0053058F40E944074A0E00E9442
:10695E004674E152FA4FA0E0A0830F5FF3CF00E040
:10696E000530C0F50E948F72E081EF3F89F10E94E1
:10697E008F72E0810E940271B9F00E949572DF0160
:10698E000E94BF7B0E94D070EA17FB0751F00E9455
:10699E0095720E94D070A083B1830E944B74A1E0C7
:1069AE00A0830E94407412C0ABE00A9FF001EA512E
:1069BE00FA4FE081E03061F40E948F72AFEFA08356
:1069CE000E9495720E94AB720E944B74A1E0A0834C
:1069DE000F5FC6CF0E942C1F1E2F1F3F11F0E1E04C
:1069EE0001C0E0E0E093590C1F3F11F40C945135B7
:1069FE0050E000E0053048F40E948F72E0811E17CF
:106A0E0011F451E002C00F5FF5CF5030E1F500E018
:106A1E000530C8F50E948F72E081EF3F91F50E941C
:106A2E008F7210830E9495720E94D070A083B183E2
:106A3E00ABE00A9FF001E052FA4FA091290C0E94A0
:106A4E004674EF51FA4FFF93EF930E94FD700E9430
:106A5E000A70AF91BF91EC930E944B74A1E0A0839A
:106A6E000E944074A1E00E944674EC51FA4FFF93CD
:106A7E00EF930E948868AF91BF91ED93FC9351E024
:106A8E0002C00F5FC5CF503029F01A930E94331FFA
:106A9E001E2FAACF30E0353010F00C949735A7E1B9
:106AAE003A9FF001E15DF94FEE83FF8350E000E085
:106ABE00053048F5503029F5ABE00A9FF001EF5153
:106ACE00FA4F20812A930E945C190E944074E08143
:106ADE00E13059F42A930E944D20E13031F4A32F76
:106AEE00AF5FE0919D0BEA1709F00BC0E22FAE816C
:106AFE00BF811396EC93E02FAE81BF811596EC9378
:106B0E0051E00F5FD5CF503049F4AE81BF8113965F
:106B1E00EFEFEC93AE81BF811596EC933F5FBBCF49
:106B2E000E94A87D0C943F380E94A37DAC81BD814C
:106B3E00EBE4EC93EC81FD813196FA93EA930E949B
:106B4E005174E052FA4FE0810E94AD6C00E00E9459
:106B5E005A74EC91E03011F00F5FF9CF0E945A7425
:106B6E00E0E2EC930F5F0E9460740E94616D0E94E0
:106B7E005174EE51FA4FDF010E94126E0E9465743D
:106B8E00EE81ABE0EA9FF001EF51FA4F10811A93BC
:106B9E000E945C1900E00E945A74EC91E03011F0F2
:106BAE000F5FF9CF0E945A74E8E7EC930F5F0E94D3
:106BBE005A74E0E2EC930F5F30E03A3060F40E94DA
:106BCE006074EA0FFB1F0F01AAE8BBE00E946C7411
:106BDE000F5F3F5FF2CF0E945A74EC930C9484388F
:106BEE0064970E94A37D00E010E0153040F40E94EF
:106BFE00F370E081EF3F09F40F5F1F5FF6CF0530B2
:106C0E0021F0A0912D08A03009F406C0E0E0E09339
:106C1E002D08EA930E94191110E0153088F5ABE0AB
:106C2E001A9FF001E152FA4FE081E03039F11A9FDC
:106C3E00F001E352FA4FE081E030B1F01A93FE0119
:106C4E0035960E949B72ABE01A9FF001EF51FA4FFE
:106C5E0030813A930E945C191A93FE013596FA938D
:106C6E00EA930E9474110AC01A930E946411ABE059
:106C7E001A9FF001E152FA4FA0E0A0831F5FCDCF23
:106C8E00053021F4A0912D08A13009F406C0E1E0F1
:106C9E00E0932D08EA930E9419110E94AA7D68962E
:106CAE0008950E94A17DA091E20BA23011F40C94E4
:106CBE001E3A30E0343168F40E9473740E94767488
:106CCE00DA011296E0E0EC93DA01EFEFEC933F5F1E
:106CDE00F1CF0E942C1F0E2F0F3F11F0E1E001C0EB
:106CEE00E0E0E093590C0F3FA1F10E94FD70FA9382
:106CFE00EA930E940C191E2F1F3F31F1A0911E081E
:106D0E00E12FEA1B3E2F3431F8F40E9473740E9477
:106D1E007674FA0132960F01E081AE2F0E947C74D8
:106D2E00B0E0EA0FFB1FD001EC93FA01A281A4366A
:106D3E0020F0DA011296E3E6EC93DA01AC91AF3F64
:106D4E0019F4E02FDA01EC930A930E94331F0E2FF1
:106D5E00CACF0E94AE1530E0343110F00C943D379E
:106D6E000E9473740E947674FA01A381AF3F11F4EE
:106D7E000C943B370E9481740E940070E83139F404
:106D8E000E948174EA930E945318E03009F408C0FF
:106D9E000E948174EA930E945318DA011296EC93C2
:106DAE00A0919A0BA07839F4FA010280DA011196BB
:106DBE00EC91E01509F458C0DA0113962C91ADE070
:106DCE002A9FF001EF5EFC4F0F01DA011296EC9153
:106DDE00D001EC930E948174EA930E946121EF3FEF
:106DEE0029F0ADE02A9FF0010E94666DDA0112963D
:106DFE00EC91E03089F00E948674DF010E94816D73
:106E0E00EC93ADE02A9FF001E25FFC4FDF01E091D1
:106E1E00980BEF70EC9313C00E94816DE03021F45B
:106E2E000E948674A0E003C00E948674A8E0A0832E
:106E3E00ADE02A9FF001E25FFC4FA7E0A0830E9425
:106E4E008174EA930E946121EF3F19F0ECE0E09328
:106E5E000F04DA011296EC91DA011196EC932A9353
:106E6E00E1E0EA930E949E473F5F76CF0C941E3A74
:106E7E00E7E0E09318080E949518A8950E94F31C6D
:106E8E00A8950E94481FA895EFEFE093B20BE093F0
:106E9E00890BE093330CE0932E0CE0932E060E94A8
:106EAE008C74EC7F29F0A8E0B0E0E0E00E94017C59
:106EBE00089524970E94A37D0E949242EAEAF8E187
:106ECE000E9485700E941E430E94BA42E0912208E1
:106EDE00E03061F0E5EBF8E10E9485700E941E4300
:106EEE00E09122080E9491740E9495740E94BA4209
:106EFE000E94F61A00E00A30A0F40A930E948B1941
:106F0E000E949E6FEFE0EA930E94F842E02FA3EA00
:106F1E00B6E00E9499740E9451700E949D740F5F9A
:106F2E00EACF0E94CC42EEEBF8E1FA93EA93EFE05F
:106F3E00EA930E941E430E94DE6E0E949D740E9480
:106F4E00CE420E94BA4210E0103110F00C943B3841
:106F5E000E941F6EE117E1F5E4ECF8E10E948570E6
:106F6E000E941E430E94A26D0E949574E0E0E09381
:106F7E001E08A0911E08A03448F5E0912208EA935D
:106F8E00E0911E08EA930E94721B0E94116F3097C7
:106F9E00B9F0E0911E08EA930E945C190E94116FED
:106FAE00FA93EA930E94A3740E941E430E94786F84
:106FBE00EAE0EA930E94F8420E94166F0E949D74C6
:106FCE00E0911E08EF5FE0931E08D3CF0E94A874D5
:106FDE000E9474710E94567011F00C943938E4ECD2
:106FEE00F8E10E9485700E941E430E94A26D0E94CD
:106FFE0095740E94AC74E0E30E94627029F40E94C2
:10700E0067700E9448629F0100240216030644F531
:10701E000E9404740E9472620E94866E0E94047422
:10702E000E94B4743A932A930E94A3740E941E4342
:10703E000E94B874EAE0EA930E94F842EC81FD8166
:10704E006E817F810E949D740E94AC74E1E30E9468
:10705E00627029F40E9467700E9448629F01D4CF2B
:10706E000E94A8741F5F70CF0E9493420E94AA7D57
:10707E00289608950E94A37DAD81BE812C910E9419
:10708E00BD740E94A26D0E94D56C0E941B6EECE333
:10709E00EA930E94B346EC81EA930E9407472A9333
:1070AE00ED81EA930E948441EEE3EA930E94B34697
:1070BE000E943D730E94DD720E9443730E94C2744F
:1070CE00333409F431E2313320F0EC81E05DE31723
:1070DE0008F407C0E32F0E948973E255FF4FE49135
:1070EE002E273D3311F0313209F401C0CACF3D33A2
:1070FE0019F4AD81BE812C93E32F0E94AA7D2796B1
:10710E0008950E94A17D20E0AF81B8855C910E9418
:10711E00BD740E94A26D0E94D56C0E941B6EE2E0AF
:10712E00EA930E9407475A930E94E4410E943D73DE
:10713E000E94DD720E9443730E94C274303310F0BD
:10714E003A3308F00EC0203009F450E021E0A52FAC
:10715E00EAE00E94757BAAE0EA9FF001E30FE0539C
:10716E005E2F3B3211F4533608F001C05F5F3D32A3
:10717E0011F4513008F401C05150333429F4203049
:10718E0009F431E250E020E03D3319F4EE81E517C9
:10719E0008F005C0AF81B8855C9130E020E03D334A
:1071AE0011F0313209F401C0B4CF3D3319F4AF817F
:1071BE00B8855C93D0C00E94A17D20E0AF81B885D8
:1071CE004D915C910E94BD740E94A26D0E94D56C7F
:1071DE000E941B6EAE81A23051F4E6E0EA930E944B
:1071EE000747FA010E9418740E94C34108C0E5E0E7
:1071FE00EA930E9407475A934A930E94CE410E94F7
:10720E003D730E94DD720E9443730E94C27430333C
:10721E0010F03A3308F01EC0203011F440E050E078
:10722E0021E04031E7E25E0734F0DA01E0E1F7E217
:10723E000E94787BAF01493BEBE05E0724F0DA0158
:10724E000E948473AF01DA010E94C7740E94CC744D
:10725E00D097AD013B3221F44033E5E75E070CF0E9
:10726E0002C04F5F5F4F3D3221F400240416050625
:10727E000CF002C041505040333431F4203009F448
:10728E0031E240E050E020E03D3311F0313209F4BC
:10729E0001C09ACF3D3321F4AF81B8854D935C93F5
:1072AE005AC00E94A17D0E94BD7420E050E04FEFB5
:1072BE000E94A26D0E94D56C0E94D1740E94D4745B
:1072CE00E885EA930E94DF46E52FE10FF0E00E9489
:1072DE00DD720E9443730E94C274303310F03A3351
:1072EE0008F021C03053431729F04F3F09F05F5F7C
:1072FE0020E005C0A22FAF5FEA2FE3702E2FE52FFF
:10730E00AF81B8850E94D9740F01E32FA6ECB6E0C9
:10731E000E949974AE0FBF1FE22F0E94D974E491A0
:10732E00D001EC93432F3B3219F4EE815E1708F037
:10733E0002C05F5F4FEF3D3211F4513008F402C0CE
:10734E0051504FEFEE815E1720F4313211F03D3384
:10735E0009F401C0ADCFE32F0E94A87D29960895B0
:10736E001A930A93A0919A0BECEDEA231E2F00E0DC
:10737E000D3040F40E94DD740E94E174E11711F0AB
:10738E000F5FF6CF0E94DD74EA0FFB1F0E94CE7BCB
:10739E000E94B96DE02F3DC4AAE9BBE00E940A6EBF
:1073AE00AE0FBF1FEC91E17011F4E3E701C0E9E409
:1073BE00EA930E94B346219608950E94A17D0E94F1
:1073CE00BD740E94A26D0E94D56C0E94D174C8DF5C
:1073DE005E2F0E943D730E94DD720E9443730E94D5
:1073EE00C2743D3211F0363311F4503009F401C03D
:1073FE0051503B3211F0333311F45C3008F001C0C0
:10740E005F5FA0919A0BE1E0EA232E2FE52FA0E01B
:10741E00B2E00E9499740E94E174E20FE0939A0B1D
:10742E003D3311F0313209F401C0CBCFE32F0E946E
:10743E00A87D269608950E94A37D0E94BD740E9489
:10744E00A26D0E94D56C0E94D174AAE9BBE0EC81BA
:10745E000E94FC6FEC91E17019F4E1EDF8E102C0CD
:10746E00E5EDF8E1FA93EA930E94CA460E943D7355
:10747E000E94DD720E9443730E94C274303310F07A
:10748E003A3308F00FC0AAE9BBE00E9420700F014A
:10749E00AAE9BBE0EC810E94FC6FAC91E1E0EA2727
:1074AE00D001EC933D3311F0313209F401C0C7CF56
:1074BE00E32F0E94AA7D259608950E94BD6CE1E0FF
:1074CE00EA930E941A0F0E94526C0E94526C0E9404
:1074DE0015470E94786FEAE0EA93E3DEE13209F4A1
:1074EE005FC40E94526C0E94526C0E94F36DE9EDD3
:1074FE00F8E10E94B96DE5E9FBE00E9485705BDE64
:10750E00E13209F44DC40E94526C0E94526C0E94EA
:10751E00F36DEFEDF8E10E94B96DE091970BEF5F1F
:10752E000E2FEDB7FEB7FA93EA930F93EAE0EA93C4
:10753E00E8DD0F91E13209F433C40024021603068C
:10754E0024F4E02FE150E093970B0E94526C0E94BE
:10755E00526C0E94F36DE8EEF8E10E94B96DECEA10
:10756E00FBE00E94E67409F41BC40E94526C0E9458
:10757E00526C0E94F36DEEEEF8E10E94B96DEEEAE8
:10758E00FBE00E94E67409F40BC40E94526C0E9448
:10759E00526C0E94F36DE4EFF8E10E94B96DE9E9D7
:1075AE00FBE0FA93EA93E3E60E94EF7409F4F8C362
:1075BE000E94526C0E94526C0E94F36DEDEFF8E146
:1075CE000E94B96DFADEE13209F4EAC310E013301D
:1075DE0010F00C94A93B0E94526C0E94526C0E94B7
:1075EE00F36DE12F0E944773E3E0F9E10E94B96D5C
:1075FE000E94F4740E941547ADE9BBE00E947471BD
:10760E000E94616DE0E10E94EF7409F4C9C3E9E0E4
:10761E00F0E00E94936C0E941547A0EABBE00E9426
:10762E0074710E94616DE0E10E94EF7409F4B8C3B9
:10763E000E94526C0E94526C0E94F36DE12F0E94C8
:10764E004773EEE0F9E10E94B96D1A93F4DEE13270
:10765E0009F4A6C30E94F4740E94F87451F40E94B7
:10766E002F720E940275E2E00E94067509F498C31B
:10767E0009C00E942F720E940275E0E00E940675FA
:10768E0009F48EC30E94526C0E94526C0E94F36DDC
:10769E00E12F0E944773E0E1F9E10E94B96D0E946B
:1076AE00F4740E941547A9EABBE0EE27A10FBE1F96
:1076BE002C913327EDB7FEB73197FA93EA933F93A8
:1076CE002F93E0E0EA9377DD2F913F91E13209F4B9
:1076DE0067C3A9EABBE00E947471EA0FFB1F208307
:1076EE00123070F50E94526C0E94526C0E94F36D23
:1076FE00E12F0E944773E7E1F9E10E94B96D0E9404
:10770E00F4740E941547A0EBBBE0EE27A10FBE1F3D
:10771E002C913327EDB7FEB73197FA93EA933F9347
:10772E002F93E0E0EA9347DD2F913F91E13209F488
:10773E0037C3A0EBBBE00E947471EA0FFB1F2083DE
:10774E001F5F45CF2DC30E94A37D10E01A930E94A8
:10775E00BD730E940B750E94526C0E9415470E94C9
:10776E002B6E0E940F750E94AC6D0E9405700E94D8
:10777E00066E0E94526C0E94B46D0E9415470E94C4
:10778E0013700E94176EE7E0F0E0FA93EA930E94FE
:10779E00B46D0E941547E091AE0BF091AF0B0E94B5
:1077AE00DD7A0E94176E0E94526C0E94A76D0E9495
:1077BE001547EEE1F9E10E94B96DE091970BEF5F8D
:1077CE00EA930E94E441E7E0F0E0FA93EA930E9424
:1077DE00A76D0E941547C4DD0E94F76DE091990BCD
:1077EE00E03029F0E091990BEA930E94E44100E029
:1077FE000330D8F50E94526CE02FED5FF0E00E944E
:10780E001B6E0E945C72EA930E94E441EBE2EA93E3
:10781E000E94B3460E946372EA930E94E4410E9462
:10782E00F76D0E946A7251F40E9472720E940D6E80
:10783E000E94126E0E941375E3E709C00E947272D5
:10784E000E940D6E0E94BF7B0E94066EE9E4EA93D1
:10785E000E94B3460E94F76D0E947C72EA930E94CA
:10786E00EA410E9417750F5FC3CF0E947A433E2FE5
:10787E003B3211F4103408F001C01F5F3D3211F499
:10788E00113008F401C011503D3439F41A930E949E
:10789E005C1913DE1A930E947C19313209F056CF0F
:1078AE007FC20E94A37D10E00E943C47012F0E94E0
:1078BE00526C0E94526C0E941547E2E2F9E10E945E
:1078CE00B96D31E03C3018F51038F8F40E94526C66
:1078DE000E94ED6C0E941B6E1A930E94B1190E94B9
:1078EE002B6E0E94F76DA091340CE3E00E941B7585
:1078FE00A091350CE7E00E941B75E0912B06EA93F0
:10790E00E8E0EA930E94844113953F5FDBCF0E942B
:10791E00300E0E947A433E2F3D34E9F50E942573C6
:10792E00102F1038C0F51A930E94B1190E94526C94
:10793E000E94526C0E94F36DE6E3F9E10E94B96D6C
:10794E000E942B6E0E940F750E94326E0E94154788
:10795E00E9E3F9E10E94B96DE4E3FCE0FA93EA93FE
:10796E00E3E00E94EF7409F41BC20E94326E0E9483
:10797E00F36DEFE3F9E10E94B96DE5E3FCE0FA93F4
:10798E00EA93E7E00E94EF7409F40AC21A930E9488
:10799E00E5191F5FC6CF313211F0103808F001C063
:1079AE0083CFFEC10E94BD6C0E940B750E94526C6B
:1079BE000E941547E5E4F9E10E94B96D10E015301B
:1079CE00F0F41A930E94F3190E94526C0E94F46E06
:1079DE000E942B6E0E940F75E0912F0C0E94207555
:1079EE00E091320C0E942075E091300C0E942075BF
:1079FE00E091310CEA930E94EA411F5FE0CF0E94B2
:107A0E007A430E2F0D34E9F50E94257310E01530E0
:107A1E00C0F51A930E94F3190E94526C0E94526C88
:107A2E000E94F36DE8E5F9E10E94B96D0E942B6E9C
:107A3E000E940F7530E03430F8F40E94326E0E94CE
:107A4E00F36D0E94ED6C0E94D07AEA55F94F0E94B8
:107A5E00CE7B0E94B96D0E94ED6C0E94D07AEA55E1
:107A6E00F94F0E942475FD013596E4910E94EF7442
:107A7E0009F496C13F5FDFCF1A930E94131A1F5F5E
:107A8E00C6CF8EC10E942E6CE1E0EA930E941A0FBF
:107A9E0000E0083210F00C94103E0E94FC0D0E9483
:107AAE00526C0E94526C0E9415470E94D56C0E9427
:107ABE0027750E94CE7B31960E94B96D0E94F76D9C
:107ACE000E94D56C0E9427753496E491E038A9F493
:107ADE000E941F6E1E2FEDB7FEB7FA93EA931F9307
:107AEE00E0E1EA930EDB1F91E13209F492C0E12F3F
:107AFE00A9E0B0E00E94017C88C0E238A9F40E949F
:107B0E008A701E2FEDB7FEB7FA93EA931F93E0E14A
:107B1E00EA93F7DA1F91E13209F47BC0E12FAAE074
:107B2E00B0E00E94017C71C0E138E1F40E948C74D7
:107B3E001E2FEDB7FEB7FA93EA931F93E3E0EA9395
:107B4E00E0DA1F91E13209F464C00E94FC0D0E943C
:107B5E008C74E11731F0E12FA8E0B0E00E94017CB7
:107B6E00FFCF53C0E03069F40E94D56C0E94277598
:107B7E0032960E94BD6DE1E00E94EF7409F449C097
:107B8E0044C0E13069F40E94D56C0E9427750E94B2
:107B9E002475FD013596E4910E94EF74D1F135C044
:107BAE00E23061F40E94D56C0E94277532960E94D5
:107BBE00BD6DEFE00E94067561F127C0E33071F4F0
:107BCE000E94D56C0E9427750E942475FD01359682
:107BDE00E491EA934FDAE132E1F017C0E430A9F410
:107BEE000E94D56C0E94277532960E94CE7BE09340
:107BFE005A0CF0935B0C0E94DD720E94277535962D
:107C0E00E491EA934EDBE13221F00E9498180F5F67
:107C1E0040CF099119910895E8810E944773ECEDC8
:107C2E00F8E10E94B96D0C9490421A930E9425734C
:107C3E0010E0133010F00C94753E0E94526C0E94AE
:107C4E00526C0E94F36D1A93E7DFECE0F0E00E94B5
:107C5E00936C0E9415471A939FDB0E94F4740E9446
:107C6E00F87451F40E942F720E940275E2E00E9495
:107C7E00067509F4FFC209C00E942F720E94027598
:107C8E00E0E00E94067509F4F5C2123028F50E9454
:107C9E00526C0E94526C0E94F36D1A93BDDFEBE59D
:107CAE00F9E10E94B96DECE0F0E00E94936C0E9445
:107CBE0015470E941775EAE0F0E00E94936C0E944F
:107CCE001547A0EBBBE00E9474710E94616DE3E664
:107CDE000E94EF7409F4CEC21F5FABCFCBC20E94DD
:107CEE00A37D10E01A930E94BD730E940B750E9433
:107CFE00526C0E9415470E942B6E0E940F750E94B7
:107D0E00AC6D21E000E0033080F5E3E0F0E00E948E
:107D1E00046D0E941B6E0A937FDF0E946A7249F403
:107D2E000E9472720E940D6E0E94126E0E94137556
:107D3E0008C00E9472720E940D6E0E94BF7B0E944C
:107D4E00066E0A9329DB2F5F023068F4E7E0F0E05D
:107D5E000E94046D0E941B6E0E9475720E94306E0E
:107D6E000E9417752F5F0F5FCECF0E947A433E2F72
:107D7E003B3211F4103408F001C01F5F3D3211F494
:107D8E00113008F401C011503D3439F41A930E9499
:107D9E005C194BDF1A930E947C19313209F0A2CF85
:107DAE000E94AA7D249608950E9425730E94526C0B
:107DBE000E94526C0E941547E1E6F9E10E94B96DEE
:107DCE00E1E0E0932208E2E2F8E0FA93EA93E5E0DC
:107DDE00EA9397D9089522970E94A17D0E947A4333
:107DEE000E2FE0911B08E03011F00C94A3400132ED
:107DFE00D1F4EAE4F6E0A0913A0CB0913B0CEA170C
:107E0E00FB0761F4E7E0E0931808EAE2EA93EAE69A
:107E1E00F9E10E9485700E942C64A8C0E0E0E09316
:107E2E00C0050E942C750D3331F4E091C005F0E0D1
:107E3E000E94F36C04910D3441F4EAE2EA93EDE60C
:107E4E00F9E10E9485700E942C64063449F4E2E741
:107E5E00F6E0E0933A0CF0933B0CE0E0E093C005C3
:107E6E00003311F00B3229F4E091C005EF5FE0937F
:107E7E00C0050D3229F4E091C005E150E093C00534
:107E8E00013329F491DFED3311F40E94337503337E
:107E9E0021F48ADFED3309F40CD8063329F4E0E03F
:107EAE00E09322080E946037043329F4E0E0E09367
:107EBE0022080E943375A0912408A13010F40C946E
:107ECE003940023301F570DFED33E9F40E9440755D
:107EDE00D1F4E0912208EA930E94AC1B30E03031DD
:107EEE0090F40E94ED6C0E94567059F4E32FE05D01
:107EFE00EA93E0E7F9E10E945B70E0E3EA930E9407
:107F0E004E643F5FECCF053331F5E0E0E09322089D
:107F1E000E94407501F511E01630E8F41A930E94A4
:107F2E00AC1B30E03031A8F40E94ED6C0E9456700C
:107F3E0071F4E32FE05DEA93E0E7F9E1FA93EA9357
:107F4E00E12FE05DEA93E0E3EA930E944E643F5F27
:107F5E00E9CF1F5FE1CF013469F4EAE2EA93E3E788
:107F6E00F9E10E940D74E1E0E09318080E94A87DEB
:107F7E00289608950A3409F4B2DE073311F00C94F2
:107F8E0039400E943C47E0E0EA930E94610EE1E036
:107F9E00E0931C08E0E0F0E0E0931408F09315087D
:107FAE00EFE2F6E00E948570E3E7F0E00E943770A2
:107FBE000E948868EE83FF830E944975E8E2F0E034
:107FCE000E94ED70B9F00E94AF120E948868EE8395
:107FDE00FF83A091190CA03021F00E941C34E030D8
:107FEE0009F408C00E943474E652F84FAEE0A08344
:107FFE000E941F72E5E0F0E00E946F6C40E050E0DE
:10800E000E941422E03868F00E941422EF573E2F8F
:10801E00313010F0313108F004C0E32F0E9441716D
:10802E00AF015A934A930E94E61F4093140850934F
:10803E0015080091DB05E0E0E093DB05013211F05D
:10804E000B3209F401C0B8CF0B3221F4E1E0EA9310
:10805E000E94610E013209F0A3CFE0E0E0931C080C
:10806E00E093DB05A0912408A23011F00C949C4003
:10807E00093309F407DD053409F494DC033611F4F1
:10808E000E94A40D083309F45EDB023409F409DC06
:10809E000334B1F51091390C0E943C4700E0E09199
:1080AE00380CE11711F00C3008F01DC00E94526C14
:1080BE000E94D56C0E941B6E1A930E943A1F1A934F
:1080CE007CD10E94F76DE091290C0E942075E09101
:1080DE002C0C0E9420750E94FD700E94066E0E945C
:1080EE00E3700395DCCF0E94300E0E947A430E2F70
:1080FE00013221F0E091380CE11709F401C0CCCF28
:10810E00043499F40E94407581F4A091D30BA030F1
:10811E0021F4A091D10BA03031F00E9491730E94F6
:10812E00526C0E94A1530E94881DE0911B08E03002
:10813E0011F40E94B90E49C0E130D1F4A09121088A
:10814E00AB3010F4013209F405C00E9445160E94AE
:10815E00300E0DC0E0E0E0931E080E944E750E94A6
:10816E000D74E0E00E945375E2E0E0931B082DC011
:10817E00E23059F5013269F4E0E0E0931B080E9409
:10818E003C47EAE2EA93EDE6F9E10E940D740E94A3
:10819E00B90E0B3211F00D3359F40E944E75FA934D
:1081AE00EA93E1E3EA930E942C64E1E00E945375A6
:1081BE000D3259F40E944E75FA93EA93E2E3EA9374
:1081CE000E942C64E2E00E945375A0911808A3301F
:1081DE0009F404CE0E94A87D0C94E6451A93E3E0C0
:1081EE00E09319080E943C470E94526C0E94526C08
:1081FE000E941547E9E7F9E10E94B96D0E94526CA1
:10820E000E94B46D0E941547E3E1F6E00E9485706E
:10821E00E0E1F0E00E94377010E0E091C90B1E170C
:10822E0000F50E941F6EE117D1F0E12FE05DEA9399
:10823E00E1E8F9E1FA93EA93E0E3EA93E0E00E94E1
:10824E00627049F40E947471ED5EF94FA1E0A08353
:10825E00E12FE05D01C0EEE2EA930E94B3461F5F9C
:10826E00DCCF0E942C75E0E0E093C005E0931B0884
:10827E000E94B90E19910895E881E03021F4E4EFDF
:10828E00F6E00E945875A881A13021F4EEEEF6E0DA
:10829E000E945875A881A23021F4EAEFF6E00E9400
:1082AE005875A881A33021F4E8E0F7E00E945875D4
:1082BE00A881A43021F4EEE0F7E00E94587529C1A0
:1082CE001A930A93E0E0E0937D05E0937E0510E0BB
:1082DE00143190F400E0033068F4A3E01A9FF0012B
:1082EE00EC57FA4FDF01EE27A00FBE1FE0E2EC9332
:1082FE000F5FF1CF1F5FECCFE9C31A9311E0E98155
:10830E00E11780F00E947471E255FF4FE491AA814B
:10831E00EA2319F0E12FE05D01C0E0E2EA931CD5FB
:10832E001F5FEDCF2DC51A9311E0E981E11778F0AB
:10833E000E947471E255FF4FE491AA81EA2311F075
:10834E00E1E301C0E0E3EA9307D51F5FEECF18C566
:10835E002A97A0911B0CA13038F0EA85FB856C851D
:10836E007D850E94137507C00E945D750E94617520
:10837E000E945D75F9D426C12A970E945D750E94F0
:10838E006A750E9473750E945D75EED41BC12A97A3
:10839E000E945D750E9486750E948D75E5D41FC181
:1083AE002A970E945D75EFE9F9E10E9492750E948D
:1083BE0018740E948D75D8D412C12A970E945D75CB
:1083CE00E2EAF9E105C02A970E945D75E6EAF9E155
:1083DE00FA93EA93EE850E94AD6C0E945D75C4D44B
:1083EE002B9608950E94A37D10E0E1E3E0933809F7
:1083FE00E89431F8EA930E94D463EAEAF9E10E9424
:10840E00FD7200E0E09182050E17E0F40E94D56C3B
:10841E00EC57FA4FE081E03258F4E3E2EA930E941F
:10842E0016630E94D56CEC57FA4FE081E05D05C0F3
:10843E000E94D56CEC57FA4FE081EA930E941663C6
:10844E000F5FE0CF0E9497759F010E94B7153A9378
:10845E002A93E8ECF0E0FA93EA930E9494680E2FC8
:10846E00A0E031FCA1E0A03011F4003009F001C011
:10847E00ECCF31FE09C0E0E0E0938205E89431F8DC
:10848E00E1E00E94AA7DEFC41F5F123008F4ADCF69
:10849E00E0E0E09382050E94AA7DE5C4E0918105AB
:1084AE00E03021F4E881EA930E94C15EA09181053B
:1084BE00A13069F4A0E09299A1E0A13021F4A89531
:1084CE000E941F6FF7CFE881EA930E946161A0912D
:1084DE008105A230F1F4E0918205F0E0EC57FA4FFD
:1084EE00A881A083E0918205EF5FE0938205E09181
:1084FE008305EF5FE0938305A03218F4EF5FE093FE
:10850E008305A0918305A83320F06CDFE0E0E093B3
:10851E0083052196089508950E94A8740E94A87458
:10852E0022D0EBE1EA93BADFE9E6EA93B7DFA09156
:10853E008105A13061F4E8ECF0E00E948F6EE091CD
:10854E009A00E069E0939A00E9E1E0939900A09126
:10855E008105A23021F446DFE0E0E0938305E0E000
:10856E00E09381050895EDE0EA9398DFEAE0EA935F
:10857E0095DF08951A9310E0E9811E1728F4EA8119
:10858E00EA938CDF1F5FF8CFFBC3EDE201C0EDE392
:10859E00EA93E8E2EA93EEDFE6DF08952A97A091E8
:1085AE001B0CA13038F00E945D750E946A750E9406
:1085BE00737504C00E945D750E946175FE010E9474
:1085CE0085700FD02E9608952A970E945D750E9491
:1085DE0086750E949B75FE010E94857002D02C96B6
:1085EE0008951A930A9310E0EA81E03011F408E23C
:1085FE0001C00A81AB81BC81EE27A10FBE1FAC91D9
:10860E00A03011F0101708F007C0AB81BC810E949A
:10861E00A0750E94A575EECFEA81E03039F0EA81AF
:10862E001E1720F4E0E20E94A575F9CF27C01A9319
:10863E000A9310E0EA81E03011F408E201C00A81E9
:10864E00E12FAB81BC810E94D974E491E03011F02E
:10865E00101708F009C0E12FAB81BC810E94D974BC
:10866E00E4910E94A575ECCFEA81E03039F0EA8101
:10867E001E1720F4E0E20E94A575F9CF198108813A
:10868E0025960895E091C405A091C305EA17B1F0AF
:10869E000E94AA750E940D6EEC91E093C6050E9491
:1086AE00AA750E948E71E181E093C505A091C40563
:1086BE000E94B075E093C405E1E00895E0E00895EE
:1086CE000E94B575A981A0830E94B5753196A881C7
:1086DE00A083A091C3050E94B075E093C305BFC0EF
:1086EE00E091DB0508951A93E091DB05E03059F433
:1086FE000E94B7150E94257221F4A091DB05A030CF
:10870E0009F001C0F5CF1091DB05E0E0E093DB0549
:10871E000E94257209F011E2E12FD6C30E94A37DBB
:10872E000E9488688F010E94B715EC81FD81E00FD1
:10873E00F11FFF93EF930E948868AF91BF91AE1B1C
:10874E00BF0B9D010024021603061CF40E94257225
:10875E0009F001C0E8CFE0E00E94AA7D26960895B8
:10876E001A93E9810E948972A0E0A0830E94BB75D2
:10877E00108117FF05C0E12F0E94C275A0E0A083F3
:10878E0016FF05C0E12F0E94C975A0E0A0830E94CC
:10879E00BB75A0E0A083E9810E948372A0E0A08354
:1087AE0018815DC00E94A37D30E0EE81ADE0EA9FAE
:1087BE00F001E05FFC4F108116FF17C0E12FEF7341
:1087CE000E2F0E94D07511F03A3008F009C00E94A9
:1087DE00D875DF010E94ED6C0E94DE753F5FF1CF10
:1087EE000E94D8750E94CC74EC9317FF17C0E12F2E
:1087FE00EF730E2F0E94D07511F0343108F009C0BE
:10880E000E94E475DF010E94ED6C0E94DE753F5FF1
:10881E00F1CF0E94E4750E94CC74EC930E94AA7D65
:10882E0042C2E881F9810E94BD6DEA81FB813296D8
:10883E000E94BD6DEC81FD8134960E94BD6DEE816E
:10884E00FF8136960E94BD6DE885F9853896E491D4
:10885E00EA93E985FA8539960E94D26C02D0229667
:10886E000895A0970E94A17DEDA5FEA5A9A9BAA97C
:10887E00EA0FFB1FAF01E5E0F3E0EE83FF8310E0AC
:10888E001431C0F5AE81BF81AC91A03049F1EE81BB
:10889E00FF81A381B481EFA5F8A9EA17FB0701F5C3
:1088AE00EE81FF81A181B281E9A9FAA9AE17BF07B6
:1088BE00BCF0EE81FF81A181B2814A175B0784F083
:1088CE000E94EA75AE0FBF1FE9A9FAA9AE17BF073E
:1088DE003CF00E94EA75AE0FBF1F4A175B070CF4FF
:1088EE0002C01A933DDFEE81FF813D96EE83FF833A
:1088FE001F5FC6CFE5E0F3E0EE83FF8310E0143197
:10890E0010F00C942D45AE81BF81EC91E03011F04A
:10891E000C942645EAA5EC93E9A9FAA9AE81BF818C
:10892E001196ED93FC93EFA5F8A9AE81BF81139636
:10893E00ED93FC93EDA5FEA5AE81BF811596ED934B
:10894E00FC93EBA5AE81BF811796EC93E0910904E1
:10895E00A0910F04EA27AE81BF811896EC93E091A7
:10896E001004AE81BF811996EC93E0911104AE8193
:10897E00BF811A96EC93AE81BF811B960E946E6DDD
:10898E001C96E0E0EC93E887E8A5F9A5309741F056
:10899E000E94F5750E94FA75E4E1EA930E9445691A
:1089AE00EEA1FFA1309751F00E94F575E8A5F9A54B
:1089BE00FA93EA93E4E1EA930E943169E0E0EC8FE6
:1089CE000E94F5750E941C693E2F3B30C8F000E0F6
:1089DE000E94E475E081E03011F0053008F002C02D
:1089EE000F5FF6CF0E94E475E081E03049F40E94FB
:1089FE00E4750E94FF75E058AE81BF811B96EC9323
:108A0E00E0E0EA8B3130C8F000E00E94D875E081DA
:108A1E00E03011F0043108F002C00F5FF6CF0E9473
:108A2E00D875E081E03049F40E94D8750E94FF7538
:108A3E00E05CAE81BF811B96EC93E12F08C0EE8106
:108A4E00FF813D96EE83FF831F5F59CFEFEF0E94AC
:108A5E00A87DE39608951A930A930E940A7630979A
:108A6E00A9F1E0916205E03061F50E940A7604906A
:108A7E0000926205E0916205E03031F4E0E0F0E052
:108A8E000E945875E0E01AC00E940F760E940A7686
:108A9E000E94CE7BF595E7958F01D801E0E0F1E0DD
:108AAE000E94467BE0938700D801E0E0F1E00E944F
:108ABE00787BE09386000E940F76E0E4E0938B00D3
:108ACE0005C0E0916205E150E093620509911991AC
:108ADE0008950E94A37D00E025E033E010E01431FC
:108AEE00B8F5D901EC91E03079F111960E94BF7B77
:108AFE000E94177624F5D90113960E94BF7BAC8194
:108B0E00BD81EA17FB07DCF4F90101801280D9015F
:108B1E0015960E94BF7BE00DF11DAE81BF81AE1791
:108B2E00BF076CF4F90103801480D9011796EC91FC
:108B3E000E942B72AC81BD81AE17BF070CF004C032
:108B4E00E12FEF5F0E2F04C0235F3F4F1F5FC7CF94
:108B5E00003049F0E0916305E01721F0A091630524
:108B6E00A03009F401C022C0A0916405A53079F4AB
:108B7E000A93E1E0EA93A4DD009363050093650593
:108B8E00D901EC91E0936605E3E0E0936105A091D5
:108B9E006405AE3119F4E4E0E0936105A09161053E
:108BAE00A33018F0E5E0E093680507C0E0E0E0933D
:108BBE006405E09361050E941C760E94AA7D2896AA
:108BCE000895E0916305E03091F0A0916405A9321B
:108BDE0020F4EA93E2E0EA9373DDA0916405AD33ED
:108BEE0030F0E0916305EA93E4E0EA9369DDE0E0BA
:108BFE00E0936105E09364050E941C76E0E0E0934B
:108C0E006305E0936705089530D15ADB0895EA8134
:108C1E00E0937F05E881E0938005E0910A04E0612E
:108C2E00E0930A0420C10E94A17DA0917F05A4318A
:108C3E0020F4A0918005A33008F033C0E0917F05A9
:108C4E00F0E0ACE0B0E00E941B7B8F01E09180056C
:108C5E00F0E0A4E1B0E00E941B7B9F010E9422760F
:108C6E00ECE0F0E00E942776F0E00E94CE7A0E94BF
:108C7E00786CEE81E030A9F0E0917F05A3E0EA9FE9
:108C8E00F001EC57FA4FDF01E09180050E94FC6F76
:108C9E004C9155270E9422764A93EFE0EA930E9468
:108CAE00D34D0E94A87D27960895E0910A04E071A5
:108CBE0041F0E2E0EA93B7DFE0910A04EF7EE09341
:108CCE000A0408950E942C76AF3EE0E0BE0744F4FD
:108CDE00A0910203B0910303AF33E1E0BE070CF0A5
:108CEE0039C00E9431760E940E700E94D34DA09121
:108CFE005D05B0915E05549734F4A0915F05B09177
:108D0E00600513970CF012C0E0915D05F0915E05C1
:108D1E00A3E0B0E00E94F37AEC57FA4FA0915F0502
:108D2E00B0916005EA0FFB1FA981A083E0910D04AD
:108D3E00ACE0EA9FF0010E942C760E94D9740E944A
:108D4E003E76E0915D05F0915E053196E0935D050E
:108D5E00F0935E050C94184BE881EA93E0911004B1
:108D6E00EA93B0DF0C94E74A1A9310E00E94437620
:108D7E00E03031F00E944376EA93EEDF1F5FF6CFCC
:108D8E001881239608950E9446760E944B76E03015
:108D9E0021F00832E0E01E070CF007C00E944B766F
:108DAE00EA93DADF0F5F1F4FF0CF198108815BC0A6
:108DBE000E944676F801AB81BC810E94527621F06A
:108DCE00EA810E9457760CF009C0F801AB81BC8194
:108DDE000E945C76C1DF0F5F1F4FECCF19810881B7
:108DEE000EC30E94A37D0E942C760E94617631975D
:108DFE008F010E9466760E9422760E946E7633C0A4
:108E0E000E94A37DAC810E9475760E2F11270E94C1
:108E1E0066760E9422760E946E76F1C2EA81FB810E
:108E2E00E0935D05F0935E05E881F981E0935F05BF
:108E3E00F0936005AA81BB81ECE0F0E00E941B7B01
:108E4E000E943E76A881B981E4E1F0E00E941B7B8E
:108E5E0006C0EA81FB810E943E76E881F981E093AB
:108E6E000203F0930303249608950E947D76143135
:108E7E0020F41A9375DC1F5FFACF0E94526C0E9489
:108E8E00526C0E94736CEFE3F1E00E94786C10E07C
:108E9E00153048F4A5E11A9FF001E051FB4FA0E018
:108EAE00A0831F5FF5CF10E0143148F4ABE01A9F9A
:108EBE00F001EC5EFB4FA0E0A0831F5FF5CFE091C9
:108ECE000A04EF7EE0930A04199108950E947D76BC
:108EDE00143100F5ADE01A9FF001BF01E85FFC4FC1
:108EEE00DF010E94BF7B0F01DF01EB81FC81AE171A
:108EFE00BF075CF0E981FA81E015F10534F0FB0162
:108F0E00E05FFC4FE081E03009F402C01A9328DCE8
:108F1E001F5FDECF0E94526C0E9485760E94736C9A
:108F2E00A985BA850E948A760E94786C67C2A2973C
:108F3E000E94A17DE9A50E9489728F01D8011B961E
:108F4E00EC91E03009F415C2D8011B96EC91E9A31F
:108F5E00E07859F0FE013696FA93EA93EBA10E945F
:108F6E00C275FA93EA930E940669E9A1E07459F07A
:108F7E00FE013696FA93EA93EBA10E94C975FA9315
:108F8E00EA930E940669FE013696FA93EA930E94CE
:108F9E001C69E8A3E0910D04EB8FE0910E04EA8FBB
:108FAE000E94D86ED80111962D913C91D80113963E
:108FBE004D915C91D80115960E94BF7BEEA3FFA345
:108FCE00D8011796EC91F0E0ECA3FDA3D80118960A
:108FDE00EC91EC8FE0910E04A0E10E94326CEAA3BA
:108FEE00FBA30E948F760E94FA750E94FA75ECA17F
:108FFE00EA930E942B4CD8011996EC91EC8FE0303D
:10900E0011F4E8E0EC8F0E948F760E9494765A93CA
:10901E004A930E949B760E949F760E94A6760E949B
:10902E00A9760E948F763A932A930E94A976EEA192
:10903E00FFA10E94B0765A934A930E9494760E94A2
:10904E00A976A8A5A130B1F43A932A93FA013196E4
:10905E000E94A676FA013196FA93EA930E949B76C5
:10906E00F90131960E94B576F9013196FA93EA9399
:10907E000E94A976A8A5A230F1F40E949F7631979E
:10908E000E94A676EAA5FBA5E40FF51F3197FA9389
:10909E00EA930E949B76EEA1FFA1E20FF31F319798
:1090AE000E94B576EAA5FBA5E20FF31F3197FA935E
:1090BE00EA930E94A976E8A5E03011F40C94904949
:1090CE00D8011996EC91EC8FE0910D04ACE00E9462
:1090DE00BA760E94467BED8FA8A1EA1710F40C9485
:1090EE00BF48E1E0E0930E04E03021F0ECA1FDA1D9
:1090FE00B5970CF402C00E94C076AAA1BBA1ECA148
:10910E00FDA1EA1BFB0BDF010E947771EAA3FBA313
:10911E00ABA1AA231AF4E0E0EAA3EBA3A8A10E9454
:10912E007576AEA1BFA1F0E00E94C876EE8FA8A51D
:10913E00A13021F40E94CB760E94CE76A8A5A23053
:10914E0031F40E94CB760E94B0760E94DA76E0E08F
:10915E00E9A30E94E076AE0FBF1FEC91E03039F02C
:10916E000E94E0760E945C760E94E576F2CFD1C036
:10917E00E1E0E0930E04E03031F0ECA1FDA1E73424
:10918E00A0E0FA070CF402C00E94C076E8A1EF8FAF
:10919E00EAA1FBA1EE0FFF1FACA1BDA1AE1BBF0B41
:1091AE00E3E0F0E00E94467BEAA3FBA3ABA1AA2377
:1091BE0022F4E1E0F0E0EAA3FBA3EF8DE150EF8FA4
:1091CE00EF8DF0E0DE011696AE0FBF1FAC91A03210
:1091DE0019F0AF8DA13008F404C0EF8DE150EF8F80
:1091EE00EFCFAF8D0E947576AE2FEEA1FFA1B0E04E
:1091FE00EA17FB0714F3EF8DE03011F4ED8DEF8FCE
:10920E00AF8DECE00E94BA760E94C876EE8FA8A5CC
:10921E00A13021F40E94CB760E94CE76A8A5A23072
:10922E0031F40E94CB760E94B0760E94DA76E0E0AE
:10923E00E9A30E94E0760E94527621F0EF8DA9A15B
:10924E00AE1708F007C00E94E0760E945C760E947E
:10925E00E576EFCFAF8DE8A1EA1BAE2FED8DEA17C5
:10926E0068F0AF8DE8A1EA1BACE0EA9FF001A09197
:10927E000D040E94BA760E94C87601C0E0E0EE8F1F
:10928E00A8A5A130A1F40E94CB76E20FF31F319670
:10929E000E942776AFE00E94326CE40FF51FDF01CB
:1092AE00ECA1FDA10E948E7131960E948B6EA8A535
:1092BE00A23089F40E94CB76E20FF31F0E9427762C
:1092CE00AFE00E94326CE40FF51FDF01ECA1FDA1AF
:1092DE000E940275BEDD0E94E076AE0FBF1FAC91FC
:1092EE00A03219F4E9A1EF5FE9A30E94E0760E9493
:1092FE00527639F0AF8DE9A1EA1BAE2FED8DEA174C
:10930E0008F407C00E94E0760E945C760E94E57623
:10931E00ECCFD8011C96EC91E03029F10E94D86E6A
:10932E000E948F7696DDF801A485A43698F4EFE0BE
:10933E00E0931004F801A485AA3028F0A485AA931E
:10934E000E94E44106C0D8011C96EC91E05DEA93C0
:10935E0003DD09C0ECE0E0931004E2E5EA93FCDCE7
:10936E00EDE4EA93F9DCEB8DE0930D04EA8DE093E6
:10937E000E040E94A87DAA9608951A9310E0E89410
:10938E0027F8143170F40E94B56EE03011F00E948F
:10939E00BC6E1F5FA895E12FE37011F40E94AE150D
:1093AE00F0CFEFE0E09310040E94AE150C94704ED7
:1093BE001A9310E01431F8F40E94C16EB1F0A85F58
:1093CE00BC4F0E94BF7BDF01EB81FC81EA17FB07DC
:1093DE0064F4F001E85FFC4FDF010E94BF7BDF0108
:1093EE00E981FA81AE17BF070CF002C00E94BC6E75
:1093FE001F5FA895DFCFEFE0E0931004188125964C
:10940E0008951A9310E0143190F40E94C16E31F059
:10941E00FD01E15FFC4FE081E17009F406C01A9393
:10942E00E0910A04E170EA9382DD1F5FECCF0C94A9
:10943E00704E2C970E94A17DAD89BE890E947771D6
:10944E000E94ED76EB8BFC8BED89FE890E94F27605
:10945E00EB89FC89E017F107FCF00E9425772E2F8F
:10946E0033270E9449770E9450770E9457770E94B7
:10947E005C770E944977F801A98DBA8D0E94616DC3
:10948E000E945777F8010E946677EA8DEA930E9450
:10949E008E4C0F5F1F4FDCCF48C02C970E94A17DD2
:1094AE00AD89BE89E4E0F0E00E94467B0E94ED7635
:1094BE00EB8BFC8BED89FE89EE0FFF1F0E94F2767F
:1094CE00EB89FC89E017F10784F10E942577AE2F16
:1094DE00ED89FE89B0E0EA0FFB1F9F010E944977DC
:1094EE000E945077E98DFA8DEE0FFF1F0E9466776E
:1094FE000E945C77ED89FE89EE0FFF1FA98DBA8D54
:10950E00AE1BBF0BBA93AA93F801A98DBA8D0E9418
:10951E00616D0E945777F8010E946677EA8DEA9393
:10952E000E948E4C0F5F1F4FCBCF0E94A87D6B9673
:10953E000895EA81F0E0EBBBF5BBF7E1F09365002F
:10954E001F98E6E1E0936500F09365001F9AE881AD
:10955E00F981EBBBF5BB1F98FFE1F0936500EEE1DF
:10956E00E0936500F09365001F9A0C94E34EE2E2DF
:10957E00EBBBE0E0E5BBE7E1E09365001F98E6E1B9
:10958E00E0936500E7E1E093650008951F9A089562
:10959E00A0910403A23021F4E881A8E4B3E10BC04A
:1095AE00A0910403A43021F4E881A8E4B3E103C040
:1095BE00E881A8E2B3E1F0E00E948E710E94CE7BBA
:1095CE0021960895E0910403E23011F4EEE40AC00E
:1095DE00E43039F4E0E2EA93A981BA810E9461761F
:1095EE0004C0E0E2EA93E981FA81FA93EA930E94D9
:1095FE00A04A17C0E0910403E23011F4EFE40AC070
:10960E00E43039F4E1E2EA93A981BA810E946A77E3
:10961E0004C0E1E2EA93E981FA81FA93EA930E94A7
:10962E00A04A22960895E0910403E230B9F4E4E4EE
:10963E00EA930E946F77AE0FBF1FFD01FE2FE0E091
:10964E00AF81B8850E94616D0E94A04AE5E4EA935D
:10965E000E9485760E94A04AE6E453C0E33089F466
:10966E00E7E3EA93FF81E0E00F010E946F77EA0FD4
:10967E00FB1F0E9474770E9485760E94A04AE6E343
:10968E0040C0E43049F5E7E3EA93AF81B8850E9424
:10969E006176DF01EB81FC81AE1BBF0BFD01FE2F5E
:1096AE00E0E00F01AF81B8850E9461760E94747769
:1096BE00AD81BE810E946A77DF01E981FA81AE1B1E
:1096CE00BF0BBA93AA930E94A04AE6E3EA93AD8138
:1096DE00BE810E946A771CC0E0E5EA930E94D474B2
:1096EE000E94A04AE1E5EA930E946F770E94616DA5
:1096FE000E94A04AE2E5EA930E9485760E94A04A63
:10970E00E3E5EA93E981FA81AD81BE81EA0FFB1FA1
:10971E00FA93EA930E94A04A28960895E0910403D2
:10972E00E33029F4E3E0EA93E0E1F1E00BC0E4304A
:10973E0029F4E3E0EA93E0E2F1E004C0E3E0EA9327
:10974E00E0E3F0E1FA93EA930E94A04A0895E091D3
:10975E000403E33029F4E3E0EA93E1E2F1E00BC025
:10976E00E43029F4E3E0EA93E1E1F1E004C0E3E060
:10977E00EA93E8E3F0E1FA93EA930E94A04A08958F
:10978E001A930A93EFE10E947D77EBE10E947D77B9
:10979E00EFE10E947D77E8EFFFEFE0935C0CF09332
:1097AE005D0CE491EF3F39F0E0915C0CF0915D0CB3
:1097BE00049000920403E6ECF3E18F01A091040300
:1097CE00A23019F4E8EAF3E18F01A0910403A4306A
:1097DE0019F4E8E6F3E18F01F801E491ED3F39F475
:1097EE00F80131960E94BD6D0E94A07A19C0EE3F1D
:1097FE0071F4F80131960E94CE7BDF01E0910403F3
:10980E00F0E0EA17FB0711F00D5F1F4F09C0F801DA
:10981E00E491EA93F80131960E94BD6D0E94A04A30
:10982E000D5F1F4FF801E491EF3FB1F60E944B6CB4
:10983E00E1E0E0930E04E0930D04E4E1E093130401
:10984E006DDF0991199108950E948177AE85AA2343
:10985E0062F0AD85BE85A03FE0E0BE0734F4AB8577
:10986E00BC85AF33E1E0BE070CF050C00E94897793
:10987E00AE0FBF1FA03FE0E0BE0734F0AD85BE8542
:10988E000E946176E987FA87EF81F885AB85BC8502
:10989E00AE0FBF1FA034E1E0BE0734F0AB85BC8530
:1098AE000E946A77EF83F8870E94C86D0E94C86D88
:1098BE000E94C86D0E94C86DB6DE0E94C86D0E94DF
:1098CE008E77498554DE0BBB15BB2EE13FE100E0E0
:1098DE0010E0EF81F885E017F10764F050E04517CE
:1098EE0030F020936500309365005F5FF8CF0F5F17
:1098FE001F4FEFCF4BDE0E94526C0E94526C0E94A3
:10990E00736CEFE3F1E0FA93EA938DDEC9C00E9427
:10991E0081770E948977EA17FB0741F0EF81F8857E
:10992E00AB85BC85EA17FB0709F03EC00E9496770F
:10993E001CF00E949D7784F42D853E85ED85FE8575
:10994E00E987FA872D873E872B853C85EB85FC853D
:10995E00EF83F8872B873C870E94C86D0E948E7715
:10996E000E948977EA17FB0749F4F1DEEB85FC8547
:10997E00ED87FE87EF81F885E987FA87F8DD0BBB67
:10998E0015BB2EE13FE10D851E85E985FA85E017B1
:10999E00F1073CF020936500309365000F5F1F4F79
:1099AE00F4CFF4DDBBDE7CC000930B0410930C04EB
:1099BE000E94A4770E94AB77FF93EF930E94AF773C
:1099CE000E94AB77AF91BF91EA17FB0780F10E941F
:1099DE009D77B4F420E030E00E94B277E217F307EF
:1099EE0074F00E94A4770E94B9770E94B2770E9409
:1099FE00BE770E94C77758D02F5F3F4FEDCF16C06E
:109A0E0020E030E00E94AF77E217F3077CF00E946F
:109A1E00A4770E94B9770E94AF770E94BE77F901B2
:109A2E000E94CE7741D02F5F3F4FECCF39C00E94BE
:109A3E009677DCF420E030E00E94D277E217F3074D
:109A4E009CF00E94AF770E94B9770E94D277D00126
:109A5E000E94467BAF010E94C777FA010E94CE7723
:109A6E0023D02F5F3F4FE8CF1BC020E030E00E9495
:109A7E00A477E217F307A4F00E94AF770E94B9779C
:109A8E000E94A477D0010E94467BAF01F9010E948B
:109A9E00CE77FA010E94CE7707D02F5F3F4FE7CFE8
:109AAE000E94A87D2F960895EA81FB81FA93EA938E
:109ABE0089DD0E94D9779EDDE2E2EA93E0910B0404
:109ACE00F0910C04FA93EA930E94A04A249608950A
:109ADE000E94A17D00910D0410E0E0910E041E176E
:109AEE0010F00C94D24DE885F985FA93EA9382DD55
:109AFE002C853D854A855B85022E032A11F40C9434
:109B0E00CA4D37FF36C05A934A935CDDE2E2EBBB97
:109B1E00E0E0E5BBE7E1E09365001F98F6E1F09326
:109B2E006500E0936500EE81EBBBEF81E5BBEFE1F5
:109B3E00FEE1E0936500F0936500E093650001FFA0
:109B4E0004C0F0936500E093650036FF11C0F093FA
:109B5E006500E093650001FF06C0F0936500E09399
:109B6E0065004F5F5F4F220F331F4F5F5F4FEDCF8B
:109B7E001F9A220F331F01FF02C04F5F5F4F4F5FCF
:109B8E005F4F0C94834DE885F9853196E887F98708
:109B9E001F5F0C94744D38C022970E94A17DE885FA
:109BAE00EA930E94CF4AEE83FF83E985A8E1EA9FFC
:109BBE00F001E85DF84F8F0130E0383028F5F801FC
:109BCE00E4915E2F0F5F1F4FF801E4914E2F407FFF
:109BDE000E94DE770E94E377EA87FB87F801E49123
:109BEE004E2F440F440F440F440F0F5F1F4FF801C9
:109BFE00E4915E2F0F5F1F4F0E94DE770E94E37786
:109C0E00EA87FB873F5FD9CF0E94A87D2E960895E5
:109C1E0024970E94A17DEA85EA930E94CF4AEE83A3
:109C2E00FF8300E010E0EB850E945776D4F5EF85B8
:109C3E00F889E887F98720E030E0EC850E94F0771C
:109C4E002CF5E989FA89449155273196E98BFA8BDF
:109C5E005A934A93EA85FB85FA93EA93E989FA893E
:109C6E00FA93EA93EC85FD85FA93EA930E946F4D81
:109C7E00E0910D04EE0FEE0FEE0FA885B9850E9450
:109C8E00D974E887F9872F5F3F4FD7CFE0910E0445
:109C9E00AD85BE850E94D974ED87FE870F5F1F4F7D
:109CAE00C2CF0E94A87D639608951A93EFEF0E948B
:109CBE005272E093390910E00E947471E05CF54F26
:109CCE00E081EF3F31F00E9474710E94F5771F5FC3
:109CDE00F3CF199108951A930A930091CF0BAA818D
:109CEE00A53411F4E0E066C0AA81A23539F4A09142
:109CFE003508A13019F40E94F87709F405C00E94C6
:109D0E00E01CE0E0E0933508AA81AB3411F0A335F6
:109D1E0099F4E02FE470E43011F414E001C013E084
:109D2E00E02FE270E23009F41C5FE02FE170E130C9
:109D3E0009F41F5FE12F3EC0AA81A13511F0A137B2
:109D4E0099F4E02FE470E43011F417E001C016E04E
:109D5E00E02FE270E23009F41C5FE02FE170E13099
:109D6E0009F41F5FE12F26C0AA81A33421F0A1348C
:109D7E0011F0A23441F413E0E02FE170E13009F468
:109D8E001F5FE12F17C0AA81A73741F417E0E02F1C
:109D9E00E170E13009F41F5FE12F0CC0AA81A034FD
:109DAE0041F415E0E02FE170E13009F41F5FE12F7F
:109DBE0001C0EFEF198108812396089524970E9420
:109DCE00A17D2091CF0BA0914009A53411F00C94E8
:109DDE00AF4FE0E0E09335080E944B72E0E0E09375
:109DEE005D0BE091D30BE03089F5E0911008A09166
:109DFE001108EA1739F00E94FE77ED55F84FE08111
:109E0E00E13009F023C0E7E7EA930E9416630E944F
:109E1E00FE77E855F84F0E949371FA93EA930E94E9
:109E2E000478EC55F84FDF010E94FF730E9404780E
:109E3E00E755F84F0E940978E2E0E09335080E945A
:109E4E00FE77ED55F84FA2E0A0832FDFE0913508A5
:109E5E00E03011F00C94AF4F0E94F87711F40C948F
:109E6E00894F0E94D51CE1E0E0933508E22FE8709F
:109E7E00E83081F40E940E78E8EEF3E00E94467B13
:109E8E00DF010E94977D14F4E1E301C0E0E3EA9361
:109E9E000E941663E22FE074E03411F413E001C067
:109EAE0012E0E091240C0E9491741A930E94736345
:109EBE00E22FE470E43049F40E940E78E0E1F7E21C
:109ECE000E94787BAF0114E006C00E940E780E94BB
:109EDE008473AF0113E0E22FE071E03111F44150D1
:109EEE0050405A934A931A930E947363E22FE07282
:109EFE00E03211F414E001C013E0E091270CF09170
:109F0E00280C17C018E0E22FE470E43009F41F5F4C
:109F1E00E22FE870E83009F41F5FE22FE072E032C2
:109F2E0009F41F5FE22FE074E03409F41F5FE0E0F4
:109F3E00F0E0FA93EA931A930E947363E22FE170B2
:109F4E00E13029F4E0915D0BEA930E941663ADDED9
:109F5E00A0914009A73729F4E2E0E0933508E030FC
:109F6E0009F473C00E944B720E9413780E94017311
:109F7E001E2F0E941C73AF01E1E0EA930E94BC62A7
:109F8E000E2FE0911008A0911108EA1739F00E94E7
:109F9E00FE77ED55F84FE081E23009F053C00E9494
:109FAE00FE77EC55F84FDF010E94BF7B4E175F071F
:109FBE0011F00C9425500E94FE77E655F84F008064
:109FCE0011800E941F6E0E94DB71EA17FB0769F178
:109FDE000E94FE77E655F84FDF010E94BF7B0E947C
:109FEE0019780E94FE77E655F84FDF010E94BF7B7D
:109FFE00EC59F44FE0810E9421780E9428780E944B
:10A00E00A26D0E942B78E1EBF9E10E94FD72003007
:10A01E0029F05A934A930E94496302C00E943178F4
:10A02E000E9435780E94EF6309C0003039F00E941B
:10A03E00397820F40E94F4730E94D426E1E1F8E00E
:10A04E000E944078E0E0E0933508A0914009A334E7
:10A05E0021F40E941C34E03009F40BC00E944B72B4
:10A06E000E9413780E9491730E94526C63D30E94D7
:10A07E00881DA0914009A13411F0A23421F40E9450
:10A08E004B720E941378A0914009A03421F40E94D3
:10A09E001C34E03009F420C00E940173E887F98770
:10A0AE00E2E0EA930E94BC621E2F0E9444780E9456
:10A0BE00AE180E9434740E944A78E152F84F108311
:10A0CE000E943474E652F84FA7E0A0830E941F72DC
:10A0DE000E944B720E941378A0914009AB3439F064
:10A0EE00A33529F0A13519F0A13709F076C00E94E9
:10A0FE001C34E03011F40C94EE500E944B720E940E
:10A10E005178E1E4F9E00E941773E22FE270E23039
:10A11E0029F4E4E0EA930E94BC6202C0E1E0F0E0C0
:10A12E00E887F987A0914009A13511F0A13721F4F4
:10A13E000E941C731E2F02C01091E50BE22FE470DB
:10A14E00E43011F4E4E001C0E3E0EA930E94BC6263
:10A15E00AF01A0914009A33511F0A13731F4E88584
:10A16E00F9850E94BA7AE887F9870E94397820F03B
:10A17E00A091D30BA13011F51A935A934A93EB8504
:10A18E00FC85FA93EA930E94A71D0E94AB77EE839B
:10A19E00FF83AE81BF810E94977D84F40E944B7233
:10A1AE00E6E6EA930E941663EE81FF813197EE8315
:10A1BE00FF83AE81BF810E94977D94F31A935A93C9
:10A1CE004A93EB85FC850E94D4726FDD06C00E9417
:10A1DE0091730E94526C0E94A71D0E94A87D2A9620
:10A1EE0008950E945578E89422F80E941374E2E7CD
:10A1FE00EA930E941663E0913B08EA930E9416636D
:10A20E00EFE0EA930E941663A0913808AA3219F47F
:10A21E001A9365D31AC0A0913B080E947471EC5931
:10A22E00F44FE081EA1721F4E0913B08E03349F462
:10A23E000E94F06CAC59B44FE0913B08EC931A932A
:10A24E004ED322FC02C00E94EF63C0C20E9455781A
:10A25E00E0913B08E053AE2F0E947471EB58F44F1F
:10A26E00E081EA1741F51A933AD3A0913608A2304D
:10A27E0019F40E945D7809F402C00E946378A091DF
:10A28E003608A33019F40E945D7809F402C00E94CA
:10A29E006378E0E0E0933608E093600C0E947471FE
:10A2AE00EB58F44FBF01E081EF5FAE2FEAE00E9462
:10A2BE00757BDB01EC938AC2E881E03019F40E94D1
:10A2CE00317806C0E881E8500E9491740E9449637B
:10A2DE00219608950E94A17D25FC28C20E945D78DA
:10A2EE0011F40C94F1520E946678E752F84F9F01D8
:10A2FE00D9011196EC91E43071F50E946C780E94B0
:10A30E006F780E947678F901A681A03021F4A2819F
:10A31E00B381109709F007C0E4EBF9E10E94FD72DA
:10A32E000E94357815C00E9428780E947A780E9483
:10A33E002B78E7EBF9E10E94FD720E947E780E9475
:10A34E008478F901A085B185BA93AA930E944963D6
:10A35E000E948A78EBC1E730C9F40E946C780E94A3
:10A36E006F780E947678EAEBF9E10E94FD720E9406
:10A37E007E780E942B78EDEBF9E10E94FD720E942F
:10A38E007A780E9449630E948A78D0C1E93089F4B4
:10A39E000E946C780E946F780E947678E0ECF9E16A
:10A3AE000E94FD720E9491780E942B780E948A78FA
:10A3BE00BDC1E63029F5EAE2EA930E94D463E3ECEC
:10A3CE00F9E10E94FD72D901EC910E949478E0911E
:10A3DE00CD0B0E949478EBE4EA930E9416630E94E0
:10A3EE007A780E944963E4E5EA930E9416630E941C
:10A3FE007E780E9449630E94EF630E94637896C143
:10A40E00E530C9F40E94E5730E941978D901EC91E8
:10A41E000E9421780E9428780E947A780E942B78D8
:10A42E00E1EBF9E10E94FD720E947E780E94496381
:10A43E000E948A787BC1E83039F50E946C780E94C0
:10A44E006F780E947678E6ECF9E10E94FD72F901D0
:10A45E00A681AA930E94F173309719F00E9405709D
:10A46E0004C0D9011696EC91F0E0FA93EA930E949B
:10A47E0049630E9435780E94EF63D9011196E0E09E
:10A48E00EC930E94637852C1E130C9F5A09119088E
:10A49E00A53029F4E091CD0BE65F1E2F01C011E02F
:10A4AE00E12F0E9498780E9474710E949D780E94FC
:10A4BE00A0780E9428780E947A780E942B78E9EC86
:10A4CE00F9E10E94FD720E947E780E948478D90183
:10A4DE001796EC910E9491740E944963A0911908FD
:10A4EE00A53041F40E94A478A481B581BA93AA93B1
:10A4FE000E94AB630E9497750E94AA7817C1E33041
:10A50E00B1F40E94E573F0960E94B5780E94E5734F
:10A51E000E949D780E94A078ECECF9E10E94FD72F9
:10A52E000E947E780E94B9780E94AA78FFC0EB3014
:10A53E0069F50E94BC780E94BF780E94A078EFEC6B
:10A54E00F9E10E94FD72F901A681AA93B5DE0E947F
:10A55E00A478A781AA93B0DE0E94A478A085B185C5
:10A56E00BA93AA930E9484780E947E780E9484787F
:10A57E00F901A481B581BA93AA930E9484780E94AE
:10A58E0091780E94B9780E94AA78D0C0EC3089F4F4
:10A59E000E94BC780E94BF780E94A078E2EDF9E19B
:10A5AE000E94FD720E9491780E94B9780E94AA784A
:10A5BE00BDC0EE3079F40E94BC780E94BF780E9434
:10A5CE00A078E5EDF9E10E94FD720E9497750E9458
:10A5DE00AA78ACC00E94F87761F0A0913608A0303E
:10A5EE0041F4A091D20BA13021F40E941F6EE130F4
:10A5FE0009F426C0A091850BA03059F0E091870B8D
:10A60E00F091880BFA93EA93E8EEF3E00E949B73C5
:10A61E00B9F4E1E30E94B578E091760BE05D0E941B
:10A62E0021780E941F6EEA930ED1E09336080E94A5
:10A63E009775E0935E0CF0935F0CE0E0E093850B72
:10A64E00A0913608A03059F0E0915E0CF0915F0CAD
:10A65E00FA93EA93E4E6F0E00E949B7309F025C0BA
:10A66E00A0913608A23019F40E945D7809F402C058
:10A67E000E946378A0913608A33019F40E945D7889
:10A68E0009F410C0A091600CA33030F00E946378E2
:10A69E00E0E0E093600C06C00E946678E652F84F48
:10A6AE00A8E0A083E0E0E0933608A091860BA130ED
:10A6BE00E9F5E091390CA091380CEA1791F1EAE234
:10A6CE000E94B578E091740BE05D0E942178E091D4
:10A6DE00390CEA930E943A1F0E942878E091290CC7
:10A6EE000E9491740E942B78E8EDF9E10E94FD72B0
:10A6FE000E94FD70FA93EA930E9484780E947C7403
:10A70E000E94C3780E94EF63E091390CEA930E9495
:10A71E007F1DE091390CEA930E944E1DE093390C97
:10A72E0005C0E0E0E093860B689420F80E94A87DB7
:10A73E00269608951A930A930E941C34E030D9F09D
:10A74E000E943474E752F84F8F01EC81FD81D801DD
:10A75E001296ED93FC93EA81FB81D8011896ED9346
:10A76E00FC93EE81D8011696EC93D8011196E4E095
:10A77E00EC930E941F721981088127960895E0912B
:10A78E00420BEA930E941663E091430BEA930E94F8
:10A79E0016630895F4DF0E94D9770E94C6780E944E
:10A7AE00C6780E942B7899C01A930E9448621E2F79
:10A7BE00103021F0E12FE150E093400BE0DFE0910B
:10A7CE00400BEF5F0E9491740E942B7819910895AF
:10A7DE000E94A37D31E00E94CD7828F00E940B7379
:10A7EE00AC91A43308F02AC030E00E940B73EC91B8
:10A7FE00E270E6951E2F0E940B73EC91E1700E2F06
:10A80E00A0915A0B1A1729F4E1E0EA27E0935A0BAC
:10A81E0031E0A0915B0B0A1729F0E1E0EA27E09303
:10A82E005B0B31E0E0915B0BEE0FE05DA0915A0BFC
:10A83E00EA0FEA930E9416630E940474E32F0E94AB
:10A84E00AA7D249608951A9310E00E94F87711F4C9
:10A85E000C9470540E94D51CECEDF9E10E94FD722F
:10A86E00E091240C0E9491740E942B78EFEDF9E197
:10A87E000E94FD72E091270CF091280C0E94C37883
:10A88E000E940E78A031E7E2BE074CF4E2EEF9E149
:10A89E000E94FD72E091250CF091260C13C0E5EE9E
:10A8AE00F9E10E94FD72E9810E941A700E940E78F1
:10A8BE00EA0FFB1F0E94BB70E091250CF091260C55
:10A8CE00E051F742FA93EA930E9449630E94357869
:10A8DE0011E00E94D178E12F1881229608952497D5
:10A8EE000E94A17D0E94D1780E94F161E13010F4A6
:10A8FE000C944A57E091420BEB3441F4E091430B38
:10A90E00E33219F40E9448621E2FBAC2E435A9F44C
:10A91E00E091430BE33221F40E944862EE83FF8301
:10A92E00E091430BEF3441F40E9448621E2F1A93BC
:10A93E000E94D4740E94AE18A3C2E23411F00C949B
:10A94E00E955E091430BE13251F4AA85AF3F29F46A
:10A95E000E9491730E94526CEDDE0E94881DE09160
:10A96E00430BE134E1F40E9448621E2F113071F462
:10A97E00A0913608A13019F40E94F87709F402C0AC
:10A98E000E94E01CE0E0E093850B09C0E1E0E0935B
:10A99E00850B0E948868E093870BF093880BE091FB
:10A9AE00430BE534A9F4E8EEF9E10E94FD720E9432
:10A9BE00BD1CF3973CF00E9448620E94BB700E943F
:10A9CE00D87801C0E0E3EA930E9416630E943578BE
:10A9DE00E091430BE634D9F40E94E47819F40E9416
:10A9EE004862AF01E885F9850E940A700E2F003487
:10A9FE0020F0A091D30BA13021F40E94F0780E9498
:10AA0E00A71DAA85AF3F19F40E94F07893DEE0915E
:10AA1E00430BE23511F00C94A6550E94E47819F41C
:10AA2E000E944862AF0130E0A091D30BA03021F418
:10AA3E000E941F6EE13009F027C00E942234E030E0
:10AA4E0011F10E94C872EC55F84FA885B985A08304
:10AA5E00B1830E94C872E655F84FDF01EA850E9465
:10AA6E001B720E94C872E855F84F10830E94C8727C
:10AA7E00E755F84F40830E94C872ED55F84FA1E09C
:10AA8E00A0830E94CE7259C00E941C34E23010F492
:10AA9E000C94A4550E9444780E94B41E3E2F3F3F52
:10AAAE0029F00E94D070A417B5070CF412C00E94B2
:10AABE007C74E41BF50B0E94DE700E94A57219F4E3
:10AACE00E0E0E093290C3A930E94411F689420F82D
:10AADE0003C0E0E0E887E9870E943474E752F84F3C
:10AAEE00DF01EA85F0E0EC59F44FE081EC930E942F
:10AAFE0034740E944A78EF51F84FDF01EA850E94C4
:10AB0E001B720E943474E152F84F10830E94347409
:10AB1E00E652F84FA5E0A0830E941F72E885F985E2
:10AB2E00309759F00E944478FA010E94BA7A0E9436
:10AB3E00D4720E94F0780E942F1D689422F8E09142
:10AB4E00430BE335F1F50E944862E887F9870E94CE
:10AB5E006678DF01E652F84FE081E23081F4FD01C4
:10AB6E00EF51F84F008011800E941F6E0E94DB7122
:10AB7E00EA17FB0721F4A0913608A23009F01FC096
:10AB8E000E946678E552F84FDF010E94BF7BDF011D
:10AB9E00E885F985EA17FB0779F40E946678DF01EC
:10ABAE00ED51F84FE081EA93FD01E752F84FE08155
:10ABBE00EA930E94D42603C0E7E0E093240668944B
:10ABCE0022F85EC1E43411F00C945256E091430B1E
:10ABDE00E33559F4EBEEF9E10E94FD720E94E65E58
:10ABEE000E949478E1E0E0933909E091430BE0355F
:10ABFE0011F00C9451560E94F478E03011F40C943C
:10AC0E00515620E00E94F87840F00E940B73AC91F0
:10AC1E00A23219F00E94FC7809F43CC0E22FE03019
:10AC2E0061F40E940B73AC91A33211F421E004C0C5
:10AC3E000E9400790E94C15E2AC0E13051F40E9448
:10AC4E000B73AC91A43211F422E001C020E010E0AD
:10AC5E001EC0E23011F0E330D1F40E9400790E9460
:10AC6E006068EF3F99F0E12FE295E07FEF930E944D
:10AC7E0000790E946068AF91EA0F1E2F2F5F24307B
:10AC8E0021F41A930E94C15E20E001C020E00E94D0
:10AC9E000474B8CFF5C0E33411F00C94BA56E091B9
:10ACAE00430BE534B9F4E8EEF9E10E94FD720E941F
:10ACBE00BD1CF3974CF00E944862E05FF84D0E9475
:10ACCE00BB700E94D87801C0E0E3EA930E9416633D
:10ACDE000E943578E091430BE634A9F441E050E050
:10ACEE000E9448620E2F0E940479E13019F40E94EE
:10ACFE004862AF011A930E94D56CE05FF84D0E9436
:10AD0E00B5760E94A71DE091430BE33591F40E94A6
:10AD1E0008790E940070E83131F4E091890BEA93D2
:10AD2E000E945D1806C0E885EA93EFEFEA930E9451
:10AD3E00D426E091430BE134A9F4EEEEF9E10E9442
:10AD4E00FD720E940879EA930E945C190E941326F4
:10AD5E00E03011F0E1E301C0E0E3EA930E941663F4
:10AD6E000E9435788DC0E63511F00C941F57E09196
:10AD7E00430BE33411F00C941E570E9448621E2FB1
:10AD8E00113010F40C941E57A0911908A13091F5B2
:10AD9E000E940479E03021F0A091A2061A1709F062
:10ADAE0028C011500E944862AF011A930E94A82138
:10ADBE003E2F0E944B730E948E710F010E944B73A7
:10ADCE000E940D6E0E940F790E940479E03071F09E
:10ADDE000E944862AF010E945F730E948E710F0144
:10ADEE000E945F730E940D6E0E940F791A930E944B
:10ADFE0039121DC01630D8F41150A12FEAE00E946E
:10AE0E00257BA3E2EA9FF001E855F94FBF01A12F80
:10AE1E00EAE00E94757BF0E0BB01AAE0B0E00E9480
:10AE2E00F37ADB01AE0FBF1F14960E94257128C066
:10AE3E00E93431F5E091430BE03551F40E9448625C
:10AE4E001E2FE0E0EA931A930E942F19E0932E062C
:10AE5E00E091430BEC34A1F40E940C62E0932806BF
:10AE6E000E940479E03021F00E940C62E0932906E2
:10AE7E000E940479E03021F00E940C62E0932A06D1
:10AE8E000E94AD6131CD0E94A87D2B960895A091B0
:10AE9E00580BA03521F4A091590BA03408F005C031
:10AEAE00E091590BEA930E947C19A091580BA3359F
:10AEBE0021F4A091590BAA3008F005C0E091590B6E
:10AECE00EA930E94A719A091580BAB3421F4A091DC
:10AEDE00590BA03808F005C0E091590BEA930E9477
:10AEEE00E519A091580BA63521F4A091590BA0316C
:10AEFE0008F005C0E091590BEA930E94131AA09135
:10AF0E00580BA43511F40E9498189CD60895E3EAC4
:10AF1E00F6E0FA93EA93E091420BEA93E0E8F0E070
:10AF2E000E94377008950E941779A0E0A083E091E7
:10AF3E00400BE093590BE091420BE093580B0895B0
:10AF4E000E94A17D0E94F161E13010F40C94A15A8F
:10AF5E00E091580BA091420BEA1709F098DFE091AF
:10AF6E00420BE33239F5E091430BEC3431F4CFDF91
:10AF7E00E4E0E09318080E941D79E091430BE4355C
:10AF8E00C1F4C5DFE091630CE03029F0EF77A9E062
:10AF9E00B0E00E94017CE091640CE03029F0EF7784
:10AFAE00AAE0B0E00E94017C0E941D79E7E0E093E8
:10AFBE00180802C0EB34E1F5E091430BE13211F4D5
:10AFCE00A6DF35C0E53211F462DF31C0E33299F409
:10AFDE000E94237921F00E942E790E94B1190E94BD
:10AFEE001779E081EB3429F4E0E0E093340CE09340
:10AFFE00350C99DF1CC0E134D1F40E9448629F01E8
:10B00E002093340C0E94347991F00E9448629F0183
:10B01E00A091340CF901E270F070EA2BE093340C3D
:10B02E000E94347921F00E944862E093350C7FC271
:10B03E00E33581F5E091430BE13211F468DF29C06D
:10B04E00E33299F40E94237921F00E942E790E9416
:10B05E008B190E941779E081E33529F4E091400BBA
:10B06E00EA930E94D01B5FDF14C0EE3491F40E946D
:10B07E00B47410E01A3068F4A3EBBBE0EE27A10F16
:10B08E00BE1F0E947471EC5BF44FE081EC931F5F66
:10B09E00F1CF4DC2E63511F00C949D58E091430B63
:10B0AE00E13211F434DF41C0E33299F40E94237986
:10B0BE0021F00E942E790E94F3190E941779E081E7
:10B0CE00E63529F4E091400BEA930E94261A2BDF15
:10B0DE002CC0E63531F40E9448629F012093300C5B
:10B0EE0024C0E53471F40E9448629F0120932F0C16
:10B0FE000E94347929F00E9448629F012093320CFD
:10B10E0014C0E43591F440E050E00E9448629F0183
:10B11E00022E032A11F042E050E00E94347919F019
:10B12E000E944862AF014093310C01C2E43511F028
:10B13E000C945759E091430BE33231F40E9448626C
:10B14E003197E093400BABC0E03511F00C9456599B
:10B15E0010E00E94F87850F00E940B73AC91AD3362
:10B16E0029F00E94FC7811F01E3008F005C00E94F4
:10B17E0074710E943A79EDCF0E9474710E944379E6
:10B18E00EDE30E94487911F00C945659E4E5E093F2
:10B19E00580B10E00E9499703496E491EF3F11F431
:10B1AE000C9456590E94B8740E9499700E94BD6DFD
:10B1BE000E94F468E03011F00C9454590E9499707A
:10B1CE003496E491E03851F40E944862E058FF4F03
:10B1DE00E093630CE0E8E093640C5FC0E23839F46E
:10B1EE000E944862E058FF4FE093640C56C0E1386D
:10B1FE0039F40E944862A8E0B0E00E94017C4DC084
:10B20E00E03011F0E13051F40E948F70FF93EF9314
:10B21E000E944862AF91BF91EC933FC0E23059F467
:10B22E000E948F70FF93EF930E944862AF91BF917F
:10B23E00ED93FC9332C0E33051F40E948F70FF9374
:10B24E00EF930E942762AF91BF91EC9326C0E4303A
:10B25E0021F50E9499703596E491EA930E94F66268
:10B26E000E948F70E093610CF093620C00E00E94DC
:10B27E0099703596E4910E1780F40E94D56CEC5BB4
:10B28E00F44FE081A091610CB091620CEC93A1E6B9
:10B29E00BCE00E94AF6E0F5FEACF1F5F7BCF47C14E
:10B2AE00E03511F00C949E5AE091430BE33299F481
:10B2BE000E94237921F00E942E790E945C190E942F
:10B2CE001779E081E03529F4E091400BEA930E9472
:10B2DE00E51B29DE2CC1E13211F419DE28C1E1345F
:10B2EE00D1F40E9448621E2F00E00D3098F40E94A7
:10B2FE00DD74EA0FFB1F3396E491E11749F40E94C7
:10B30E00DD740E94E174A0919A0BEA2BE0939A0BE4
:10B31E000F5FEBCF0CC1E63559F5E0E0E093410B42
:10B32E00ADE9BBE00E944D79FF93EF930E94486216
:10B33E00AF91BF91EC93EBE2EA930E94BD61E030D6
:10B34E0059F0A0EABBE00E944D79FF93EF930E9463
:10B35E004862AF91BF91EC930E945079A091410B3E
:10B36E00A33018F40E94347909F401C0D9CFDFC09C
:10B37E00ED34D1F4E0E0E093410BA9EABBE00E948A
:10B38E004D79FF93EF930E944862AF91BF91EC937A
:10B39E000E945079A091410BA33018F40E94347989
:10B3AE0009F401C0EACFC3C0E735D1F4E0E0E09381
:10B3BE00410BA0EBBBE00E944D79FF93EF930E94EF
:10B3CE004862AF91BF91EC930E945079A091410BCE
:10B3DE00A23018F40E94347909F401C0EACFA7C054
:10B3EE00E434C9F5E0E0E093410B0E9448629F010E
:10B3FE00E2E0EA930E94CA61AF01E3E70E94487956
:10B40E0059F40E945679BF01D9010E941672E40FB9
:10B41E00F51FDB01ED93FC93E9E40E94487979F482
:10B42E000E94567920833183AAE9BBE00E944D79B0
:10B43E000F010E945D79EC91E160D001EC930E94C6
:10B44E005079A091410BA33018F40E94347909F47D
:10B45E0001C0CBCF6CC0EE3499F40E94B47410E0EE
:10B46E001A3068F4AAE8BBE0EE27A10FBE1F0E94B7
:10B47E007471EC5BF44FE081EC931F5FF1CF57C01A
:10B48E00E33449F40E94F4780E944862E093950BED
:10B49E00F093960B4CC0E33589F40E9448629F01ED
:10B4AE0000240216030624F42B30E0E03E070CF0D5
:10B4BE0004C0F9013197E093970B39C0E53529F4B3
:10B4CE000E944862E093990B32C0EF3491F40E94CF
:10B4DE0048621E2FECE2EA930E94BD61E12FE295D5
:10B4EE00E07FEF930E944862AF91EA0FE093980BD2
:10B4FE001EC0E035E1F4E0E0E093410BACEABBE0C6
:10B50E000E9463790E948E71FF93EF930E94D66220
:10B51E00AF91BF91ED93FC930E945079A091410B96
:10B52E00A23018F40E94347909F401C0E7CF0E94CA
:10B53E00AD6108CDE0E0E093430A0E94A87D269617
:10B54E0008950E94A37D0E94F161E13010F40C94E5
:10B55E005A5DE091420BE332A9F4E091430BE035E2
:10B56E0019F4E1EFF9E109C0E83419F4E2E1FAE186
:10B57E0004C0E33531F4EDE2FAE1FA93EA930E9466
:10B58E0027638EC2E43511F00C94655BE091430B9A
:10B59E00E43229F4E8E2F0E00E9467798EC0E332EB
:10B5AE0011F402D98AC0E03511F00C94645BE7D82F
:10B5BE00A091400BA83210F00C94645B0E946B7942
:10B5CE000E94BD6D0E942763EDE3EA930E9416630D
:10B5DE000E946B793496E491E03839F40E941F6E24
:10B5EE000E9491740E94496368C0E23839F40E9447
:10B5FE008A700E9491740E9449635FC0E13839F4E9
:10B60E000E948C740E9491740E94496356C0E0306F
:10B61E0011F0E13051F40E946B7932960E94CE7B8C
:10B62E000E9493710E946F7948C0E23059F40E94D3
:10B63E006B7932960E94CE7BDF010E94FF730E94CF
:10B64E0049633BC0E33051F40E946B7932960E94FD
:10B65E00CE7BE081EA930E9457632FC0E43069F5F8
:10B66E000E946B7932960E94CE7BE093610CF09330
:10B67E00620C10E00E946B793596E4911E1790F4DF
:10B68E000E947471EC5BF44F0F01A091610CB091AC
:10B69E00620CEC91D001EC93A1E6BCE00E94AF6E7F
:10B6AE001F5FE8CF0E946B793596E491F0E00E941F
:10B6BE0043790E94B8740E94A063F2C1E33579F514
:10B6CE00E091400BEA930E948B19E091430BE43218
:10B6DE0029F4EAE0F0E00E94677920C0E33211F429
:10B6EE0063D81CC0EE34D1F44AD810E01A3068F496
:10B6FE000E947471EC5BF44F0F01A3EBBBE00E9450
:10B70E00A075D001EC931F5FF1CFE0E0E0934E0BFC
:10B71E000E94B8740E94A0630E943578C1C1E635BC
:10B72E00D9F5E091400BEA930E94F319E091430B97
:10B73E00E43229F4E5E0F0E00E9467792CC0E332B0
:10B74E0011F432D828C0E53451F419D8E0912F0CF9
:10B75E000E9491740E947379E091320C19C0E63503
:10B76E0029F40E94C653E091300C12C0E43599F4CE
:10B77E000E94C653E091310CE03011F0E1E301C0BC
:10B78E00E0E3EA930E9416630E947979E091310C0E
:10B79E00F0E00E94C37884C1E03511F00C94245D72
:10B7AE00E091400BEA930E945C19E091430BE43266
:10B7BE0029F4E0E4F0E00E9467793EC1E33219F427
:10B7CE000E94DB5339C1E13411F00C94305C0E94BD
:10B7DE00C65312E0A0919A0BECEDEA233E2F00E047
:10B7EE000D3078F40E94DD740E94E174E31739F491
:10B7FE000E94DD74EA0FFB1F3396149102C00F5F97
:10B80E00EFCF0E94A26D0E942B78E091980BE03052
:10B81E0089F0E8E4FAE10E94FD720E94816D0E94B7
:10B82E0091740E947379E091980BEF700E9491745D
:10B83E000E942B78E091990BE03051F0EBE4FAE1A5
:10B84E000E94FD72E091990B0E9491740E942B78D8
:10B85E00F3C0E43479F50E947D79A091410BA330B9
:10B86E0040F5E091410BE03011F00E9479790E9491
:10B87E005D79EC91E17061F4A3EABBE00E9463791B
:10B88E000E940D6E0E94FF730E94AB63E3E70BC034
:10B89E00A3EABBE00E9463790E940D6E0E94FF73C3
:10B8AE000E944963E9E4EA930E9416630E9450796C
:10B8BE00D4CFBEC0ED34C9F40E947D79A091410B66
:10B8CE00A33090F4E091410BE03011F00E947979B1
:10B8DE00A9EABBE00E948379EC910E9491740E94C8
:10B8EE0049630E945079EACFA3C0E735C9F40E949C
:10B8FE007D79A091410BA23090F4E091410BE030A4
:10B90E0011F00E947979A0EBBBE00E948379EC9153
:10B91E000E9491740E9449630E945079EACF88C0B8
:10B92E00E63531F50E947D79A091410BA330F8F4F4
:10B93E00E091410BE03011F00E947979ADE9BBE066
:10B94E000E948379EC910E9491740E944963EBE20C
:10B95E00EA930E941663A0EABBE00E948379EC9101
:10B96E000E9491740E9449630E945079DDCF60C09D
:10B97E00EE34D1F40E94C65310E01A3068F40E94DF
:10B98E007471EC5BF44F0F01AAE8BBE00E94A07546
:10B99E00D001EC931F5FF1CFE0E0E0934E0B0E94DD
:10B9AE00B8740E94A06344C0E33499F40E94C65355
:10B9BE000E94B874E3E5FAE1FA93EA930E940570E7
:10B9CE000E9418740E949B750E94B8740E94A06316
:10B9DE002FC0E035A9F40E94C653E091AC0BF09154
:10B9EE00AD0BFA93EA930E94C3630E947979E091BA
:10B9FE00AE0BF091AF0BFA93EA930E94C36318C09B
:10BA0E00E33531F40E94C653E091970BEF5F0DC002
:10BA1E00EF3491F40E94C6530E94816D0E9491747E
:10BA2E000E947379E091980BEF70F0E00E946F79AD
:10BA3E00EBE3EA930E94166333C0EB3489F5E09191
:10BA4E00400BEA930E94B119E091430BE43229F4C2
:10BA5E00E0E8F0E00E94677923C0E33219F40E9417
:10BA6E00DB531EC0E134E1F40E94C653A091340CA6
:10BA7E00E1E0EA230E9491740E947379A091340C44
:10BA8E00E3E0EA230E9491740E947379E091350CF1
:10BA9E000E9491740E944963E6E5FAE10E94FD72EC
:10BAAE000E94AD6150CD0E94D1780E94AA7D24964D
:10BABE0008951A930E944B72E0E4F9E00E94177306
:10BACE000E94D1780E948779E181E43471F40E945A
:10BADE00877902800E941F6EE05DE01529F00E94BA
:10BAEE008779E281EA3209F401C057C00E948C794D
:10BAFE000E948779E1810E9490790E948779E28184
:10BB0E000E9490790E940B731C910E948779339644
:10BB1E000E941773E12FE23131F40E949679E6E02C
:10BB2E00EC930EDA3AC0E13131F40E949679E2E1FB
:10BB3E00EC9307DD32C0EF30A9F40E949679EEE067
:10BB4E00EC930E94EF53E13039F4A0913508A03008
:10BB5E0019F00E94F87709F402C00E94E01C0E94BE
:10BB6E009C791BC0EE30C9F40E949679EFE0EC93FD
:10BB7E000E94EF53E13089F4A0913508A03019F0FE
:10BB8E000E94F87709F402C00E94E01CE0E0E09306
:10BB9E003508EFEFEA930E94765463C21A930E941F
:10BBAE0013740E946770EAE7EA930E9416630E947C
:10BBBE000B7311971C91E12FE23131F4E6E0EA9319
:10BBCE000E941663BDD937C0E13131F4E2E1EA9348
:10BBDE000E941663B6DC2FC0EF3099F40E94A07855
:10BBEE000E94EF53E13039F4A0913508A03019F0DE
:10BBFE000E94F87709F402C00E94E01C0E949C7912
:10BC0E001AC0EE30C1F4EFE0EA930E9416630E9470
:10BC1E00EF53E13081F4A0913508A03019F00E9465
:10BC2E00F87709F402C00E94E01CE0E0E0933508CA
:10BC3E00EA930E947654A0913808AA3211F00E941D
:10BC4E00EF630FC2EFEFE093580BE093590B08959B
:10BC5E00AC81A03310F0AA3308F006C00E94A3797D
:10BC6E00E0530E94AB7999C4AC81A13410F0A73493
:10BC7E0008F006C00E94A379E7530E94AB798DC4E9
:10BC8E00A881B981E0E0EC9388C4AA93EA93FA9371
:10BC9E00EFB7EA931A930A931BB10CB1E0919D0C86
:10BCAE00F0E0E559F34F0083A0919D0CAF5FA09398
:10BCBE009D0CA23319F4E0E0E0939D0C09911991CB
:10BCCE00F3C21A93E0919E0CA0919D0CEA17D1F34A
:10BCDE00F0E0E559F34F1081A0919E0CAF5FA09359
:10BCEE009E0CA23319F4E0E0E0939E0CB9C1A09132
:10BCFE009D0CAE5CE0919E0CAE1BE2E30E94757B48
:10BD0E0008950A921A92FA926A937A938A939A9360
:10BD1E00AA93BA93EA93FA93EFB7EA930E94B07993
:10BD2E0049F0A0913909A03021F00E94700DE13048
:10BD3E0009F401C011C0E091040DF0E0E156F34F9B
:10BD4E00E081ECB9A091040DAF5FA093040DA43671
:10BD5E0019F4E0E0E093040DE991EFBFF991E99158
:10BD6E00B991A9919991899179916991F9901990C7
:10BD7E00099018951A930E94B07959F45D9B09C0E9
:10BD8E00A0913909A13021F40E94700DE03009F024
:10BD9E0013C01091030D0E947471E156F34FA981E7
:10BDAE00A0831F5F143609F410E0E091040DE11733
:10BDBE00E1F31093030D02C0E981ECB9A1C20E9418
:10BDCE00B07921F40E94700DE13009F001C019C361
:10BDDE0050C10E94A37D8BDFE03011F40C94EE5F16
:10BDEE0070DF1E2FA091680CA53618F0E0E0E093EE
:10BDFE003A0930913A09E0913A09E03011F00C9489
:10BE0E00555FA091E40BA13021F0A091E40BA2307C
:10BE1E0031F4E12FEF77E0934009EBE4CEC01A3511
:10BE2E0021F4E1E0E0933A09CAC0123049F4E4E1AA
:10BE3E00E0933A09E0E0E0933B09E0933D09BFC08F
:10BE4E00A091E40BA33069F4173729F01A3310F4DC
:10BE5E00103308F402C0E7E001C0E0E0E0933C09D3
:10BE6E0005C01A930E94724EE0933C09A0913C09C2
:10BE7E00AF3F99F010934009E1E0E0933B09109336
:10BE8E003D09E0913C09E03011F4E5E404C0EAE03C
:10BE9E00E0933A09E0E0E0933F0991C0E13069F4A4
:10BEAE00103039F4E2E0E0933A09E0E0E0933F0924
:10BEBE0003C0E0E0E0933A0982C0E23059F41093F7
:10BECE003C0910933D09E0E0E0933B09E3E0E09389
:10BEDE003A0975C0E330F1F40E94B6790E94BC793C
:10BEEE00EA0F0E94C679A9F4E0913D09E03071F4A1
:10BEFE00E4E0E0933A09E0913B090E94AD6F0E94A5
:10BF0E00CF790E94B679A0E0A08303C0E0E0E09371
:10BF1E003A0955C0E43049F41D3019F4EAE5E093CE
:10BF2E003F09E0E0E0933A094AC0EA3079F40E9412
:10BF3E00B6790E94BC79EA270E94C67931F4E0E016
:10BF4E00E0933A09E5E4E0933F0939C0E431B9F4EE
:10BF5E000E94B6791083E12FA0913D09EA27E09364
:10BF6E003D09E0913B09EF5FE0933B09E0E0E09390
:10BF7E00670C133019F4E5E1E0933A0920C0E5317E
:10BF8E0011F0E63159F41A93E7E6FCE0FA93EA93DE
:10BF9E00EAE3F9E0FA93EA935BDE11C0E73179F454
:10BFAE00E0E0E0933A09173131F4E091670CA0918B
:10BFBE003D09EA1709F003C0E3E4E0933F09A091BD
:10BFCE003A093A1719F0E0E0E093680C04CF0E94AA
:10BFDE00AA7D44C4AA93BA93EA93FA93EFB7EA936D
:10BFEE001A930A9310919B0000919C00E12FEC7123
:10BFFE00A9F4E091CD0DF091CE0DEB5FF24F0083E1
:10C00E00ADECBDE00E94AF6EE83CA0E0FA0731F463
:10C01E00E0E0F0E0E093CD0DF093CE0D0991199193
:10C02E00E991EFBFF991E991B991A99118951A93F8
:10C03E000E94D4790E94D979D9F30E94D479EB5F0A
:10C04E00F24F1081AFECBDE00E94AF6EE83CA0E075
:10C05E00FA0731F4E0E0F0E0E093CF0DF093D00D6D
:10C06E00E12F199108950E94D4790E94D97909F08F
:10C07E00C8C1E0E008950E94A37DF5DFE03021F015
:10C08E00A091660CA03009F0E5C0D1DF1E2FA09163
:10C09E00D90DA53618F0E0E0E093D30D3091D30D15
:10C0AE00E091D30DE03059F4113019F4E4E0E0934F
:10C0BE00D30D1A3519F4EAE0E093D30DC3C0E43082
:10C0CE00C1F4E0E0E093D30D1A3229F00E941F6E06
:10C0DE00E05DE11769F4109338081093D40DE5E094
:10C0EE00E093D30DE0E0E093660CE1E0E093D60D33
:10C0FE00A9C0E530A9F4E0E0E093D30D0E941F6ED5
:10C10E00E05DE11761F00E94E0790E94E979E0912B
:10C11E00D60DEF5FE093D60DE6E0E093D30D92C01F
:10C12E00E63091F4E091D60D0E94E9790E94E07913
:10C13E00EF5FE093D60DE0E0E093D70D133019F4E6
:10C14E00E7E0E093D30D7EC0E73011F0E83059F40C
:10C15E001A93E7EDFDE0FA93EA93E3EDFDE0FA932F
:10C16E00EA9376DD6FC0E93081F4E0E0E093D30D21
:10C17E00173131F4E091D70DA091D40DEA1709F0E3
:10C18E0003C0E4E5E093660C5DC0EA3041F4103084
:10C19E0011F4EBE001C0E0E0E093D30D53C0EB30BF
:10C1AE0071F4E0E0E093D60D1093D50D1093D40DFD
:10C1BE00ECE0E093D30DE0E0E093660C43C0EC308E
:10C1CE00A1F5E091D60DF0E0E05CF64F10830E94F1
:10C1DE00E079EF5FE093D60DE091D50DE150E0935D
:10C1EE00D50DA091D50DA03021F4A091D40DA03085
:10C1FE0009F00EC0EDE0E093D30DE091D60D0E9454
:10C20E00AD6F0E94CF79E091D60DF0E00E94CF790C
:10C21E00A091D50DA03021F4A091D40DA03009F439
:10C22E0003C0E0E0E093D30D0DC0ED3059F4E0E033
:10C23E00E093D30D1D3031F4EAE5E093660CEFEF99
:10C24E00E093650CE091D30DE31719F0E0E0E09375
:10C25E00D90D13CF0E94AA7D01C3AA93EA93FA9334
:10C26E00EFB7EA93E091DB0EA091DA0EEA1791F0A8
:10C27E00E0913708E03019F0E89426F80AC00E94E1
:10C28E00EE79F0E0E030A1E0FA0719F4E0E0E09397
:10C29E00DB0E03C0E89425F826F8E091650CE0303B
:10C2AE0019F0E0E0E093D30DE991EFBFF991E99138
:10C2BE00A99118951A93E091DB0EA091DA0EEA1768
:10C2CE0021F4E0919B00E072C1F4E091DA0EF0E00F
:10C2DE00E652F24FA981A0831091DA0E1F5F0E94E1
:10C2EE00F06CA030E1E0BE0709F410E0E091DB0E47
:10C2FE00E117E1F31093DA0E03C0E981E0939C009D
:10C30E00188122960895E0E0E093DB0EA091DA0EFC
:10C31E00A13020F00E94EE79689426F80895AA9331
:10C32E00BA93EA93EFB7EA93E091650CE03041F4EB
:10C33E00E0E0E093DB0E0E941F6EEF5FE0933708A4
:10C34E00E991EFBFE991B991A99118950E94F878FA
:10C35E0018F00E94FC7809F403C00E940474F6CF12
:10C36E000E94FC7811F40E94047408950E940B73CD
:10C37E00AC91E881EA1729F40E9404743197E1E048
:10C38E005DC1E0E05BC10E94A37D00E010E0EEE243
:10C39E000E944879E9F420E030E0EC810E94F077C9
:10C3AE00BCF4D8010E94C7748F010E94CD7818F09A
:10C3BE000E94FC7908F009C00E940B73EC910E9458
:10C3CE0089730E0F1F1F0E9404742F5F3F4FE5CF1E
:10C3DE00F801E1C00E94F87828F00E948779E18187
:10C3EE00E03208F410C00E940B73EC91E093420B04
:10C3FE000E9404740E940B73EC91E093430B0E9415
:10C40E000474E1E008950C94C2660E9446760E9480
:10C41E0000790E946068EF3F89F0F8010E94CE7AA1
:10C42E00FF93EF930E9400790E946068AF91BF91D5
:10C43E000E94D9748F010E940474E9CFF8011EC0C6
:10C44E001A930A9310E00E940B730C910B3311F0A8
:10C45E00003208F412C0013310F0093308F007C09F
:10C46E00E02F0E948973E255FF4FE4911E2B0E942C
:10C47E0004740E940B730C91E9CFE12F099119916D
:10C48E0008950E94A37D00E010E00E940B73AC9112
:10C49E00AD3221F40E94047431E001C030E00E94FC
:10C4AE00CD7818F00E94FC7908F009C0D8010E94DE
:10C4BE00C7740E94007A8F010E940474F0CF30304E
:10C4CE0021F4F8010E94AA7DC9C1F8010E94BA7A2E
:10C4DE000E94AA7DC3C124971A93E0E0E983EA8300
:10C4EE00EB83EC830E940B73AC91AD3221F40E946E
:10C4FE00047411E001C010E00E94CD7818F00E9483
:10C50E00FC7908F022C0A981BA818B819C81EAE076
:10C51E00F0E060E070E00E94207B7F936F93FF93CA
:10C52E00EF930E940B73EC91E053AF91BF918F91FB
:10C53E009F91FF27662777270E94B07AE983FA83B7
:10C54E006B837C830E940474D7CF103031F4E98161
:10C55E00FA816B817C81188120C0E981FA816B811F
:10C56E007C810E94BE7A188118C00E94A37D20E0B3
:10C57E0030E000E010E0EC810E9457765CF4D901C7
:10C58E000E94C7740E94007A9F010E9404740F5F7C
:10C59E001F4FF1CFF9010E94AA7D259608950E94A2
:10C5AE00A37D6FDF8F0120E030E0EEE20E9448793C
:10C5BE0011F467DF9F01112322F4F9010E94BA7A68
:10C5CE009F01A0911B0CA13030F0D8010E94167271
:10C5DE00E20FF31F8F01F8010E94AA7D3FC11A934B
:10C5EE0010E00E94F478E030A1F00E94F87858F044
:10C5FE000E940B73AC91A23231F00E94FC7819F0BC
:10C60E00E9811E1708F005C00E9474710E943A79E4
:10C61E00ECCF0E9474710E9443790C941E67E881DE
:10C62E000E949079E881A0915C0BEA0FE0935C0B7D
:10C63E00E881A0915D0BEA27E0935D0B21960895AA
:10C64E001A9310E0E12FA981BA810E94D974E49166
:10C65E00E03049F0E12FA981BA810E94D974E491AA
:10C66E000E94067AEFCF0BC01A9310E00E94437619
:10C67E00E03029F00E9443760E94067AF7CF1881A7
:10C68E002396089564970E945D750E940B7AE88D3B
:10C69E00F98D0E9418740E948D75E6DF66960895D6
:10C6AE001A93ECE3EA93BBDF11E0193080F40E9499
:10C6BE007471E255FF4FE491A981EA2319F0E12F3D
:10C6CE00E05D01C0E0E2EA93AADF1F5FEECFEEE38A
:10C6DE00EA93A5DF0C941E6764971A930E94107A52
:10C6EE000E940B7AEA8DFB8D0E9418740E949B7536
:10C6FE000E94107A0E941C691E2FED891E1720F4CD
:10C70E000E9431781F5FF9CF0E94107AADDF188139
:10C71E000EC064970E945D750E940B7AE88DF98DAC
:10C72E006A8D7B8D0E9465740E945D759DDF689693
:10C73E000895E2E2EA9373DF0E94D97795DFE2E291
:10C74E00EA936DDF0C941F67A881B981E4E6F0E0EF
:10C75E000E94467B0E946F79EEE2EA9360DFA88129
:10C76E00B981E4E6F0E00E94787BFA93EA93E2E086
:10C77E00EA93B2DF0C941F67A0911B0CA13020F03E
:10C78E000E94D977E1DF07C00E94D9777BDFE4E60C
:10C79E00FAE10E94FD720C941F6725FE06C0E5E0CB
:10C7AE00F0E00E948F6EA895F8CFEAEDFDE0E093E1
:10C7BE005E0BF0935F0BE1E00E945272E0935C0B14
:10C7CE000E94157A0E941F6E0E9494780C945D69E7
:10C7DE001A930A93E091650CE03011F00C94916875
:10C7EE00E3E0EA931CDFE0915C0BE295EF70EA93D5
:10C7FE000E9477681E2FE0915C0BEF70EA930E9407
:10C80E0077680E2F1A930BDF0A9309DFE7E1EA939D
:10C81E0006DFEAEDFDE0A0915E0BB0915F0B0E948A
:10C82E00E27BEA1BE093DA0E689425F80C9491688B
:10C83E00EE81EA93B2DFEC81FD810E94FD720E94CF
:10C84E00197A67DFC5DF0C948469EB81EA93A5DF63
:10C85E000E946F71F5DE0E94157ABADF2496089554
:10C86E00ED81EA939ADFEB81FC810E94FD72EA81F1
:10C87E00EA93D5DEE981E03011F0EA93D0DEE8816B
:10C88E00E03011F00E94157AA3DF269608950E94DB
:10C89E00A17D10E0E8E6FAE1A885B985EA17FB0765
:10C8AE0019F444E150E002C048EC50E0EA85E09310
:10C8BE003809E89431F8EA93E985FA85FA93EA9310
:10C8CE00EA85EA93EA85EA93E0E0EA93C9DF0E94FB
:10C8DE0088689F010E94B7150E948F760E94946807
:10C8EE000E2F31FC02C0003009F001C0F3CF31FE33
:10C8FE0004C0E89431F8E1E004C01F5F1230B0F2DA
:10C90E00E0E00E94A87D2B9608951A930A93E09179
:10C91E00400AE03011F40C949168E0E0E09339099C
:10C92E00E2E0EA9327DA10E003E00E9474710E94BD
:10C93E00207A61F00E9474710E94F5770E947471E2
:10C94E00E05CF54FE0810E271F5FEFCFE3E0EA9347
:10C95E0011DAE02FE295EF700E94257AE02FEF704A
:10C96E000E94257AE7E1EA9305DA0C9491681A930E
:10C97E000A93E091400AE03011F40C9491680E9401
:10C98E008A70E03021F0E091420AEA3209F405C0E3
:10C99E000E948A70E05DE093420AE0E0E09339097C
:10C9AE00EAE5EA93E7D9E0E0EA93E4D910E00E94E1
:10C9BE0074710E94207A11F01F5FF9CF1F5F012F53
:10C9CE000A93D8D910E00E9474710E94207A61F007
:10C9DE000E9474710E94F5770E947471E05CF54FAD
:10C9EE00E0810E0F1F5FEFCFE02FE195EA93C2D9E2
:10C9FE00EDE0EA93BFD90C9491681A930A93F894D8
:10CA0E00E0E0E0933708E091DB0EE093DA0E7894E5
:10CA1E00E091400AE03011F40C949168EAE5EA9353
:10CA2E0049DCE0E0EA9346DC10E00E9474710E945B
:10CA3E00207A11F01F5FF9CF1F5F012F0A933ADCA6
:10CA4E0010E00E9474710E94207A79F00E94747135
:10CA5E00E05CF54FE081EA932DDC0E947471E05C9E
:10CA6E00F54FE0810E0F1F5FECCFE02FE195EA93BB
:10CA7E0021DCEDE0EA931EDC0C949168E881EA93E8
:10CA8E008CDEEAE5EA93CBDDE0914009EA93C7DD5F
:10CA9E000E940B73EC91E03031F00E940079BFDD03
:10CAAE000E940474F5CF94DE0C945D691A930E9473
:10CABE004B72E0913B08EA93B2DDE4E4EA93AFDD1A
:10CACE00E0913908EA93ABDD14E00E947471E85CE2
:10CADE00F74FE081E43040F00E947471E85CF74F4C
:10CAEE00E0810E94067AF1CFE0E0EA9398DD3FDF25
:10CAFE003DC11A930A936DD9E0913F09E03011F4CC
:10CB0E000C94FD65A0913F09AA3541F4A0913B0913
:10CB1E00A33020F0E0914109E43409F04BC00E94AB
:10CB2E008A70E03021F0E0914209EA32C1F40E94AD
:10CB3E001F6EE05DA0914209EA1721F0E0914209D3
:10CB4E00EA3221F40E94605D12DF08C0E3E4F9E0EE
:10CB5E000E941773E09142090E942B7A2BC00E940B
:10CB6E008A70E05DA0914209EA1721F50E941F6EBE
:10CB7E001E2FE0914309ED3421F4E0914409E33294
:10CB8E0009F007C0E5E4F9E00E9417737ADC1E2F66
:10CB9E00DDDB0E941F6EE11729F0E12FE05D0E94A0
:10CBAE002B7A08C00E941F6EE05DE09342090E943E
:10CBBE00605DDDDEA0913F09A53449F4A091E40B40
:10CBCE00A33019F40E945B2B02C00E94E54EA09187
:10CBDE003F09A33411F40E94132BA0913F09AB34EB
:10CBEE0011F40E940E2BE0E0E0933F09A091E40BBC
:10CBFE00A33011F40E945B2BE0E00C9491683BDAB9
:10CC0E00A091660CA43529F4A0E025FCA1E0A0308B
:10CC1E0009F03AC0E0913A08E03581F4E0913B0822
:10CC2E00EA93E6E0EA930E946743A0913B08A0389E
:10CC3E0020F0E0913B08E093650523C0E03721F436
:10CC4E00E0E0E09365051DC0EA3519F40E94D55D5C
:10CC5E0018C0EA3711F42ADF14C0E23519F40E9425
:10CC6E00F8500FC0E23719F40E942D510AC00E94ED
:10CC7E00DF30E0913908A0913809EA1711F4689471
:10CC8E0031F8E0E0E093660CA091660CAA3531F421
:10CC9E000E94605DB2DEE0E0E093660C6CC0A09195
:10CCAE00690CA13050F0E091690CE150E093690CF1
:10CCBE00E03019F4E1E0E0936A0CA0E025FCA1E07D
:10CCCE00A13049F4A0E026FCA1E0A03021F4A0910F
:10CCDE003708A03009F001C016DBE0913708E030CC
:10CCEE0019F0E150E09337080895E091D90DEF5F08
:10CCFE00E093D90DE091680CEF5FE093680CE09142
:10CD0E00650CE03019F0E150E093650C0895A091A8
:10CD1E00E40BA13021F0A091E40BA23029F4E3E062
:10CD2E00E0939000E8E3E9B90895E0E00E94126C08
:10CD3E00E1B3E360E1BB85E38A95F1F7E1B3EC7F04
:10CD4E00E1BBE4E4E09374000E94296C08951A9309
:10CD5E0014EAE4EA0E94327A41F40E94377A1830DB
:10CD6E0011F0103111F4E0E001C0E2E019910895E4
:10CD7E00E4E9E0937400E0E008951A93E981E1603C
:10CD8E000E943C7A31F40E94377A103411F4E0E0BC
:10CD9E004EC04CC01A93E9810E943C7A31F40E9435
:10CDAE00377A183111F4E0E042C040C01A93E9819D
:10CDBE000E943C7A31F40E94377A183211F4E0E086
:10CDCE0036C034C01A93E981E03011F0E4EC01C0B2
:10CDDE00E4E80E94327A79F40E94377AE091730087
:10CDEE00AA81BB81EC93103511F0183521F4E0E0E7
:10CDFE0018810C94DA6BE1E018810C94DA6B1A93BB
:10CE0E00E981E093740010E0E0917400E07811F491
:10CE1E00163908F005C08BE18A95F1F71F5FF4CF44
:10CE2E00E0917400E07811F0E0E001C0E1E01881DB
:10CE3E00229608950E94A37D3D810C8120E087DF1C
:10CE4E00E03011F5EE810E943A6FF1F43A93AEDFC5
:10CE5E00E030D1F40E94407AB9F479DFE030A1F4E9
:10CE6E00EE810E94206C81F4EDB7FEB7FA93EA933F
:10CE7E001F930E94256C1F91E03031F479DFE12F72
:10CE8E000E94AA7D0C94846950DFD9CF0E94A37DA5
:10CE9E0030E00E811D815BDFE03099F4EF810E945E
:10CEAE003A6F79F40E94407A61F41A937FDFE03092
:10CEBE0041F4EC81EA937ADFE03019F459DFE0E0D7
:10CECE0002C033DFE8CF0E94AA7D289608952297EC
:10CEDE000E94A17D50E02B853A85A89538DFE03081
:10CEEE0011F00C94D067EE850E943A6F11F00C94FD
:10CEFE00D0672A935BDFE03011F00C94D0673A9341
:10CF0E0055DFE03011F00C94D06721DFE03011F0E6
:10CF1E000C94D067EE850E94206CD9F5E0E0EE838C
:10CF2E00EF83EC85FD8531970E94177649F4EDB7B6
:10CF3E00FEB7FA93EA931F930E94256C1F9109C0C6
:10CF4E00EDB7FEB7FA93EA931F93E1E0EA933ADF67
:10CF5E001F910E2FEE81FF81A885B985EA0FFB1F69
:10CF6E001083EE81FF813196EE83FF83003039F41A
:10CF7E00EC85FD85AE81BF81AE17BF0708F001C0FD
:10CF8E00D0CFEC85FD850E94177619F4F1DEE0E036
:10CF9E0002C0CBDEA3CF0E94A87D2F96089568977E
:10CFAE000E94A17D20E0E0E0EC8FED8F31E0A895AE
:10CFBE00E9A1FAA1662777270E94787CEA87FB878A
:10CFCE006C877D87EE8D0E94457AEE83FF8368879E
:10CFDE007987AA85BB858C859D850E944E7DEA8BBF
:10CFEE00FB8B6C8B7D8B0E94D27BFE017296FA932B
:10CFFE00EA930E94DC6BEE8BFF8B688F798F0E9419
:10D00E004B7A0E943F7CAF010E944B7AAE8DBB27BC
:10D01E00882799270E94D97B0E945E7ADE015A9654
:10D02E000E943F7CED93FC930AA119A190DEE030A3
:10D03E00D1F5EDA10E943A6FB1F50E94407A99F5B3
:10D04E001A93B4DEE03079F5303051F14F5F5F4F17
:10D05E00EC8DFD8D3196EC8FFD8FAC8DBD8D1197C6
:10D06E00EBA1FCA1EA17FB0711F430E018C0EC8D20
:10D07E00FD8D3197AF8DB8A10E945C7697DEEE8D57
:10D08E00DA01F0E0EA17FB0751F472DEEA8DFB8D50
:10D09E00A9A1BAA1EA0FFB1FE9A3FAA389CFD4CFA6
:10D0AE0067DEE0E002C041DEC1CF0E94A87DA696F9
:10D0BE000895A881A03310F0AA3308F004C0E881C7
:10D0CE00E0530C945D69A881A13410F0A73408F0E8
:10D0DE0004C0E881E7530C945D69EFEF0C945D6931
:10D0EE00A881AA3020F4E881E05D0C945D69A881E6
:10D0FE00AA3020F0E881E95C0C945D69E8E50C94B7
:10D10E005D691A930A93F8940091620B1091630B68
:10D11E007894F8010991199108951A930A93F1DF01
:10D12E008F01EA81FB81AC81BD81EA0FFB1FE01B01
:10D13E00F10BDF010E94977D2CF4E0E0198108814C
:10D14E000C94086CE1E0198108810C94086CECE9F0
:10D15E00F4E1FA93EA93E8E2F0E0FA93EA930E949C
:10D16E00A76DE4E1EA93EBE1EA93EFE0EA930E9424
:10D17E000F4EE8EBF6E1FA93EA93E0E7F0E0FA936C
:10D18E00EA93EDE1F0E0FA93EA93E9E0EA93E2E163
:10D19E00EA93EFE0EA930E940F4E08950895998165
:10D1AE008881009641F0BD81AC81FB81EA810590BA
:10D1BE000D920197E1F7FD81EC810C94086CB98119
:10D1CE00A881109631F0FC81EB816A8161931197F1
:10D1DE00E9F7EB81FC8125960895E991F991A991E2
:10D1EE00B9911D900590011421F40020D1F7EE277E
:10D1FE0008951018E1F3E1E008F4E2500895E99182
:10D20E00F991A991B991CD0161916D936623E1F7E1
:10D21E00FC010895E991F991A991B991CD0105907B
:10D22E000D920020E1F7FC010895A991B991EE2726
:10D23E00FF276D91662311F03196FBCF0895AA2733
:10D24E00BB27E991F9910590002011F01196FBCFC3
:10D25E00FD0108957991E991F991A991B991CD01C5
:10D26E00772351F07A9561916D936623C9F77723F1
:10D27E0019F07A956D93FBCFFC0108956991E991B0
:10D28E00F991A991B991CD01662351F06A95059056
:10D29E000D920020C9F7662319F06A950D92FBCF07
:10D2AE00FC0108955D9BFECFE881ECB921960895AF
:10D2BE001A930A93AC81BD810E94BF7B3097C1F057
:10D2CE00AA81BB810E94BF7B8F01309749F002304B
:10D2DE00E0E01E0760F0F80131978F01ED93FC93AB
:10D2EE00AC81BD810E94AF6E3197AE81A08303C029
:10D2FE00EE81EA93D7DF19810881279608952C973E
:10D30E000E94A17D10E0E88DF98D3196E88FF98F9E
:10D31E003197E4912E2FE03011F40C94446BE12FF1
:10D32E00E03039F4253211F411E002C00E94637A24
:10D33E00A3C1E130C1F4253219F40E94637A9BC176
:10D34E0012E0E0E0E98B00E02D3211F401E094C12F
:10D35E002B3219F4EBE2E98B8FC1203219F4E0E2A3
:10D36E00E98B8AC102C0E23039F450E013E0203379
:10D37E0011F4006881C102C0E330A1F4203310F033
:10D38E002A3308F009C0A52FEAE0EA9FF0015E2FCC
:10D39E00E22FE0535E0F70C140E02E3211F414E024
:10D3AE006BC110C0E430A1F4203310F02A3308F022
:10D3BE0009C0A42FEAE0EA9FF0014E2FE22FE053BE
:10D3CE004E0F5AC12C3619F4026015E055C104C037
:10D3DE00E53011F00C94436BE22FE33649F40E94D2
:10D3EE006E7AEE89FF89A481AA930E94747A43C152
:10D3FE00E33741F40E946E7A0E947E7A0E941C6985
:10D40E001E2F0AC0E037A1F40E946E7A0E947E7A27
:10D41E000E9426691E2F08600F77403011F04117C9
:10D42E0008F001C0142F40E0E0E0E88B30E076C059
:10D43E00E43611F0E93611F4046002C0E537A1F4C8
:10D44E00EAE0E88B01FF08C0E0E0FAEC6AE97BE372
:10D45E000E946E6E1AE023C0E0E1F7E260E070E039
:10D46E000E946E6E15E01BC0E83511F4086004C012
:10D47E00E83711F00C94426BE0E1E88B01FF08C035
:10D48E00E0E0F0E060E070E10E946E6E18E007C030
:10D49E00E0E0F0E160E070E00E946E6E14E040307B
:10D4AE0011F00F7701C041E001FF08C00E946E7AB3
:10D4BE00AE89BF8914960E94C37B13C002FF08C0B9
:10D4CE000E946E7AAE89BF8914960E94126E09C0B0
:10D4DE000E946E7AAE89BF8914960E94BF7B662722
:10D4EE007727EC87FD876E877F8702FF16C0AF8593
:10D4FE00AA2362F4EC85FD856E857F850E94BE7A37
:10D50E00EC87FD876E877F87EDE2E98BE989E03056
:10D51E0019F01F5F4F5F01C00B7F342F00FD14C049
:10D52E00151710F4351708F00FC007FF08C002FFDB
:10D53E0004C00B7F2989115001C020E301C020E2F5
:10D54E000E94637A5150ECCF1417B0F4006102FFC1
:10D55E000AC00B7FE989EA930E94747A503009F071
:10D56E00515011504150E0E3EA930E94747A5030CA
:10D57E0009F051504150E8CF312FE889E030D1F415
:10D58E003030B9F003FF08C0EE81FF813196EE8393
:10D59E00FF833197E49105C0AE81BF81ED91AE83DB
:10D5AE00BF83EA930E94747A503009F05150315083
:10D5BE00E7CF57C00E94867A0E944B7B2E2F2A30CF
:10D5CE0030F003FF02C0295C01C0295A01C0205D62
:10D5DE0004FD25C0213360F4A885B9858A859B8515
:10D5EE00A130E0E0BE07E0E08E07E0E09E0709F420
:10D5FE000BC0431740F4531710F000FF01C014C0C6
:10D60E0020E207FF0CC020E3006102FF08C00B7F81
:10D61E00E989EA930E94747A503009F051500E94C1
:10D62E00637A503009F0515031500E94867A0E9430
:10D63E00867BEC87FD876E877F87E889A885B9850D
:10D64E008A859B85FF27662777270E944B7B0E9442
:10D65E006E6EE885F9856A857B850E94937D09F05B
:10D66E00A9CF00FF08C0503031F05150E0E2EA93EC
:10D67E000E94747AF8CF10E046CE0E94A87D6A967A
:10D68E000895FF92F82E22971A930A93DE010E94B4
:10D69E00AC7A8D01DE0116960E94AC7A0E94BF7B99
:10D6AE00EA83FB83DE0114960E94AC7A0E94FF731C
:10D6BE001A930A93FE0136960E94936C20DEAA817D
:10D6CE00BB81E0E0EC93198108812496FF900895C8
:10D6DE00A991B991EE27002460E8E894162E1694CD
:10D6EE0007941E2A1EF0A015B10518F0A019B10955
:10D6FE00E62BB7FBAA0FBB1F669580F708957B81BB
:10D70E006A81F981E88177FB770F67FD7160972F4A
:10D71E009E5781F078F0983190F4AA27BB2788277E
:10D72E0008948795B795A7959A95D1F7EA23FB2389
:10D73E00682305C0E8947727EE27FF2766276F77C3
:10D74E00769508F4606877F9A991B99189919991C4
:10D75E00EA17FB076807790797FB08950E94197A65
:10D76E000E948F7A19F40E94967A1DC0E6F7A8815E
:10D77E00B9818A819B81E0E0F0E060E87FE30E945E
:10D78E005E7A11C00E94197A0E948F7A19F40E9453
:10D79E00967A09C0E6F30E94967AA0E0B0E080E89F
:10D7AE009FE30E94B27C249608950E949B7A0E9469
:10D7BE00937D39F4A881B9810E943B700E94C97B88
:10D7CE0020C0AA81BB818C819D810E949B7D34F4F7
:10D7DE000E949B7A0E94D27BC1DF05C00E949B7A79
:10D7EE000E94D27BCFDFA881B9810E94C97BA8811C
:10D7FE00B9810E94C37BAA81BB818C819D810E94CD
:10D80E005E7A26960895E991F99130971AF4E0958B
:10D81E00F09531960895E0937100E0E0E093740086
:10D82E00E2B3E360E2BB089588EC90E00197F1F774
:10D83E000895EA930E94C466E0300895E0E0EA930A
:10D84E000C94E96680E991E00197F1F708951A9337
:10D85E000A930C943C47EA9FF001F0E00895FA9386
:10D86E00EA93A02FB0E00895ECE3F0E00E941B7B5A
:10D87E000895ECE3F0E0FA93EA930895EAE3F3E017
:10D88E00FA93EA930C941844E0E0E0930F04EFE06F
:10D89E00E09310040895E0E0F0E0FA93EA9308951F
:10D8AE00FA93EA93E8E2F0E0FA93EA93E0E0EA937F
:10D8BE000C942B4CE0915905F0915A05FA93EA938A
:10D8CE000895E0915B05F0915C05FA93EA93089553
:10D8DE00FA93EA930C949543EFEEF0E0FA93EA9301
:10D8EE000895FA93EA93E0E0EA930C942B4CFA93A2
:10D8FE00EA930C941844E12FA0E4B2E0F0E00E9409
:10D90E00D27AEA0FFB1F0895A12FB0E0ADCFFA93A4
:10D91E00EA93E2E3F0E00895FA93EA93BCCFE09144
:10D92E001004E0930F0408950E94070E0C94C4494E
:10D93E00E32FF0E0E05BFD4FE4910895EA930E943F
:10D94E001D0EFE013696FA93EA930895FF27662779
:10D95E0077270E94D27B84E00E94486B2896089518
:10D96E00FE017196FA93EA930C9438440E94A37DBB
:10D97E000C943C47E8E0F0E0FA93EA930895E4E073
:10D98E00F0E0FA93EA930895FA93EA93E8E3F0E06D
:10D99E00FA93EA9308950E94CE7BBECFE02FF0E07B
:10D9AE000895A0913A0CB0913B0CBD01A3E0B0E0FC
:10D9BE000E94F37AE60FF71FE491E0300895E091AC
:10D9CE00C005EE0FEE0FEF5F3E2F0895E32FF0E050
:10D9DE000895A12FB0E00895A0913A0CB0913B0CA0
:10D9EE00BD01A3E0B0E00E94F37AE60FF71F0895A1
:10D9FE000E94D07AE05AFD4F0895FA93EA93E22FEF
:10DA0E00F0E008950E94A17DA09119080895E0917B
:10DA1E00C20BF0E00895AFE3B1E00E94467B08959B
:10DA2E0030911E08E1E0E0930D04E2E0E0930E0475
:10DA3E003A930E945C19E091980BE295EF70E09397
:10DA4E000F04E091980BEF70E09310040895FA9391
:10DA5E00EA93E52FF0E0FA93EA930895E7E3F0E016
:10DA6E00FA93EA930895E22FE450F0E0FA93EA93E2
:10DA7E000895FA93EA93F7CFE32FE058EA930BCF8A
:10DA8E00EAE8FBE0FA93EA930C9438443A930E9446
:10DA9E005C19A0918A0BAD320895E091980BE29536
:10DAAE00EF70E0930F04E091980BEF700895E52F5F
:10DABE00F0E00895EA0FFB1FFA93EA930895EF5EE4
:10DACE00FC4FBF01E081E058DB01EC930895E0E0EC
:10DADE00EC93AE81BF810895E3E0F0E0FA93EA9310
:10DAEE000895E52FE450F0E0FA93EA930895E55097
:10DAFE00F0E00895E091980BE295EF700895EA1B1F
:10DB0E00A2E5B7E0F0E00E94D27A0895F0E0EE0FC1
:10DB1E00FF1FEA5CFD4F0895A4E3B2E0F0E0EE0FC4
:10DB2E00FF1FEA0FFB1F0895FA93EA93E12FF0E02F
:10DB3E00FA93EA930895E12FF0E0FA93EA930895A9
:10DB4E00E2E0F0E0FA93EA930895EAE8FBE0FA9354
:10DB5E00EA93EAE0EA930C94DF46E1E0F0E0FA9310
:10DB6E00EA930895FA93EA930C94CA460E94CE7BE8
:10DB7E00FA93EA930895ABE0EA9FF001E252FA4F6E
:10DB8E000895ED85FE85FA93EA9308951A930A9304
:10DB9E003ECF1A930A93E0E0EA930E942B4CDDCF1E
:10DBAE00E1E0E0933C0C0E948868E0933D0CF0931A
:10DBBE003E0C0895BD01AAE0B0E00E94F37AE60F94
:10DBCE00F71F0895FA93EA93EAE0EA930C94DF467E
:10DBDE00E1E0E0930E045FCE0E9415470C94F846E8
:10DBEE00E0E2EA930C94B346A3E2B7E0E881F0E0FA
:10DBFE00EE0FFF1FAE0FBF1F0E94BF7B0895FA935B
:10DC0E00EA930C94CE41E881F0E00895EE0FFF1FE9
:10DC1E00AE0FBF1F08950E94BF7B0E94DD7A08954C
:10DC2E000E94D27B0C94AF41FA93EA930C94154761
:10DC3E00A9E0B0E00E94ED7B0895A7E11A9FF001E4
:10DC4E00EF5CF94FE0810895E12FEF5FEA930C94BA
:10DC5E00E441F0E0D4CFE8E0F0E05ECEEA93E6E017
:10DC6E00EA930E949A4186CEE0916D05F0916E0581
:10DC7E000895E0916905F0916A050895AE0FBF1FF2
:10DC8E00E3E0F0E00E94467B0895FA93EA931A933C
:10DC9E000A930C944013FA93EA933A932A930C94B2
:10DCAE004013A0917105B09172050895A09173056E
:10DCBE00B09174050895A0E0B0E00E94E97B08954C
:10DCCE000E94E27BEA1BFB0B0E94DD7A0895E88737
:10DCDE00F9876A877B870895A885B9858A859B858C
:10DCEE00EFEEF0E060E070E008950E94DD7A0E94B1
:10DCFE00707B0895A4E0B0E00E94E97B0895EC8368
:10DD0E00FD836E837F830895FA93EA930C943047D4
:10DD1E00FA93EA930C94A07AA9E01A9FF001E058C6
:10DD2E00FC4F089537960E94CE7BDF010E94BF7B89
:10DD3E0008950A921A92FA926A937A938A939A9310
:10DD4E00AA93BA93EA93FA93EFB7EA931A930895C4
:10DD5E00ED91FD913196FE93EE930895ADE01A9FED
:10DD6E00F001EB5FFC4FE08108951A93E1E0EA9336
:10DD7E000C949E47ADE01A9FF001DF01EB5FFC4F64
:10DD8E00E081E0300895E2E0EA930C949E47FA9326
:10DD9E00EA93E4E6F0E0FA93EA930E949468E030A6
:10DDAE000895E1E0E0930D04E0930E040895E091F0
:10DDBE002908F0912A0860912B0870912C0808957B
:10DDCE00E0912108E150A3EAB6E0F0E00E94D27A99
:10DDDE00AE0FBF1F0E94C37B0895E12FEF5FF0E0EF
:10DDEE0023CFE0912208EA93E0911E08EA930E9465
:10DDFE00721BA0911E0CB0911F0C10970895A0914C
:10DE0E00200CB091210C8091220C9091230C0E9439
:10DE1E009B7D0895E0911E0CF0911F0C0895E091EA
:10DE2E00200CF091210C6091220C7091230C08951E
:10DE3E00E2E3F0E06DCF1A93E0EAEA93EA81F0E0D4
:10DE4E00E054F14FFA93EA930E9421671E2F089532
:10DE5E00E0EAEA93EA81F0E0E054F14FFA93EA93B4
:10DE6E001A930C944D67EA930E94D166E0300895A0
:10DE7E00E0EAEA93EEE5F0E0FA93EA93E0E0FFE001
:10DE8E00FA93EA93EEEBFBE00895FA93EA93E0E25D
:10DE9E00EA930C94D667E0EAEA93E981FA81E050BE
:10DEAE00FE4EFA93EA930895EA81F0E0A8E2B0E01C
:10DEBE000E941B7B0895E0EAEA9342CEFA93EA931E
:10DECE000C946E67FA93EA930C942167E0EAEA9356
:10DEDE00E8E2F0E0FA93EA931A930A93EAE8FBE099
:10DEEE000895EAE8FBE0FA93EA930895EDE2EA93E7
:10DEFE00EAE0F0E0FA93EA930E94E668E0E0089523
:10DF0E00EA81F0E0ABE0B0E00E941B7BE050F24F04
:10DF1E008F01AA81AA300895E0EAEA93EBE0F0E0DF
:10DF2E00FA93EA931A930A93E2EBFBE00895E3EB7C
:10DF3E00FBE0FA93EA930895EA81F0E0EE0FFF1FFB
:10DF4E00E050F04F8F01AA81A0380895E150F0E023
:10DF5E000895EA81F0E00E94D27AE058F14F8F01E5
:10DF6E00AA81A5300895EFE2FCE0FA93EA93E0E08F
:10DF7E00EA9305CDECE1FCE0FA93EA93E0E0EA9354
:10DF8E00F9CC0E94D27A0E94CE7ADF01EA85F0E0C7
:10DF9E00AE0FBF1FE8E0F0E00E941B7BE050FA4E90
:10DFAE008F01E0EAEA93E6CC1A930A93ECE1FCE0E7
:10DFBE0085CFAE81BF81888599850E94B07AEE8328
:10DFCE00FF8368877987089540931E0C50931F0C2A
:10DFDE00EE81FF8168857985E093200CF093210C0A
:10DFEE006093220C7093230C0895F0E0AE0FBF1FC8
:10DFFE000895EA930E945C190C942C20E091950BE5
:10E00E00F091960B0895FA93EA930C94FB18ED8118
:10E01E00EA93ED81EA930895E091AC0BF091AD0B8C
:10E02E000E94DD7A0895F0E0A4E6B0E00E941B7B2A
:10E03E000895EC81F0E0EA0FFB1F0895E0912708A8
:10E04E00F09128080895E093270CF093280C0C9477
:10E05E00C31CE3EAF6E0FA93EA93E0E0EA9308954C
:10E06E00FA93EA930C94E668E0E0F0E060E070E08A
:10E07E000895E0932908F0932A0860932B08709373
:10E08E002C080895E091970BA3EAB6E0F0E00E9409
:10E09E00D27A0895AE0FBF1F0E94C37B0895ED5E26
:10E0AE00F94FE081E1300895FA93EA93E091220866
:10E0BE00E05DEA930895EA930E944E64E13008957C
:10E0CE00ECE3F8E0E093600BF093610B0895E12F21
:10E0DE00A3EAB6E0F0E00E94D27A08950E94D668D4
:10E0EE00A881AF5FEAE00E94257BE05D0895A881DC
:10E0FE00AF5FEAE00E94757BE05D0895FA93EA93C4
:10E10E00E0E0EA930895AAE0B0E00E94ED7B089566
:10E11E00E12FF0E00E94D07AE854FF4F32960E9431
:10E12E00CE7B0895E12FF0E00E94D07AE854FF4FA5
:10E13E0008953696E491D901EC930895E0EAEA93B6
:10E14E00E5E0F0E0FA93EA930895EA930E94B41C96
:10E15E00FA93EA93E4E2FCE00895FA93EA93EFEF80
:10E16E00EA93E5E0F0E07CCFE093250CF093260CEB
:10E17E0008950E94E27BEA1BFB0B0895A0912A0CE6
:10E18E00B0912B0C0895E0E0E093380CE093390C3D
:10E19E000895A0912C0CB0912D0C0895E0912C0CAB
:10E1AE00F0912D0CAC81BD81EA0FFB1F0895E09319
:10E1BE002C0CF0932D0C08951A930E944E1D1E2FB9
:10E1CE000895E0932A0CF0932B0C0895FA93EA939A
:10E1DE000E949468E0300895ABE01A9FF001E4527B
:10E1EE00FA4F08951A930E943A1FD3CFE0912A0C4A
:10E1FE00F0912B0C0895EA930E943A1F0E94D71EAD
:10E20E00E0300895EB81EA930E94751DFA93EA932C
:10E21E00E9E2FCE00895E0E0E0934D0CE0934C0C55
:10E22E0008951A930A93E0911208ABE0EA9FF00169
:10E23E00E752F84F8F01D80111960895E0E0F0E013
:10E24E00ED93FC930895EA81D801EC93E2E1F8E0B6
:10E25E00FA93EA930E941034198108810895E12FF0
:10E26E00ACE8B0E0F0E0EE0FFF1FEA0FFB1F0E94DC
:10E27E00CE7B0895ACE8B0E0F0E0EE0FFF1FEA0FA2
:10E28E00FB1F0E94CE7B0895A0911608B09117082F
:10E29E00EA2BFB2BE0931608F09317080895E15034
:10E2AE00A7E1EA9FF0010895A7E10A9FF001E15D61
:10E2BE00F94FAF010895A3E21A9FF001ED55F94F02
:10E2CE000895EC93EC81E150ADE0EA9FF0010895E2
:10E2DE00E981FA81FA93EA930895E12FF0E0089527
:10E2EE00E2E0F0E00E94467B0895AAE9BBE0E091EF
:10E2FE001A080895ADE9BBE0E0911A0876CEA0EABF
:10E30E00BBE0E0911A0871CEA3E2B7E0D0CBEE0FDE
:10E31E00FF1FEA0FFB1F0895E081F0E00895A7E1CB
:10E32E001A9FF001E15DF94FEE83FF83AE81BF814D
:10E33E000895EE81FF81A481AA930C9473200D9011
:10E34E001C90AE81BF811296EC91F0E0E00DF11DB4
:10E35E00DB01ED93FC930895ED91FD913197FE93C2
:10E36E00EE9308950E9409220E2EAA85BB85EC918C
:10E37E00E0150895A3E20A9FF001E855F94F0895BC
:10E38E00E0911208ABE0EA9FF001E752F84FEC87FC
:10E39E00FD87AC85BD85119608951296EC91AC85DE
:10E3AE00BD851696EC930895D001F0E00895A885EA
:10E3BE00B98518960E94BF7B0895AC85BD85EC93F8
:10E3CE00E2E1F8E0FA93EA930C941034E885F985CB
:10E3DE00A281AA9308950A930E946320E0300895C3
:10E3EE00AA85BB85EC91EA93E3E0EA930C9467432C
:10E3FE00AA85BB85E0E0EC93E2E0E0932406089565
:10E40E00BF0100801180AE81BF811296EC910895FC
:10E41E00DB01ED93FC93AE81BF81129658CBE4E6FF
:10E42E00F0E00E941B7B0895F0E0ED93FC930895BD
:10E43E00E2E1F8E0FA93EA930C941034E0911908B3
:10E44E00A0911808EA170895F0E0E00DF11D089567
:10E45E00A3EABBE042CFADE9BBE0EE27A10FBE1FA2
:10E46E00EC910895A0EABBE0EE27A10FBE1FEC9140
:10E47E000895BD01AAE0B0E00E94F37ADB01089591
:10E48E00E081EA930C94C15EE0E4FAE0E0935E0B67
:10E49E00F0935F0B0895EA930E941663E0E00895EF
:10E4AE00EA930E9416630C948C64ADE9BBE0EE27F0
:10E4BE00A00FBE1FEC910895A0EABBE0EE27A00FBF
:10E4CE00BE1FEC910895AAE9BBE0EE27A00FBE1F78
:10E4DE00EC91E1700895A3EABBE060CAA0EBBBE04B
:10E4EE00EE27A00FBE1FEC910895A9EABBE0EE2720
:10E4FE00A00FBE1FEC910895ADE0EA9FF001E15F21
:10E50E00FC4F0895ADE0EA9FF001EB5FFC4F0895DC
:10E51E00ABE00A9FF001E452FA4F0895ABE00A9F78
:10E52E00F001EE51FA4F0895FA93EA930C949B354D
:10E53E00FA93EA930E94D9433A9325CCE0912C0C9E
:10E54E00F0912D0C30970895AFEFBFEFA083B183FC
:10E55E0008950E948868E093520CF093530C08952E
:10E56E00FA93EA93E0E0F0E80895E0911208ABE048
:10E57E00EA9FF001E752F84FFA93EA930E946F294F
:10E58E0057CFE0911008ABE0EA9FF0010895E0E16B
:10E59E00F8E0FA93EA930C941034FA93EA930C94FD
:10E5AE00A153E88DABE0EA9FF0010895FA93EA9348
:10E5BE00F5C9E0E1EA93E0912506EA930E942F194E
:10E5CE001E2F08953BDDFA93EA930895FA93EA938A
:10E5DE000C94051FE0932506E0E0E0934F0CE1E379
:10E5EE00E093500C0E94AE2A0C948C26FA93EA9378
:10E5FE000C942763E1E4F9E0E093600BF093610B78
:10E60E00E3E0EA930C94BC62A091600BB091610BB5
:10E61E0008950E948868E093470CF093480C089583
:10E62E00E093600BF093610B0895E3E0EA930C9492
:10E63E00BC62E0932708F093280808950E943C4797
:10E64E00E0E0EA930C941A0FE0E0F0E0E093250886
:10E65E00F0932608E2E0E0930E040895E09113048F
:10E66E0046CAE0912508F0912608C9CAE0915D05D9
:10E67E00F0915E0531970895FA93EA930C940E4645
:10E68E00EF5CEA930C94B346A3EEB6E09FC9A3EAFF
:10E69E00BBE0E0911A08F0E03ACE0E94BF7BD001B9
:10E6AE00ED93FC9322CEF0E0EA0FFB1F0F011DCE7F
:10E6BE00A3E2B7E08BC9E7E0E0931808EA93E0E045
:10E6CE00EA93E9C8EA930E9443410E947A431E2FBF
:10E6DE000895EAE2EA93E7E7F8E110CD0E945A2C9A
:10E6EE00E1E0EA930C94422C1F771A930C945C1978
:10E6FE00A0912508B09126080895E8EEF3E00E9457
:10E70E00787B0895E053F0E00895A0E024FCA1E0AA
:10E71E00A0300895E0E0EA93BEC8E0913308F0918E
:10E72E003408FA93EA930895FA93EA930E94946850
:10E73E00E13008950E948868E0933308F09334081E
:10E74E000895E0E0E0934C0C0895D2DFEA17FB0742
:10E75E000895E0931808E0E0E093300808950E94D1
:10E76E002C640E94C32DE093240808950E945C1926
:10E77E000C943C47E0911908EA93E0E0EA930E947A
:10E78E006D2D0C9421290E947A431E2F1A930E94FC
:10E79E00F32D103808951A93E091C605EA93089563
:10E7AE00E091890BEA930E946718E03008950E9469
:10E7BE008868E093540CF093550C0895D90118967F
:10E7CE000E94BF7B0895E4E6F0E060E070E00E94F6
:10E7DE00707B08950E945C1911CC0A93E091C605D6
:10E7EE00EA930895E0912F08EA930A930C94911AF4
:10E7FE000E94BF7BFA93EA930895A0E6BBE0A8CAF5
:10E80E00E0913C08E053E09322080895FA93EA93CE
:10E81E00E0E3EA930C942C64E0913908EA930C94AB
:10E82E00D4630E94DD7A0E94D27B08950E94906389
:10E83E00EBE3EA930C941663E89423F8E0E0F0E03F
:10E84E00F8DE0A93E1E0EA930C946D2D0A93E1E071
:10E85E00EA930E946D2DE1E00895E0911208ABE07D
:10E86E00EA9FF0010895A881B981EC91EF5FEC93D6
:10E87E000895ABE00A9FF001E352FA4F0895A0838A
:10E88E00ABE00A9FF0010895ABE00A9FF001E15260
:10E89E00FA4F0895E7EAF8E1FA93EA93EA85ABE0D6
:10E8AE00EA9FF0010895AC81BD81EE27A00FBE1F37
:10E8BE000895E02FAC81BD81F0E008950E94D27BD7
:10E8CE0084E00E94486B28960895EE27A30FBE1F82
:10E8DE00EC91D001EC930895A2E5B7E077C80E94C1
:10E8EE00D27AEA0FFB1FAF010895E0912C0CF09144
:10E8FE002D0C0895E32FA0911E08EA0F0895ADE0A8
:10E90E002A9FF001E35FFC4F0895A8E0B0E00E945B
:10E91E00ED7B0895F0E0FA93EA9308950E94EB429E
:10E92E000C94BA42F0E00E94D27A08950E94D27BF3
:10E93E000E94D5420C94BA420E94EB42EBECF8E1F5
:10E94E00DDCB0E94BA420C94BA4220E030E0E12FB7
:10E95E00E05DEA93EEECF8E1A7CBEAE0EA930C94E3
:10E96E00F662E4E4FBE0FA93EA93089510915D05F4
:10E97E0000915F0508950E947A433E2F0C945C46E9
:10E98E00EAE0F0E00E941B7B0895DF01EE27A30F63
:10E99E00BE1F0895FA93EA931FC9EF81F885FA9383
:10E9AE00EA930895F0E0EA0FFB1F0895E02FA0E030
:10E9BE00B2E0B8CFEA0FFB1F3296E4910895FA93B6
:10E9CE00EA93E0911B0CEA930E94E238E13208953B
:10E9DE00EA930E948838E1320895E6E0F0E00C9464
:10E9EE00936C0E941547AAE9BBE0EE27A10FBE1F4C
:10E9FE00EC91E1700895EE0FFF1F0C94616DEA9398
:10EA0E000E94E238E13208950E94300E0C94526C4E
:10EA1E00EAE3EA930C94B3460E94D27B0C94C34172
:10EA2E00E3E7EA930C94B346EA23EA930E94EA41A1
:10EA3E00D7C8EA930E94EA41D3C8DF01329696C83E
:10EA4E000E94D07AE854FF4F0895EAE4F6E0E0938E
:10EA5E003A0CF0933B0C08950E94F61AE0E0E09316
:10EA6E0021080E9445160E94300EE1E0E0931B083B
:10EA7E0008950E943C470E94CC100E947A430E2FAC
:10EA8E000D330895EE81FF81FA93EA930895EAE239
:10EA9E00EA93E6E7F9E10895EA930E9495160C943D
:10EAAE00300EE093C105F093C2050895FE01FA936E
:10EABE00EA930895EEE8F9E1FA93EA93EE85FF857D
:10EACE0068897989FBCEE2E9F9E1FA93EA93AE859A
:10EADE00BF858889998977CE0E94D27BAA89BB8906
:10EAEE008C899D89E4E6F0E060E070E00E948A7B0C
:10EAFE000E94D27B88E00E94486B2C960895EBE929
:10EB0E00F9E1FA93EA93EE85FF858BCE84E00E94BD
:10EB1E00486B2896CBCFFA93EA93EE85FF8508953E
:10EB2E000E94EF630C94886884E00E94486B2896DC
:10EB3E000895EE27A10FBE1FEC910895EA930E944F
:10EB4E0055421F5F0895E091C405A7ECB5E0F0E0D3
:10EB5E000895AF5FEAE00E94757B0895E091C305CA
:10EB6E00A7ECB5E0F0E0D3CBE981ADE0EA9FF00190
:10EB7E00E05FFC4F0895EF73A5E1EA9FF001E051CD
:10EB8E00FB4F0895EF73ABE0EA9FF001EC5EFB4F95
:10EB9E000895AC81BD81EE27A30FBE1FAC91A030AE
:10EBAE000895ABE00A9FF001EC5EFB4F0895EA0F6B
:10EBBE00FB1F0F01AC81BD8188CEA5E10A9FF0013C
:10EBCE00E051FB4F0895EE81FF8101801280AE81EE
:10EBDE00BF8115960E94BF7BD0010895FE01389625
:10EBEE00FA93EA930895EAA5FBA5FA93EA9308959A
:10EBFE00FA93EA93FE013A96FA93EA930E94066913
:10EC0E0030E0E02F0895E091C105F091C20508951E
:10EC1E00A1ECB5E0ED91FD913296FE93EE93089541
:10EC2E00AE81BF81EA17FB070895E0E0E09365052A
:10EC3E00E093660508951A930A933A932A930895DA
:10EC4E00FA93EA93E0910E040895A0910003B09117
:10EC5E0001030895E0910003F0910103FA93EA9302
:10EC6E00E0910203F0910303FA93EA930895E0937F
:10EC7E000003F09301030895A981BA815ACF1A9324
:10EC8E000A9300E010E00895F801AA81BB81EA0F13
:10EC9E00FB1FE4910895AE0FBF1FAC91A0300895F5
:10ECAE00D801F0E0AE17BF070895AE0FBF1FEC916D
:10ECBE00EA930895EFEEF0E0EA1BFB0B0895A091A6
:10ECCE000E04E4E1EA9FF0012E2F3327C3CFE0E0DC
:10ECDE00EA930E942B4C0E94AA7D0895ECE0EA9FD5
:10ECEE00F001A0910D04EA9FF00108951A93E1E05E
:10ECFE00E0930E04E0930D0410E00895ED81FE8183
:10ED0E00FA93EA930895EF81F885EA1BFB0B0895B9
:10ED1E003A932A935A934A930895EAA5FBA5E20FD4
:10ED2E00F31FFA93EA930895ECA1EA930C948E4C98
:10ED3E003A932A93EEA1FFA1E40FF51F0895FA93DB
:10ED4E00EA93EBCFEAA5FBA5E40FF51FFA93EA933E
:10ED5E00EBCFE20FF31FFA93EA930895FA93EA9337
:10ED6E005A934A930895EA9FF001AEA1BFA1F0E035
:10ED7E000895E2E0E0930E04E0E2F0E0EAA3FBA3E4
:10ED8E000895AE1BBF0BACCAEE8DF0E00895E20FF6
:10ED9E00F31F3196FA93EA93ECA1FDA1E40FF51F50
:10EDAE0031960C948B6EECA1FDA1E40FF51F0C9423
:10EDBE008B6EE9A1F0E0DE0116960895ED8DEA93D3
:10EDCE000E946946E9A1EF5FE9A30895ED8BFE8BE2
:10EDDE00AB89BC8985CAA98DBA8DEA0FFB1FE98F55
:10EDEE00FA8FEB89FC89AF89B88DEA0FFB1FEF8B89
:10EDFE00F88FED89FE89AD89BE890E941B7B0E942A
:10EE0E00DD7A0E94787CEE87FF87688B798BEB89A1
:10EE1E00FC89AB89BC890E941B7B0E94DD7A0E9413
:10EE2E00787CAE85BF85888999890E944E7DEA8758
:10EE3E00FB876C877D8700E010E00895F8010E9443
:10EE4E00DD7A0E94787CEE83FF8368877987AE81B6
:10EE5E00BF81888599850E94007DAA85BB858C859A
:10EE6E009D850E94007DAE85BF85888999890E9407
:10EE7E00DC7B0E94AB7C0E94417CAF015A934A938B
:10EE8E000C946F6BE98DFA8DE21BF30BFA93EA93F8
:10EE9E000895E98DFA8DE01BF10BFA93EA9308952C
:10EEAE00F901AD8DBE8D0C94616DED8DFE8DE01B67
:10EEBE00F10BFA93EA93EA8DEA930C948E4CAD8D96
:10EECE00BE8D0C94616DEFE3F1E0EA1BFB0B089530
:10EEDE00EB81FC81AF81B8850895E00DF11DFA93A9
:10EEEE00EA930E94A04AE5E3EA930895E093650051
:10EEFE000C941F6F0E94A17DEE81EA930E94CF4A6F
:10EF0E008F010895E985FA85AD85BE8508950E9425
:10EF1E00E94AEB85FC85FA93EA930C94014BED8557
:10EF2E00FE85A985BA85AE17BF070895EB85FC85CA
:10EF3E00AF81B885AE17BF070895AD85BE85E9854B
:10EF4E00FA85EA1BFB0B0895FA93EA930C940A6C6C
:10EF5E00AB85BC85D8CEAF81B885EB85FC85EA1B29
:10EF6E00FB0B0895D9010E941B7B0F010895D00160
:10EF7E000E94467BAF01FA01AD85BE850C94616D92
:10EF8E00ED85FE85E21BF30BFA93EA930895AD85AA
:10EF9E00BE850C94616DA985BA85ED85FE85EA1B4B
:10EFAE00FB0B0895E881F981FA93EA9308955A9339
:10EFBE004A93EE85FF85AFCDFA93EA93EC85FD85F6
:10EFCE00FA93EA930E946F4DE0910E04AA85BB85D9
:10EFDE00E9CCD901F0E0AE17BF070895E05CF54F1C
:10EFEE004FCAE091370CA091360CEA170895E091C4
:10EFFE001108ABE0EA9FF0010895E3E0EA930E9466
:10F00E007363F5CFE081E05DEA930C941663A091F3
:10F01E00250CB091260C0895E2E5EA930E94166342
:10F02E000C945C4EF096EA930E94D463E2E7EA9366
:10F03E000C941663EA930E941663EEE0EA930C9426
:10F04E001663EEEAF9E1D2CA0E944963EBE3EA9352
:10F05E000C941663E0E3EA930C941663EBE3EA93E5
:10F06E000C9416635A934A930E94FB180E2F003489
:10F07E000895FA93EA930C9410341A93E985FA855D
:10F08E00FA93EA930895E552F84FA885B985A083BF
:10F09E00B183E3CBE2E5EA930C9416631A93E09105
:10F0AE003908E0531E2FEDE3F8E0BACAE0911208DA
:10F0BE00A0911308EA170895E3E1F8E0DACFE091A2
:10F0CE001308ABE0EA9FF0010895A091740B41CDB7
:10F0DE00E093740BEAE2EA930E94D463DBCFE091F3
:10F0EE00740BE05AA7CFD9011696EC9113CCF90107
:10F0FE00A281B381BA93AA9308950E944963EAE369
:10F10E00EA930C941663D9011196E0E0EC930E94F9
:10F11E00EF63D2CFD901EC91FDCBE05DEA930C9475
:10F12E001663E05DEA930E94D463B4CFEB58F44FBC
:10F13E0069CFEEE0EA930C941663EAE3EA930E9439
:10F14E001663F9010895E0935E0CF0935F0CE2E014
:10F15E00E0933608D9011196EC930895EA930E9434
:10F16E00D46398CF0E944963DBCCE091190CD9CFC0
:10F17E00E091190CF0E0DACFFA93EA9365CF0E9492
:10F18E004963ECE2EA930E9416630CCF3DDAAC9130
:10F19E00A0330895A0915E0BB0915F0BE0E0EC936D
:10F1AE000895EE81FF81E093270CF093280C1093C5
:10F1BE00240C0E94C31CE1E3089541E050E00E943C
:10F1CE004862E887F987EAE3EA930E94BD61E1307D
:10F1DE0008951A93E985FA85C1CDE2E2EA930C947B
:10F1EE00BD6112DAAC91A03208950EDAAC91AB3358
:10F1FE0008950ADAEC91EA930895EAE3EA930C94FF
:10F20E00BD610E9448623197E887F987E8850895C5
:10F21E000E94BF7BE40FF51FD001ED93FC93089580
:10F22E00E091400BF0E0ED55F94F0895E0E0E093EA
:10F23E00630CE093640C08950E9448623197E0934A
:10F24E00400BE091590BA091400BEA1708950E94D4
:10F25E004E57E091400BEA930895ECE2EA930E9438
:10F26E00BD61E0300895EC5BF44F0F01CDD9EC9108
:10F27E00D001EC931F5FC1CAEC5BF44FA0E0A083FA
:10F28E000895EA930E94BD61E1300895E091410B2B
:10F29E0089CBE091410BEF5FE093410B0895A3EA18
:10F2AE00BBE0E091410BF0E00C948E71AAE9BBE05B
:10F2BE00E091410B0C94FC6FE091410BF0E008954E
:10F2CE00FA93EA930C94D153E091400BF0E0B8CB53
:10F2DE00FA93EA930C9449630E944963ECE2EA9331
:10F2EE000C941663ECE2EA930C9416630E94C653D8
:10F2FE00E0E0E093410B0895E091410B0C94FC6F1C
:10F30E00E091600BF091610B0895AEE5BBE00C94BB
:10F31E00AF6EA0915E0BB0915F0BEC93F6CFA09108
:10F32E005E0BB0915F0B13970895E0E0EA930E9495
:10F33E002A54E09335080895AA81BB81EC91E29599
:10F34E00E07FAE2FEC810895EA0FAA81BB81EC938A
:10F35E008ACAE091040DA091030DEA170895E09179
:10F36E003B09F0E0E05CF64F08951083E0913B0915
:10F37E00EF5FE0933B09E12FA0913D090895E093E3
:10F38E003D09E0913C09E150E0933C09E0300895DD
:10F39E00E05CF64FA0E0A0830895E091CF0DF091D0
:10F3AE00D00D0895A091CD0DB091CE0DEA17FB07AB
:10F3BE000895E12FA091D40DEA0FE093D40DE091C2
:10F3CE00D60D0895F0E0E85CF74F10830895E091B4
:10F3DE00DB0EF0E0E652F24FE081E0939C00E0910C
:10F3EE00DB0EEF5FE093DB0E08950ED9AC91AA33DE
:10F3FE0008950F0109D9EC91E0530C942B72EA9306
:10F40E000E9416631F5F0895ECE5FAE1FA93EA9302
:10F41E000895FE013196FA93EA930895E881EA93EE
:10F42E000C941663E881F9816A817B810E94D27BFC
:10F43E000895E05CF54FE081E0300895EA930E9474
:10F44E007768EA930C94C15EEA930E944565EAE5FB
:10F45E00E0933E090895EA930E940667E03008950E
:10F46E00E0917100E87F1E2F0895E0937300E4E8A9
:10F47E00F2CF0A930E94DD66E0300895FF276627DB
:10F48E0077270E94787C0895EE8DAE85BF8588899A
:10F49E009989F4DF0E94007DA9A1BAA18827992736
:10F4AE000E94D97B0E94DC7B0E94AB7C08950E9457
:10F4BE00DC7B0E94AB7C08952A93ED89FE89FA933A
:10F4CE00EA93FE017596FA93EA930C945F69EE89BE
:10F4DE00FF893497EE8BFF8B0895ED89FE89FA93A1
:10F4EE00EA93FE017596FA93EA930C945F69AE89DE
:10F4FE00BF8914960E94BF7BEE83FF83C3CAE88543
:10F50E00F9856A857B85AC85BD858E859F85089539
:10F51E000E94866BE883F9836A837B830895E88172
:10F52E00F9816A817B810895EA81FB816C817D81FD
:10F53E000895E991F991309639F080EA9FE00197AC
:10F54E00F1F7A8953197C9F708950024AF0DB01DB6
:10F55E000895EA0FFB1F681F791F0895EA1BFB0B26
:10F56E00680B790B0895F195E195F0400895F095AB
:10F57E0060957095E195FF4F6F4F7F4F0895EE2385
:10F58E000E2EEA2F19F0EE0F0A94E9F70895EE0FFA
:10F59E00FF1FEE0FFF1FEE0FFF1FEE0FFF1F089551
:10F5AE00FE2FFF0FFF0B6F2F7F2F08956F2F660F0C
:10F5BE00660B762F0895BA2FBB0FBB0B8B2F9B2F8D
:10F5CE0008958B2F880F880B982F0895EA17FB0745
:10F5DE00E1E00CF0EE270895FA9FF02DEB9FF00D71
:10F5EE00EA9FE02DF10D08957A9F702D6B9F700D9F
:10F5FE00F89F700DE99F700D6A9F602D710DFB9F36
:10F60E00600D711DE89F600D711D8827FA9FF02D0A
:10F61E00610D781FEB9FF00D611D781FEA9FE02DA5
:10F62E00F10D681F781F089582D0D6DF0EF49BDF90
:10F63E0008958BD0D9DF0EF49ADF0895002498E058
:10F64E00AA0F001C0E1A10F40E0E01C0A1609A959E
:10F65E00B9F7EA2FA02D08950024112490E1AA0FE6
:10F66E00BB1F001C111C0E1A1F0A18F40E0E1F1EB3
:10F67E0001C0A1609A9599F7FD01D001089557D068
:10F68E00EBDF0EF470DF08953F934F935F930024EA
:10F69E0011244427552730E2AA0FBB1F881F991F3C
:10F6AE00001C111C441F551F0E1A1F0A460B570B28
:10F6BE0028F40E0E1F1E461F571F01C0A1603A955B
:10F6CE0059F7FD01BC01D001CA015F914F913F91E5
:10F6DE0008953BD0D9DF0EF44ADF0895AFDFEA2F4D
:10F6EE000895E894B7FF04C0A095B095119668945C
:10F6FE00F7FD39DFB1DFFD010EF435DF0895C4DF0C
:10F70E00FD01BC010895E89497FF09C0A095B0953E
:10F71E0080959095AF5FBF4F8F4F9F4F689477FD49
:10F72E0026DFB2DFFD01BC010EF421DF0895E8945F
:10F73E00F7FF02C018DF6894B7FF06C0A095B0951A
:10F74E00119600F8039400FA0895E89477FF02C02A
:10F75E000EDF689497FF0BC00024A095B09580959E
:10F76E0090951196801D901D00F8039400FA08954F
:10F77E00ED91FC9111970895ED91FD916D917C9114
:10F78E0013970895ED93FD936D937C9308950590D3
:10F79E00F491E02D08957A936A93FA93EA9308957B
:10F7AE00689401C0E89401D09DD0182E862F612D4B
:10F7BE00192E972F712D1B2EBF2FF12D1A2EAE2F16
:10F7CE00E12D0895119602D0FE2F1197E199FECFEB
:10F7DE00FF93FFB7F894AEBBBFBBE09AEDB3FFBF8C
:10F7EE00FF91089507D01196EF93EF2F03D0EF916D
:10F7FE0011970895E19B02C0A895FCCF9FB7F8948E
:10F80E00AEBBBFBBE09A8DB3E81719F0EDBBE29A21
:10F81E00E19A9FBF0895552342F4503811F4E0FF4A
:10F82E0004C03196691F791F6BF050E8572711F409
:10F83E005F93CDC05F3F31F0660F000C5795679513
:10F84E00752F08955F9300200AF0CDC0C6C050E812
:10F85E00192E1522880F991F9527550F879550E859
:10F86E00072E0522660F771F7527550F679508958A
:10F87E00689401C0E8945F93F2DF703818F07F3F10
:10F88E0008F4A5C056E1571BAAF4519558300EF452
:10F89E00593030F0EFEFFFEF6FEF7FE777F91AC0D7
:10F8AE0077275523B9F0EE0FFF1F661F771F5A9566
:10F8BE00D1F710C07727583028F0EF2FF62F672F8B
:10F8CE005850F9CF552331F076956795F795E79512
:10F8DE005A95D1F700200AF44ADE5F910895689494
:10F8EE0001C0E894309760407040B1F0002426F0DB
:10F8FE00772312F400943BDE172E7EE1112032F0B6
:10F90E007A95EE0FFF1F661F111CF9CFEF2FF62F02
:10F91E00612D5F938ADF5F9108954F93AF01FD01D3
:10F92E00DA01AB01BC01CA01402D012C142E4F91FE
:10F93E000895EA0FFB1F681F0895E095F0956095F6
:10F94E00EF5FFF4F6F4F08955F9381DF903871F136
:10F95E0050E8152604C05F937ADF903839F170387D
:10F96E0021F1572F591B13F112F4D7DFFACF58316B
:10F97E0018F0AA27BB278827583028F0AB2FB82FAE
:10F98E0088275850F9CF552329F08695B795A79516
:10F99E005A95D9F7502D512562F0CBDF38F4679583
:10F9AE00F795E795739513F41EC0B7DF3EDF5F91B1
:10F9BE000895EA1BFB0B680B51F010F40094BDDFA9
:10F9CE006623A2F3EE0FFF1F661F7A95CBF7EE2785
:10F9DE00FF27662777275F910895EFEFFFEF6FE719
:10F9EE007FEF5F910895EFEFFFEF6FE77FE75F9196
:10F9FE0008955F932CDF703851F3903841F3012452
:10FA0E000894791F23F41CF300203AF3ECCF0F92E5
:10FA1E001F932F933F934F93112722279927689F68
:10FA2E00A0018F9F302D410D591F6B9F300D411D31
:10FA3E00591F8E9F27D0BF9F25D06A9F23D0BE9F70
:10FA4E001DD0AF9F1BD0AE9F110D291F391F491F0F
:10FA5E00591FE32FF42F652F522F4F913F912F9166
:10FA6E001F910F9066232AF0550FEE1FFF1F661F82
:10FA7E0002C073954BF2CFDE5F910895100D211DDC
:10FA8E00391F02C0200D311D491F591F08955F9364
:10FA9E00DEDE703821F411200AF49FCFA4CF903807
:10FAAE0009F495CF01240894970B1BF4D4F300208E
:10FABE00F3CF792F1F932F933F934F931124112739
:10FACE00222733274427552790E2AE17BF07860714
:10FADE00410730F0AE1BBF0B860B410B089401C0E3
:10FAEE008894551F221F331F111CAA1FBB1F881F6E
:10FAFE00441F9A9551F7F901612D4F913F912F9126
:10FB0E001F91662332F0550FEE1FFF1F661F7A9569
:10FB1E0043F281DE5F910895309760407040089502
:10FB2E0000240A160B06089500240A160B06080672
:10FB3E00090608955A934A933A932A931A930A936D
:10FB4E0008955D814C813B812A8119810881089538
:00000001FF
